:100000000C94221A0C94531A0C94531A0C94531AED
:100010000C94531A0C94531A0C94531A0C94531AAC
:100020000C94531A0C94531A0C94531A0C94531A9C
:100030000C94531A0C94531A0C94531A0C94531A8C
:100040000C94531A0C94A4D10C94531A0C94531A74
:100050000C94531A0C94531A0C9477BA0C9417A658
:100060000C94531A0C9455520C944B520C94531AF2
:100070000C94531A0C94531A0C94531A0C94531A4C
:100080000C94531A0C94531A0C94531A0C94531A3C
:100090000C94531A0C94531A0C94531A0C94531A2C
:1000A0000C94531A0C94531A0C94531A0C94531A1C
:1000B0000C94531A0C94531A0C94531A0C94531A0C
:1000C0000C94531A0C94531A0C94531A0C941C3419
:1000D0000C94E6330C94531A0C94531A0C94531A40
:1000E0000C94531A084AD73B3BCE016E84BCBFFD2B
:1000F000C12F3D6C74319ABD56833DDA3D00C77FF8
:1001000011BED9E4BB4C3E916BAAAABE0000008090
:100110003F05A84CCDB2D44EB93836A9020C50B91F
:10012000918688083CA6AAAA2ABE000000803F004B
:100130000C94F3520C94B6340C94AE340D948F0896
:100140000C9418F70C94CF9E0C9449A30C94ED3E9C
:100150000D9465040C9457F90C94F7520C94F7FF26
:100160000C948EA20D9490030C9408410C9411539E
:100170000C94A99E0C9484A20D9428050C94B39E13
:100180000C94CD340C94A2A20C94529F0D949F0811
:100190000C94C2340C94B2340C94D3FB0C9475417F
:1001A0000C9451A20C94E0340C942CF90C949834D7
:1001B0000C949F9E0C94403F0C9454FD0D94EC02C3
:1001C0000C94B79E0C9419530C94BA340C945A3472
:1001D0000C94989E0C94C59E0C94AF9E0C949352D4
:1001E0000D948C010C9498A20C94E0520C94C19E36
:1001F0000C94C5A30C94BE340C94E3A20C94EF525F
:100200000D94C0010C94C5A20C94D8340D94220313
:100210000D9492070C94FB520C94949E0C9456A24D
:100220000C942AA50C94D9A20D9478040C94A59E44
:100230000D945C020C947E9E0C94C2FA0C94BD9EAC
:100240000D94390C0C9442F80C946AA20D94B307E7
:100250000C94A7340C94799E0C94B1A20C9449A2EE
:100260000C94D59F0C94FDA40D943D010C94D49F47
:100270000D9423040C947CA20D94B9030C94FF52AA
:100280000D94CD030D9470010D9432070C9474A25B
:100290000D9459070C94CFA20D947A070D9462091E
:1002A0000C94D1520C94EB520D949F190C94EBA426
:1002B0000D9462070D9404040C94909E0C9466A314
:1002C0000C94C2520C949C9E0C94CB9E0D945F0790
:1002D0000C9434410C940EA40C9460A20D948119DA
:1002E0000C9489340D94A6070C9406530C94E75291
:1002F0000D94F0030C94AD410C946DA40C943C3F10
:100300000C9452A40C94BBA20C94C6340D94880790
:100310000C944DA54E414E494E495459494E46CD37
:10032000CCCC3D0AD7233C17B7D13877CC2B3295AC
:1003300095E6241FB14F0A000020410000C842008A
:10034000401C4620BCBE4CCA1B0E5AAEC59D740054
:10035000407A10F35A00A0724E18090010A5D4E894
:100360000000E87648170000E40B54020000CA9A27
:100370003B000000E1F50500008096980000004079
:10038000420F000000A086010000001027000000BE
:1003900000E803000000006400000000000A000004
:1003A0000000000100000000002C76D888DC674FB8
:1003B0000823DFC1DFAE59E1B1B796E5E3E453C6E8
:1003C0003AE651997696E8E6C28426EB898C9B62E0
:1003D000ED407C6FFCEFBC9C9F40F2BAA56FA5F48A
:1003E00090055A2AF75C936B6CF9676DC11BFCE0B2
:1003F000E40D47FEF520E6B500D0ED902E03009405
:100400003577050080841E080000204E0A00000099
:10041000C80C333333330F986E12831141EF8D21A3
:1004200014893BE65516CFFEE6DB18D1844B381B0A
:10043000F77C1D901DA4BBE424203284725E2281CF
:1004400000C9F124ECA1E53D27434F4D4D554E49E0
:10045000434154494F4E0044525952554E00455263
:10046000524F525300494E464F004543484F0045B6
:1004700072726F722077726974696E6720746F2070
:10048000454550524F4D210A0053544F505045445A
:100490002E20005072696E7465722073746F7070D4
:1004A00065642064756520746F206572726F727365
:1004B0002E2046697820746865206572726F7220FC
:1004C000616E6420757365204D39393920746F2051
:1004D000726573746172742E202854656D70657234
:1004E00061747572652069732072657365742E205E
:1004F0005365742069742061667465722072657337
:1005000074617274696E67290A004E6F20436865D2
:10051000636B73756D2077697468206C696E6520F4
:100520006E756D6265722C204C617374204C696E1F
:10053000653A20004E6F20436865636B73756D20CC
:1005400077697468206C696E65206E756D6265727E
:100550002C204C617374204C696E653A20006368EE
:1005600065636B73756D206D69736D617463682C61
:10057000204C617374204C696E653A20004C696EA2
:1005800065204E756D626572206973206E6F7420F0
:100590004C617374204C696E65204E756D62657296
:1005A0002B312C204C617374204C696E653A20000D
:1005B0004D3131300053657269616C207374617420
:1005C0007573206D69736D617463680A0077616982
:1005D000740A0053442072656164206572726F7200
:1005E0000A002121204B494C4C20636175736564DE
:1005F00020627920746F6F206D75636820696E6169
:1006000063746976652074696D65202D2063757249
:1006100072656E7420636F6D6D616E643A20004880
:100620006F74656E642049646C652054696D656FF4
:10063000757400486F74656E642049646C6520545D
:10064000696D656F75740A003D3D6F6E46696C613A
:100650006D656E7452756E6F75743D3D0070617599
:100660007365004D363030002066696C616D656ED3
:10067000745F72756E6F7574200066696C616D656C
:100680006E745F72756E6F757420540046696C618C
:100690006D656E7452756E6F75742054002A2A2A27
:1006A000496E6974696E67206361726420697320A2
:1006B0004F4B2A2A2A004D6564696120496E736593
:1006C00072746564004D656469612052656D6F7672
:1006D0006564004D313030305300627573793A20D3
:1006E00070617573656420666F7220696E707574D1
:1006F0000A00627573793A207061757365642066CB
:100700006F7220757365720A00627573793A207092
:10071000726F63657373696E670A002A2A2A6B69B0
:100720006C6C2A2A2A00706F7765726F6666004BC0
:10073000494C4C45442E20005072696E74657220FD
:1007400068616C7465642E206B696C6C2829206369
:10075000616C6C6564210A006563686F3A004572DC
:10076000726F723A0042696C696E656172204C6505
:1007700076656C696E6720477269643A0A002F2FAC
:10078000616374696F6E3A0070726F6D70745F00B0
:10079000656E640053656E64204D31303820746F8F
:1007A00020726573756D650A00496E7365727420F9
:1007B00066696C616D656E7420616E642073656E30
:1007C00064204D3130380A005265686561742066D6
:1007D000696E69736865642E00526568656174208E
:1007E000446F6E6500526568656174696E672E2E90
:1007F0002E005265686561740048656174657220F9
:1008000054696D656F75740053656E64204D3130A9
:100810003820746F2068656174206E6F7A7A6C6519
:100820000A004E6F7A7A6C65205061726B656400C5
:10083000486F74656E6420746F6F20636F6C640A18
:10084000007061757365640050617573650044697B
:100850007361626C6552756E6F7574005075726766
:10086000654D6F7265005061757365640073686FE4
:100870007700627574746F6E00626567696E004C14
:100880006F61642046696C616D656E74004C6F61C8
:10089000642046696C616D656E74205400496E7306
:1008A0006572742066696C616D656E7420616E643A
:1008B0002073656E64204D3130380A00726573759F
:1008C0006D656400526573756D696E670057616987
:1008D00074696E6720666F72206865617475702E2A
:1008E0000A004C656176696E6720473236003F53D7
:1008F000706563696669656420582C5920636F6F61
:100900007264696E617465206F7574206F66206211
:100910006F756E64732E0A003F28522965706561F9
:10092000742076616C7565206E6F7420706C6175D3
:100930007369626C653B206D75737420626520611C
:1009400074206C6561737420312E0A003F2852298F
:100950006570656174206D757374206265207370B5
:1009600065636966696564207768656E206E6F747B
:10097000207573696E6720616E204C43442E0A0017
:100980003F537065636966696564206E6F7A7A6C3F
:10099000652074656D7065726174757265206E6F27
:1009A0007420706C61757369626C652E0A003F5328
:1009B00070656369666965642066696C616D656E02
:1009C000742073697A65206E6F7420706C61757322
:1009D00069626C652E0A003F5370656369666965DC
:1009E00064207072696D65206C656E677468206E36
:1009F0006F7420706C61757369626C652E0A003FBC
:100A00005072696D65206C656E677468206D7573D2
:100A10007420626520737065636966696564207718
:100A200068656E206E6F74207573696E6720616EE5
:100A3000204C43442E0A003F537065636966696524
:100A400064206E6F7A7A6C652073697A65206E6FA8
:100A50007420706C61757369626C652E0A003F5278
:100A6000657472616374696F6E204D756C74697022
:100A70006C696572206D7573742062652073706592
:100A80006369666965642E0A003F53706563696631
:100A90006965642052657472616374696F6E204D7C
:100AA000756C7469706C696572206E6F7420706CFF
:100AB00061757369626C652E0A003F5370656369E6
:100AC00066696564206C617965722068656967682C
:100AD00074206E6F7420706C61757369626C652E22
:100AE0000A0043292E0A003F5370656369666965F1
:100AF00064206265642074656D70657261747572DE
:100B000065206E6F7420706C61757369626C65200E
:100B10002834302D00473236207374617274696E48
:100B2000672E2E2E0A004F46460A00466164652055
:100B30004865696768742000426564204C65766585
:100B40006C696E6720004661696C656420746F2073
:100B5000656E61626C6520426564204C6576656CEB
:100B6000696E670A00496E76616C6964206D657311
:100B7000682E0A0050726F62696E6720506F696E4E
:100B8000740025532025692F2569002E0A002F00A7
:100B900050726F62696E67206D65736820706F694F
:100BA0006E742000202844525952554E2900473275
:100BB00039204175746F20426564204C6576656C00
:100BC000696E67003F20284C2C522C462C4229206D
:100BD0006F7574206F6620626F756E64732E0A00E5
:100BE0003F2856296572626F7365206C6576656C67
:100BF00020696D706C61757369626C652028302D99
:100C000034292E0A00426164205A2076616C756591
:100C10000A004E6F2062696C696E656172206772AE
:100C200069640A00446576696174696F6E002553D2
:100C30003A2025730046696E6973686564210A006D
:100C40003A207A3A2000206F662000476F696E676D
:100C500020746F3A20580043570A00206469723AA2
:100C60000020616E676C653A005374617274207283
:100C700061646975733A004D343820506F696E7441
:100C80000025533A2025642F256400506F73697442
:100C9000696F6E696E67207468652070726F626537
:100CA0002E2E2E0A003F4C656773206F66206D6FF5
:100CB00076656D656E7420696D706C6175736962BF
:100CC0006C652028302D3135292E0A003F20285808
:100CD0002C5929206F7574206F6620626F756E64C1
:100CE000732E0A0050726F6265206F7574206F66F4
:100CF00020626F756E6473003F53616D706C652088
:100D000073697A65206E6F7420706C6175736962A7
:100D10006C652028342D3530292E0A004D343820BA
:100D20005A2D50726F626520526570656174616200
:100D3000696C69747920546573740A003F285629D8
:100D40006572626F7365206C6576656C20696D7085
:100D50006C61757369626C652028302D34292E0A08
:100D6000005374616E6461726420446576696174D5
:100D7000696F6E3A20002052616E67653A2000204C
:100D80004D61783A2000204D696E3A200020536969
:100D9000676D613A20004D65616E3A2000574152FF
:100DA0004E494E4721204C6F77205A204A65726B7E
:100DB000206D6179206C65616420746F20756E7799
:100DC000616E746564207061757365732E0A004FDF
:100DD0004646004F4E0020204D61783A200020000A
:100DE00020204D696E3A2000536F667420656E6452
:100DF00073746F70733A20003D3D4F6E506F77658E
:100E0000724C6F7373526573756D653D3D004D3265
:100E1000342053256C642054256C64004739322EED
:100E20003920452573004731204625640047393273
:100E30002E39205A2573004731205A30204632304F
:100E40003000473120582573205925732046333010
:100E50003030004D34323020532569205A2573003C
:100E60004D3130362050256920532569004D3230F0
:100E700030204425730047323852305859004739E2
:100E8000322E39204530205A300A47315A25730016
:100E90004D31303920532569004D313930205325EB
:100EA00069004D343230205330205A300020496ED2
:100EB00076616C696420657874727564657220006F
:100EC00047322F47332062616420706172616D6523
:100ED000746572730A00536C6565702E2E2E005A6D
:100EE0002050726F62652050617374204265640AFD
:100EF000005A2050726F6265205061737420426501
:100F000064004732384C30004D3131372050726F19
:100F10006265206661696C65642E0A4732380A0092
:100F200070726F62655F726577697065004732390C
:100F3000205265747279696E670050726F62696ED3
:100F400067204661696C6564004D31313720426528
:100F500064206C6576656C696E67206661696C6596
:100F6000642E0A4730205A31300A4D333030205039
:100F7000323520533838300A4D3330302050353038
:100F80002053300A4D33303020503235205338381A
:100F9000300A4D333030205035302053300A4D3335
:100FA00030302050323520533838300A4D3330300D
:100FB000205035302053300A4734205331007072AE
:100FC0006F62655F6661696C6564004D3131372021
:100FD000426564206C6576656C696E6720646F6E2F
:100FE000652E00205A3A200020593A2000426564BC
:100FF00020583A20004D65736820706F696E742028
:101000006F7574206F662072616E67650A004D30DF
:101010002053746F70004D312053746F7000436F14
:101020006E74696E756500436C69636B20746F2024
:10103000526573756D652E2E2E004E6F204D6F76A6
:10104000652E00456E642066696C65206C6973745A
:101050000A00426567696E2066696C65206C697379
:10106000740A004E6F206D656469610A00526573F1
:10107000756D696E6720534400286E6F2066696C39
:1010800065290043757272656E742066696C653AF5
:1010900020005072696E742074696D653A20000AF0
:1010A00053746174733A2046696C616D656E742087
:1010B000757365643A20002C204C6F6E67657374FD
:1010C000206A6F623A2000546F74616C2074696DFD
:1010D000653A200053746174733A20002C204661F5
:1010E000696C65643A20002C2046696E69736865F6
:1010F000643A20005072696E74733A200053746130
:1011000074733A2000436F6F6C696E672E2E2E0049
:1011100048656174696E672E2E2E004520255300A8
:101120006F6B006F6666006A0465045E04570449CD
:101130000444454255473A004D3131332053004273
:10114000656420436F6F6C696E672E2E2E004265BA
:10115000642048656174696E672E2E2E00544D33ED
:1011600044203130532050726F204F46462E002FBE
:101170002F00205200416363656C65726174696F72
:101180006E3A2050004D32303620580046523A0018
:1011900020466C6F773A200020643A0020693A00BC
:1011A00020703A00496E76616C69642065787472CB
:1011B000756465720A0020643A0020693A00207064
:1011C0003A0064697300656E0043290A0061626C2D
:1011D000656420286D696E2074656D702000436F12
:1011E0006C64206578747275646573206172652023
:1011F00000504944204175746F74756E6500504904
:1012000044204175746F74756E65206661696C6504
:10121000642120426164206865617465722069649C
:101220000A0046696C616D656E742072756E6F752B
:10123000742064697374616E636520286D6D293A4A
:10124000200046696C616D656E742072756E6F75F5
:101250007420004D34323120696E636F72726563A1
:101260007420706172616D65746572207573616759
:10127000650A004D65736820706F696E74206F7524
:1012800074206F662072616E67650A004F66667330
:10129000657473204170706C696564004572723AC0
:1012A00020546F6F206661722100546F6F20666159
:1012B000722066726F6D207265666572656E636519
:1012C00020706F696E740A00454550524F4D204F93
:1012D0004B0A00506F7765722D6C6F7373207265C7
:1012E000636F7665727920004D383400446F6E6507
:1012F000207072696E74696E672066696C650A0099
:101300004D3737004D3331004361703A004D454150
:10131000545041434B00434F4F4C45525F54454D51
:101320005045524154555245004348414D42455263
:101330005F54454D5045524154555245004241423B
:10134000595354455050494E470041524353004D64
:101350004F54494F4E5F4D4F4445530054484552FA
:101360004D414C5F50524F54454354494F4E004CF1
:101370004F4E475F46494C454E414D4500415554FF
:101380004F5245504F52545F53445F53544154554C
:10139000530053445F57524954450052455045410C
:1013A00054005344434152440050524F4D50545FF7
:1013B000535550504F525400454D455247454E43AA
:1013C000595F50415253455200434153455F4C4988
:1013D0004748545F4252494748544E45535300547E
:1013E0004F47474C455F4C494748545300534F467D
:1013F00054574152455F504F574552004255494C52
:10140000445F50455243454E54004C4556454C4967
:101410004E475F44415441005A5F50524F4245008D
:1014200052554E4F5554004155544F4C4556454C1E
:10143000005052494E545F4A4F420050524F47525B
:10144000455353004155544F5245504F52545F54E9
:10145000454D5000564F4C554D455452494300455B
:101460004550524F4D0042494E4152595F46494CFA
:10147000455F5452414E53464552005345524941EF
:101480004C5F584F4E5F584F4646004649524D57A5
:101490004152455F4E414D453A4D61726C696E2037
:1014A000322E302E375F4457372E332E3120544D95
:1014B00033442053534D444E422028417072203211
:1014C0003920323032312031333A34333A33302913
:1014D00020534F555243455F434F44455F55524C4F
:1014E0003A68747470733A2F2F6769746875622E46
:1014F000636F6D2F496E73616E6974794175746F96
:101500006D6174696F6E2F4D61726C696E2F7472AC
:1015100065652F437265616C6974794477696E5FA4
:10152000322E302050524F544F434F4C5F5645524D
:1015300053494F4E3A312E30204D414348494E4594
:101540005F545950453A544D334420313053205064
:10155000726F2045585452554445525F434F554E83
:10156000543A3120555549443A63656465326132D5
:10157000662D343161322D343734382D39623132B1
:101580002D6335356336326633363766660A00506A
:10159000726F6265204F6666736574205A005072E0
:1015A0006F6265204F6666736574205A00290A00D1
:1015B00020746F20003F5A206F7574206F66207270
:1015C000616E6765202800290A0020746F20003FA3
:1015D00059206F7574206F662072616E67652028D0
:1015E0002D00290A0020746F20003F58206F757469
:1015F000206F662072616E676520282D0050726F23
:101600006265204F666673657420580043616E6E94
:101610006F74206F70656E2073756264697220004C
:101620002569730025696D20256973002569682087
:1016300025696D2025697300256964202569682066
:1016400025696D2025697300256979202569642045
:101650002569682025696D20256973003D3D447723
:10166000696E20496E697420436F6D706C65746596
:101670003D3D002A2A2A4E6F7A7A6C6554656D705A
:101680005374617475735B325D203D003D3D486568
:101690006174696E6720446F6E65204368616E6790
:1016A000652046696C616D656E743D3D0020207358
:1016B0007461727470726F677265737320003D3D60
:1016C0007761697477617920353D3D003D3D7761F3
:1016D000697477617920343D3D003D3D77616974DF
:1016E00077617920333D3D003D3D776169747761D5
:1016F0007920313D3D003D3D6F6E5072696E7454EE
:10170000696D657253746F707065643D3D003D3D59
:101710006F6E466163746F727952657365743D3D97
:1017200000270A0A0000272027002027002D006E2E
:101730006F74696669636174696F6E200063616EBE
:1017400063656C005072696E742041626F727465DB
:1017500064004469736D6973730055492041626F79
:101760007274656400726573756D65004D32340086
:101770002A2A2A43506C617920546F6E652A2A2ADE
:10178000003D3D6F6E5072696E7454696D657250A4
:1017900061757365643D3D00486F6D696E672046F5
:1017A00061696C6564006F70656E0054524947470B
:1017B00045524544003A200066696C616D656E745F
:1017C000007A5F6D696E00795F6D696E00785F6D9C
:1017D000696E005265706F7274696E6720656E6421
:1017E00073746F70207374617475730A0020746F62
:1017F0006F206C6F6E6720657874727573696F6E99
:101800002070726576656E7465640A0020636F6C83
:101810006420657874727573696F6E207072657676
:10182000656E7465640A00486F6D652025732573C5
:101830002573204669727374005761726E696E6712
:101840003A20486F6D696E672042756D702044695B
:101850007669736F72203C20310A00020204000096
:101860000000000000000000000000809D43000018
:101870009B430000C84300000041000000410000FD
:1018800000400000000100000001000080005555EC
:1018900055000000400033333300AAAA2A004992C1
:1018A000240000002000C7711C0099991900D1453F
:1018B0001700555515003BB11300244912001111B2
:1018C0001100000010000F0F0F00E3380E004379E5
:1018D0000D00CCCC0C00C3300C00E8A20B0064213E
:1018E0000B00AAAA0A00703D0A009DD80900427B9D
:1018F000090092240900DCD30800888808001042FF
:10190000080000000800F0C1070087870700755035
:101910000700711C07003EEB0600A1BC06006990A1
:10192000060066660600703E06006118060017F4A1
:10193000050074D105005BB00500B290050062722D
:1019400005005555050078390500B81E0500050548
:1019500005004EEC040087D40400A1BD040090A74C
:10196000040049920400C17D0400EE690400C756DA
:101970000400444404005C320400082104004110C7
:101980000400000004003FF00300F8E0030026D24A
:101990000300C3C30300CCB503003AA803000A9BAD
:1019A0000300388E0300C08103009F750300D069D7
:1019B0000300505E03001D53030034480300913DB3
:1019C00003003333030016290300381F0300971563
:1019D0000300300C0300030303000BFA020049F17B
:1019E0000200BAE802005CE002002DD802002DD00F
:1019F000020059C80200B0C0020031B90200DAB1D9
:101A00000200AAAA0200A0A30200BC9C0200FA9550
:101A100002005C8F0200DF88020082820200457CA7
:101A200002002776020027700200436A02007C64ED
:101A30000200D05E02003F590200C8530200FFFDC1
:101A4000FCFAF8F6F4F2F0EEECEAE9E7E5E3E1E0BF
:101A5000DEDCDAD9D7D5D4D2D0CFCDCBCAC8C7C572
:101A6000C3C2C0BFBDBCBAB9B7B6B4B3B2B0AFADF4
:101A7000ACAAA9A8A6A5A4A2A1A09E9D9C9A99984B
:101A80009795949392908F8E8D8B8A898887868480
:101A9000838281807F7E7D7B7A7978777675747397
:101AA0007271706F6E6D6C6B6A696867666564638E
:101AB0006261605F5E5D5C5B5A5958585756555479
:101AC00053525150504F4E4D4C4B4A4A494847464D
:101AD00046454443424241403F3E3E3D3C3B3B3A0B
:101AE00039383837363535343332323130302F2EBD
:101AF0002E2D2C2B2B2A2929282727262525242360
:101B00002322212120201F1E1E1D1C1C1B1B1A19F5
:101B1000191818171616151514131312121111107F
:101B20000F0F0E0E0D0D0C0C0B0A0A090908080701
:101B300007060605050404030302020100003D3DFB
:101B40006F6E5072696E7454696D65725374617210
:101B50007465643D3D0000809D4300009B43000090
:101B6000C8430000000000000000000000003D3DF0
:101B70006F6E53746F726553657474696E67733DED
:101B80003D003D3D6F6E436F6E66696775726174AF
:101B9000696F6E53746F72655772697474656E3DC8
:101BA0003D0053657474696E67732053746F72657A
:101BB00064000A20696E6974207A70726F62655FD2
:101BC0007A6F6666736574203D20003D3D6F6E43FD
:101BD0006F6E66696775726174696F6E53746F7248
:101BE00065526561643D3D00454550524F4D204969
:101BF0006E697469616C697A65640A003B20003A19
:101C00000A0020204D363033200020440020204D93
:101C100034313220530046696C616D656E742072F8
:101C2000756E6F75742073656E736F723A00205510
:101C3000004C0046696C616D656E74206C6F616468
:101C40002F756E6C6F6164206C656E677468733A93
:101C50000020204D3835312058005A2D50726F62C7
:101C600065204F66667365740020204D3431332043
:101C70005300506F7765722D4C6F737320526563FC
:101C80006F766572793A0020440020490020204D8B
:101C900033303420500020440020490020204D33B0
:101CA00030312050005049442073657474696E6768
:101CB000733A00204A00202047323920572049003B
:101CC00020204D3432302053004175746F2042651E
:101CD00064204C6576656C696E673A0020204D3251
:101CE0003036205800486F6D65206F6666736574E6
:101CF0003A0020580020530020204D323035204239
:101D000000416476616E6365643A20423C6D696EA1
:101D10005F7365676D656E745F74696D655F75731C
:101D20003E20533C6D696E5F6665656472617465E3
:101D30003E20543C6D696E5F74726176656C5F66BF
:101D4000656564726174653E20583C6D61785F78AA
:101D50005F6A65726B3E20593C6D61785F795F6A9E
:101D600065726B3E205A3C6D61785F7A5F6A65727E
:101D70006B3E20453C6D61785F655F6A65726B3EC6
:101D80000020540020520020204D323034205000DA
:101D9000416363656C65726174696F6E2028756E4E
:101DA0006974732F7332293A20503C7072696E74D3
:101DB0005F616363656C3E20523C7265747261635F
:101DC000745F616363656C3E20543C747261766538
:101DD0006C5F616363656C3E0020204D32303120C2
:101DE00058004D6178696D756D20416363656C6560
:101DF000726174696F6E2028756E6974732F733207
:101E0000293A0020204D3230332058004D61786946
:101E10006D756D20666565647261746573202875E3
:101E20006E6974732F73293A005374657073207050
:101E3000657220756E69743A0020440020204D328E
:101E400030302053002044697361626C65640A007D
:101E500046696C616D656E742073657474696E6734
:101E6000733A0020286D6D29002020473231202050
:101E700020203B20556E69747320696E206D6D00C3
:101E80003D3D6F6E4C6F616453657474696E67732A
:101E90003D3D000000FA430000FA430000204100ED
:101EA000008C420000A0420000A0420000C8430095
:101EB000000C43EE020000EE020000640000003C53
:101EC00000000024F4D43050C38E20C2A2401782F8
:101ED0008B7011127A910D816CD90AA861E108C743
:101EE000586607615143061E4B5D05C145A7041A9C
:101EF000411104093D9803713931034036DB026515
:101F0000339102D4305402802E1D02632CEE0175F1
:101F10002AC501B028A001102781018F2564012B5B
:101F2000244B01E0223401AC211F018D200D0180E2
:101F30001FFC00841EED00971DDF00B81CD200E6D8
:101F40001BC600201BBC00641AB200B219A8000A0C
:101F500019A0006A189900D117910040178B00B59D
:101F600016840031167E00B31579003A157300C748
:101F7000146F0058146A00EE13660088136300257E
:101F8000135E00C7125B006C12570015125400C19B
:101F900011510070114F0021114B00D61049008DD6
:101FA0001047004610440002104200C00F4000805D
:101FB0000F3E00420F3C00060F3B00CB0E38009353
:101FC0000E37005C0E3500270E3400F30D3200C1D1
:101FD0000D3100900D3000600D2E00320D2D0005EA
:101FE0000D2C00D90C2B00AE0C2900850C29005CAF
:101FF0000C2700350C27000E0C2600E80B2400C42B
:102000000B2400A00B23007D0B23005A0B21003969
:102010000B2100180B2000F80A1F00D90A1E00BB74
:102020000A1E009D0A1D00800A1D00630A1C00474D
:102030000A1B002C0A1B00110A1A00F7091A00DDFE
:10204000091900C4091900AB091900920917007B8E
:10205000091800630917004C0916003609160020FC
:102060000916000A091500F5081500E0081400CC4F
:10207000081400B8081400A4081400900813007D88
:102080000812006B081300580812004608120034AA
:10209000081100230811001208110001081100F0B6
:1020A000071000E0071000D0071000C0071000B0B4
:1020B000070F00A107100091070E0083070F00749F
:1020C000070F0065070E0057070E0049070E003B7B
:1020D000070D002E070E0020070D0013070D000648
:1020E000070D00F9060C00ED060D00E0060C00D40B
:1020F000060C00C8060C00BC060C00B0060C00A4C0
:10210000060B0099060C008D060B0082060B00776B
:10211000060B006C060B0061060A0057060B004C0C
:10212000060A0042060A0038060A002E060A0024A3
:10213000060A001A060A001006090007060A00FD32
:10214000050900F4050900EB050900E2050900D9BD
:10215000050900D0050900C7050900BE050900B53D
:10216000050800AD050800A50509009C05080094B8
:102170000508008C050800840508007C050800742B
:102180000508006C050700650508005D0507005699
:102190000508004E05070047050700400508003800
:1021A000050700310507002A050700230507001C65
:1021B000050600160507000F0507000805060002C2
:1021C000050700FB040600F5040700EE040600E81E
:1021D000040600E2040700DB040600D5040600CF75
:1021E000040600C9040600C3040600BD040600B7C7
:1021F000040600B1040500AC040600A6040600A015
:102200000405009B04060095040500900406008A5E
:1022100004050085040500800406007A04050075A5
:10222000040500700405006B0405006604050061E8
:102230000405005C04050057040500520405004D28
:1022400004050048040500430405003E0404003A68
:1022500004050035040500300404002C04050027A3
:10226000040400230405001E0404001A04040016DC
:10227000040500110404000D040400090405000411
:1022800004040000040400FC030400F8030400F448
:10229000030400F0030400EC030400E8030400E47A
:1022A000030400E0030400DC030400D8030400D4AA
:1022B000030400D0030400CC030400C8030300C5DA
:1022C00003030024F404D9201BC40C5C0E9804C43E
:1022D000095F0265077101F405F900FB04B30048CA
:1022E000048700C10369005803550003034500BE7D
:1022F000023A008402310053022A00290225000418
:10230000022000E4011C00C8011900AF0117009869
:1023100001140084011300710110006101100051CB
:10232000010E0043010D0036010B002B010B0020B4
:10233000010B00150109000C01090003010800FB55
:10234000000800F3000800EB000700E4000600DED0
:10235000000600D8000600D2000600CC000500C729
:10236000000500C2000500BD000400B9000400B56E
:10237000000400B1000400AD000400A9000400A5A1
:10238000000300A20003009F0004009B00030098CC
:102390000003009500020093000300900003008DED
:1023A0000002008B00030088000200860002008407
:1023B000000300810002007F0002007D0002007B1C
:1023C000000200790002007700010076000200742C
:1023D00000020072000100710002006F0002006D37
:1023E0000001006C0002006A000100690002006741
:1023F0000001006600010065000100640002006247
:1024000000010061000100600001005F0002005D4A
:102410000001005C0001005B0001005A000100594E
:10242000000100580001005700010056000100554E
:10243000000100540001005300000053000100524D
:1024400000010051000100500001004F0001004E4A
:102450000000004E0001004D0001004C0001004B47
:102460000000004B0001004A000100490001004843
:10247000000000480001004700010046000000463F
:102480000001004500000045000100440001004338
:102490000000004300010042000000420001004132
:1024A00000000041000100400001003F0000003F2B
:1024B0000001003E0000003E0001003D0000003D24
:1024C0000001003C0000003C0000003C0001003B1B
:1024D0000000003B0001003A0000003A0001003912
:1024E000000000390001003800000038000000380A
:1024F0000001003700000037000100360000003600
:1025000000000036000100350000003500000035F5
:1025100000010034000000340000003400010033EA
:1025200000000033000000330001003200000032E0
:1025300000000032000100310000003100000031D5
:102540000001003000000030000000300001002FCA
:102550000000002F0000002F0000002F0001002EBF
:102560000000002E0000002E0001002D0000002DB4
:102570000000002D0000002D0001002C0000002CA8
:102580000000002C0000002C0001002B0000002B9C
:102590000000002B0000002B0001002A0000002A90
:1025A0000000002A0000002A000100290000002984
:1025B0000000002900000029000000290001002877
:1025C000000000280000002800000028000000286B
:1025D000000100270000002700000027000000275E
:1025E0000000002700010026000000260000002651
:1025F0000000002600000026000100250000002544
:102600000000002500000025000000250000002536
:102610000001002400000024000000240000002429
:10262000000000240001002300000023000000231C
:10263000000000230000002300000023000000230E
:102640000001002200000022000000220000002201
:1026500000000022000000220001002100000021F3
:1026600000000021000000210000002100000021E6
:1026700000000021000100200000002000000020D8
:1026800000000020000000200000002000000020CA
:10269000000000200001001F0000001F0000001FBC
:1026A0000000001F0000001F0000001F0000001FAE
:1026B0000001001E0000001E0000001E0000001EA1
:1026C000000000393000003325000087190000B0F9
:1026D0000F0000DB080000BD040000740200003F92
:1026E00001000020436F756E7420583A0023646522
:1026F00066696E652044454641554C545F00006252
:102700006564004B6420004B6920004B7020005032
:102710004944204175746F74756E652066696E69F1
:1027200073686564212050757420746865206C613D
:102730007374204B702C204B6920616E64204B64B5
:1027400020636F6E7374616E74732066726F6D2098
:1027500062656C6F7720696E746F20436F6E666977
:102760006775726174696F6E2E680A005049442063
:102770004175746F74756E65206661696C6564215E
:102780002074696D656F75740A0050494420417565
:10279000746F74756E65206661696C656421205480
:1027A000656D706572617475726520746F6F2068F5
:1027B0006967680A00204B643A2000204B693A2080
:1027C00000204B703A200020436C617373696320D2
:1027D000504944200A00204E6F206F76657273685E
:1027E0006F6F740A002054753A2000204B753A2010
:1027F00000206D61783A2000206D696E3A2000203B
:10280000643A200020626961733A200050494420F4
:102810004175746F74756E652073746172740A000B
:10282000504944204175746F74756E652066616906
:102830006C6564212054656D706572617475726594
:1028400020746F6F20686967680A004265640045FC
:102850003100626564002C2073797374656D207398
:10286000746F7070656421204865617465725F499A
:10287000443A200048656174696E67204661696C5E
:1028800065640048656174696E67206661696C659E
:1028900064004D3131322053687574646F776E0077
:1028A0001000C90210012C01400122017001180121
:1028B000B0010E01F00104015002FA00B002F00074
:1028C0003003E600D003DC009004D2007005C8009D
:1028D000A006BE000008B400B009AA00D00BA000FA
:1028E000600E960060118C0000158200201978009F
:1028F000C01D6E00A0226400B0275A00902C50002A
:1029000000314600E0343C0010383200903A280094
:10291000603C1E00A03D1400803E0A00203F0000E5
:10292000544845524D414C2052554E415741590053
:10293000546865726D616C2052756E6177617900C3
:102940004572723A204D415854454D50004D415802
:1029500054454D502074726967676572656400451F
:1029600072723A204D494E54454D50004D494E54D7
:10297000454D502074726967676572656400202F49
:10298000002042403A0020403A0020573A002057A9
:102990003A00496E76616C6964206578747275647A
:1029A00065720A007C3C3E5E2B3D3F2F5B5D3B2CFD
:1029B0002A225C0043616E6E6F74206F70656E201A
:1029C0007375626469722000534420496E697420F3
:1029D0004661696C0053442063617264206F6B0A26
:1029E000006F70656E526F6F74206661696C65640C
:1029F0000A00766F6C756D652E696E69742066616C
:102A0000696C65640A004E6F2053442063617264F0
:102A10000A000A4D3234004D3233202573002E0A4D
:102A2000006F70656E206661696C65642C20466974
:102A30006C653A200046696C652073656C6563744B
:102A400065640A002053697A653A200046696C651E
:102A5000206F70656E65643A2000454E44205355E2
:102A600042524F5554494E450A002220706F730060
:102A70002220706172656E743A2200535542524FA3
:102A80005554494E452043414C4C20746172676552
:102A9000743A220053756263616C6C204F766572E4
:102AA000666C6F77004578636565646564206D6169
:102AB0007820535542524F5554494E452064657015
:102AC00074683A002E0A0044656C6574696F6E2064
:102AD0006661696C65642C2046696C653A20004625
:102AE000696C652064656C657465643A00534420C4
:102AF0007072696E74696E67206279746520004E29
:102B00006F74205344207072696E74696E670A0096
:102B100057726974696E6720746F2066696C653AD4
:102B20002000667265736800646F696E67002066D6
:102B3000696C653A20004E6F7720002F6175746FC5
:102B400025632E67002020506C616E6E65724275A1
:102B50006666657242797465733A20002046726534
:102B600065204D656D6F72793A2000436F6D706915
:102B70006C65643A20417072203239203230323133
:102B80000A00204C61737420557064617465643A66
:102B900020323032312D30342D3138207C204175B7
:102BA00074686F723A2054696E794D616368696E1A
:102BB000657333440A00322E302E375F4457372E68
:102BC000332E310A004D61726C696E0020536F66BE
:102BD00074776172652052657365740A00205761CD
:102BE000746368646F672052657365740A002042DD
:102BF000726F776E206F75742052657365740A006A
:102C00002045787465726E616C2052657365740A34
:102C100000506F77657255700A0073746172740AA0
:102C2000004739310A47315A350A4739300A4D3899
:102C3000340A4D31303453300A4D31343053300082
:102C40004D31303031006572726F72207772697465
:102C5000696E6720746F2066696C650A00446F6E48
:102C60006520736176696E672066696C652E0A005F
:102C70004D323900456E6473746F707300255320B4
:102C8000256320256320256320256300205A3A0010
:102C900020593A0020583A00656E6473746F70735F
:102CA000206869743A200000000A0B02090C0D0E1E
:102CB00008070304010000000000000000000000FD
:102CC0000000000000000000000000000000000004
:102CD00000000012111000000000000000000000C1
:102CE0000000000000000000000000000070012C47
:102CF0000190012701B0012201C0011D01F001185E
:102D0000011002130130020E016002090190020459
:102D100001C002FF000003FA004003F5008003F049
:102D200000D003EB002004E6007004E100E004DCC6
:102D3000004005D700C005D2004006CD00D006C82F
:102D4000008007C3003008BE00F008B900C009B415
:102D500000B00AAF00B00BAA00D00CA500000EA076
:102D600000500F9B00C01096005012910000148C70
:102D700000C0158700B0178200B0197D00D01B7805
:102D800000001E730040206E0090226900F0246451
:102D90000040275F0090295A00E02B5500102E506C
:102DA0000020304B0010324600E033410090353CAB
:102DB000001037370070383200A0392D00B03A28A3
:102DC00000A03B2300603C1E00103D1900903D1404
:102DD00000103E0F00703E0A00C03E0500003F009C
:102DE00000403FFBFF803FF6FFC03FF1FFFFFFFFCA
:102DF00050726F62696E67204661696C656400207D
:102E00005A3A200020593A200042656420583A205E
:102E1000003D3D6F6E55736572436F6E6669726DEE
:102E200052657175697265643D3D00220A00556EF8
:102E30006B6E6F776E20636F6D6D616E643A2022EA
:102E4000002042002050006F6B00204500205A00F7
:102E5000205900204D393220580020453A00205A90
:102E60003A0020593A00583A0020746F6F206C6F76
:102E70006E6720657874727573696F6E2070726505
:102E800076656E7465640A0020636F6C64206578F3
:102E900074727573696F6E2070726576656E746595
:102EA000640A0043616E6E6F7420656E74657220F3
:102EB0007375626469723A20004D323520500A4DB4
:102EC000323400526573756D650055492050617547
:102ED0007365004E6F204D61746368203A004D3277
:102EE000320A4D3231005265667265736800506770
:102EF0005570005067446F776E0049732046696CC7
:102F00006520004973204469722000476F55704462
:102F1000697200486173204D656469610046696C9F
:102F2000656E616D652053656C6563746564004D05
:102F30003130303043004D313030300046696C6103
:102F40006D656E7420537461742030202D20330021
:102F500046696C616D656E74205374617420302015
:102F60002D20320046696C616D656E74205374616A
:102F7000742030202D2031002046696C616D656E13
:102F80007420526573706F6E7365204E6F005265CA
:102F900073756D652059657320647572696E67205D
:102FA0007072696E74000A204E6F2046696C616D04
:102FB000656E7400496E76616C6964204F70746947
:102FC0006F6E004D3530300053746F72652053655D
:102FD0007474696E677300426564205049442053DD
:102FE000746172746564004D3939390A4D32383074
:102FF00050305331363000424C546F756368205264
:1030000065736574004D3530320A4D3530300049F6
:103010006E697420454550524F4D00486F74656E7F
:103020006420504944205374617274656400456E95
:10303000676C69736820416C7265616479205365BF
:1030400074004368696E657365204E6F7420537514
:1030500070706F7274656400496E4C616E6743688E
:103060006F696365000A202A2A2A726563646174A5
:103070002E646174615B305D203D004732380A4741
:1030800031204631303030205A313000556E737562
:1030900070706F72746564204F7074696F6E205326
:1030A000656C6563746564004732365232353500AD
:1030B0004D3139305335350A4732380A4732390AEB
:1030C0004D3430300A4D313034533231350A4732C5
:1030D000380A4D313039533231350A4D343230539C
:1030E000310A47315831303059313030463530307F
:1030F000300A47315A300A4D3530300A4D313137B8
:1031000020536574205A204F6666736574004731FA
:10311000204631303030205A302E30004732380AC5
:103120004731204631303030205A302E30004D3576
:103130003030005A204F6666736574203A2025733C
:10314000004D353030005A204F6666736574203A62
:10315000202573004732380A473146313530305A1E
:10316000302E30004732385A0A4731463135303038
:103170005A302E30004D383400473146313030302F
:103180005A302E30004732380A473146313030301D
:103190005A302E30004D616E75616C536574546504
:1031A0006D7000526571756573746564204F666655
:1031B000736574204265796F6E64204C696D697423
:1031C00073005A204F6666736574203A2025730099
:1031D000526F756E64696E6720746F2073746570CA
:1031E00000526571756573746564204F666673651A
:1031F00074200053746F702054726967676572653C
:10320000640053746F70204E6F0053746F7050726F
:10321000696E740048616E646C652044617461205D
:1032200041646A75737420322053657474696E67E3
:103230002053637265656E200048616E646C652082
:1032400044617461205072696E7446696C65203304
:103250002053657474696E672053637265656E20D0
:103260000048616E646C652044617461205072692D
:103270006E7446696C6520322053657474696E679C
:103280002053637265656E20004D38340048616ECE
:10329000646C652044617461205072696E74466983
:1032A0006C6520506F73740048616E646C652044D7
:1032B000617461205072696E7446696C6520507249
:1032C0006500426567696E537769746368003D3DC8
:1032D00020436865636B6B65793D3D00726563648F
:1032E00061742E61646472203D3D007265636461A7
:1032F000742E646174615B305D203D3D00776169CF
:1033000074776179203D3D0020202A2A2A2A2A2A22
:103310002A5254535F48616E646C65446174612A3B
:103320002A2A2A2A2A2A2A2000526573656E643ABC
:10333000200000002200250028002B002E00310074
:10334000340002010000050108010B01000021000A
:10335000240027002A002D00300033000101000066
:10336000040107010A010505050507050808080805
:10337000020202020A0A080804040404010101010D
:103380000101010103030303030303030407070708
:103390000C0C0C0C0C0C0C0C0202020206060606AD
:1033A000060606060B0B0B0B0B0B0B0B010210207A
:1033B000200808102040102040800201020108046B
:1033C00002010102040810204080804020100804FF
:1033D0000201800402018040201008040201080458
:1033E000020101020408102040800102040810209C
:1033F0004080544D3344203130532050726F20525E
:10340000656164792E005072696E74696E672E2E44
:103410002E005072696E7420506175736564006E81
:103420006F74696669636174696F6E200050494406
:103430002054756E652046696E6973686564000086
:1034400054016E0111241FBECFEFD1E2DEBFCDBF0C
:1034500000E00CBF13E0A0E0B2E0E4EDF4E502E030
:103460000BBF02C007900D92A83FB107D9F725E125
:10347000A8EFB3E001C01D92A53DB207E1F71AE144
:10348000C1E2DAE100E006C021970109802FFE01C8
:103490000F949726C032D10780E00807A9F70F9450
:1034A000B5140D94582A0C9400009F92AF92BF92CD
:1034B000CF92DF92EF92FF920F931F93CF93DF9300
:1034C00000D01F921F92CDB7DEB7EEE3FAE10027DE
:1034D000BB27462F572FA82FAA2341F4A52F542FDF
:1034E000B85FAA2319F4A52F5527B85FA03138F487
:1034F0005295A295452F4F70507FA42BBC5FA034EE
:1035000028F4550FAA1F550FAA1FBE5FA03818F444
:10351000550FAA1FB395550FAA1FEA0FF01F44912C
:1035200051E0AA27B85081F1C8F0B0FF02C0440FA3
:10353000551FB1FF04C0440F551F440F551FB2FF64
:1035400006C052954295142F1F70407F512BB3FF38
:103550001BC0A52F542F44270C94C41AB195B0FF5B
:1035600002C055954795B1FF04C0559547955595AF
:103570004795B2FF05C05295407F4295452B5F703D
:10358000B3FF02C0452F5527DD24CC24BB24B2E075
:10359000649FD018C108B00AB00B749FC018B1085E
:1035A000B00B849FB018B109659FC018B108B00B6B
:1035B000759FB018B109859FB0196A9FB018B109FD
:1035C0007A9FB0194D9DA12C992433279927222742
:1035D0005D9DA00C911C301F901F201FAD9D900C75
:1035E000311D901F201F4C9DA00C911C301F901F5F
:1035F000201F5C9D900C311D901F201FAC9D300D35
:10360000911D201F4B9D900C311D901F201F5B9D15
:10361000300D911D201FAB9D900D211D4B9F300D36
:10362000911D201F5B9F900D211DAB9F200DB1E0D0
:10363000BB24CC24DD24639FD018C108B00AB00B92
:10364000739FC018B108B00B839FB018B109699F70
:10365000C018B108B00B799FB018B109899FB01993
:10366000629FB018B109729FB019D61AC70AB80A7A
:1036700020F0B1E03B0F901F201F1124792F632F02
:1036800090E0822F0F900F900F900F900F90DF918E
:10369000CF911F910F91FF90EF90DF90CF90BF904F
:1036A000AF909F900895AF92BF92CF92DF92EF922A
:1036B000FF920F931F93CF93DF93CBE2DCE00EEDED
:1036C00018E08BE3A82E8CE0B82EC12CD12C76010B
:1036D000C39469917991899199910F94E11F2889F7
:1036E00039894A895B890F9442200F941328F80185
:1036F00061937193819391938F01C616D706E80663
:10370000F90610F46B017C01AC16BD0611F76FEFE2
:103710007FEFCB01A70196010F9420262093EE089E
:103720003093EF084093F0085093F108DF91CF9168
:103730001F910F91FF90EF90DF90CF90BF90AF90CF
:103740000895CF92DF92EF92FF928091EA0788234B
:1037500009F457C0C090E607D090E707E090E8076B
:10376000F090E90720E030E0A901C701B6010F940D
:10377000DC1F882309F445C020E030E040E05FE32F
:10378000C701B6010F9442209B01AC010F94422067
:103790002BED3FE049E450E40F9442209B01AC0143
:1037A00060E070E080E89FE30F949A276B017C0152
:1037B000C092730CD092740CE092750CF092760C5F
:1037C0006091650270916602072E000C880B990BC0
:1037D0000F94E31F2AE037ED43E25CE30F944220AD
:1037E000A70196010F9442206093610270936202D8
:1037F0008093630290936402FF90EF90DF90CF90EC
:103800000895C12CD12C80E8E82E8FE3F82ED0CF7C
:103810000F931F93CF93DF9350E0FC01E40FF51F4C
:103820008081440F551F440F551F4C565A4FEA01D3
:10383000882329F188819981AA81BB81EB010881C4
:1038400019812A813B810097A105B10569F40C59C2
:103850001F4F2F4F3F4FDA010D931D932D933C9334
:1038600013978FEF808306C0081B190B2A0B3B0BA5
:1038700037FDF7CFDF91CF911F910F9108951882F7
:1038800019821A821B82F6CFCF93DF9324E0829FA6
:10389000C0011124EC01CF53D74FFC01E950F84F80
:1038A0008551984FDC012D913D914D915C91608146
:1038B0007181828193810F94A026688379838A83A2
:1038C0009B83DF91CF91089580918F059091900512
:1038D000A0919105B091920580934102909342028C
:1038E000A0934302B093440280918D0590918E0580
:1038F00090936802809367020895809141029091AD
:103900004202A0914302B091440280938F059093AC
:103910009005A0939105B0939205809167029091D4
:10392000680290938E0580938D0584E690E09093D5
:10393000680280936702089580912F12909130124F
:10394000891B877089F48091830D81110DC080914E
:10395000770C9091780C892B39F481E090919D0639
:10396000911103C080E0089581E00895CF93DF9323
:10397000DB01F9019C919130C1F0943080F09450BA
:103980009C938830D1F480819181009771F00197E8
:1039900091838083480F591FEA01188206C08C3535
:1039A00039F49C5F9C93943041F4DF91CF9108955A
:1039B0008B3339F781E08C93F8CF20813181B901C5
:1039C0006F5F7F4F71836083420F531FEA018883CB
:1039D000808191818F3591056CF7E7CF0F931F930D
:1039E00081E00091D3131091D4132091D51330911D
:1039F000D6134091CF135091D0136091D113709191
:103A0000D213041715072607370708F480E01F9123
:103A10000F91089590E080E00895282F9091E50798
:103A2000833021F495FD0FC094FD0FC0892F90E0E5
:103A3000B0E0A0E004C0B695A795979587952A9524
:103A4000D2F78170089581E0089580E00895FC0127
:103A5000659175918591949108958F929F92AF92FF
:103A6000BF92CF92DF92EF92FF92CF93DF93EC0160
:103A70008090BD089090BE08A090BF08B090C0088C
:103A800020E030E0A901C501B4010F94DC1F8823B8
:103A900009F454C0C880D980EA80FB80A701960150
:103AA000C501B4010F94DC1F18160CF04CC0209116
:103AB000B5083091B6084091B7085091B808C701D1
:103AC000B6010F94DC1F882331F1C092B508D09263
:103AD000B608E092B708F092B8082091B908309182
:103AE000BA084091BB085091BC08688179818A81ED
:103AF0009B810F9442209B01AC0160E070E080E864
:103B00009FE30F949F2660930F027093100280939F
:103B100011029093120260910F0270911002809135
:103B2000110290911202DF91CF91FF90EF90DF9000
:103B3000CF90BF90AF909F908F90089560E070E01D
:103B400080E89FE3F0CF60E070E0CB01ECCFCF9254
:103B5000DF92EF92FF92CF93DF93EC01CC80DD8078
:103B6000EE80FF8027E137EB41ED58EBC701B6014E
:103B70000F94002987FD23C023E030E04BE953E494
:103B8000C701B6010F94DC1F1816CCF0C880D9808D
:103B9000EA80FB8027E137EB41ED58EBC701B60126
:103BA0000F94002987FD0BC0C1E023E030E84DE908
:103BB00053E4C701B6010F94DC1F18160CF4C0E0E3
:103BC0008C2FDF91CF91FF90EF90DF90CF900895F1
:103BD0002FEB280F2A3108F047C0E22FF0E0809148
:103BE0002C0590912D05A0912E05B0912F0504C0B4
:103BF000B695A795979587952A95D2F780FD02C02F
:103C000081700895E25FFA4FE081EE2341F18091E7
:103C10007B0790917C07E80FF92FF11D808190EDD3
:103C2000980F9A3030F08E3251F4818180538A306F
:103C300098F4F093FD04E093FC0481E008958D3244
:103C400011F08B3249F4818190ED980F9A3088F30E
:103C50008E3211F48281EACFF0E0E0E0EACF1092F8
:103C6000FD041092FC04E9CF80E008950E94E81D55
:103C7000882341F081E02091FC043091FD04232B46
:103C800009F480E008958F929F92AF92BF92CF92F5
:103C9000DF92EF92FF92C090CB05D090CC05E090E0
:103CA000CD05F090CE0520E030E0A901C701B601B6
:103CB0000F94DC1F8823E1F1A701960160E070E01A
:103CC00080E89FE30F949A276B017C018090CF05D9
:103CD0009090D005A090D105B090D20520E030E0C2
:103CE000A901C501B4010F94DC1F882329F1A501A6
:103CF000940160E070E080E89FE30F949A27C092FF
:103D0000D204D092D304E092D404F092D50460930C
:103D1000D6047093D7048093D8049093D904FF906D
:103D2000EF90DF90CF90BF90AF909F908F900895CD
:103D3000C12CD12C7601CACF60E070E0CB01DFCF7F
:103D4000129A08955F9A8091290C8E7F8093290C96
:103D50008A9A8091290C8D7F8093290C809108018B
:103D600080958170809306018091290C8B7F8093D0
:103D7000290C0C94A01E269A2E9A08958C3221E0CC
:103D8000920714F08CE291E09093E0118093DF11A0
:103D90000C9492EDE7E0F6E0108211821282138219
:103DA00014820C9492ED4F925F926F927F928F9259
:103DB0009F92AF92BF92CF92DF92EF92FF920F93BA
:103DC0001F93CF93DF93EC012091C3053091C4057D
:103DD0004091C5055091C605688179818A819B8192
:103DE0000F949F266B017C012091C7053091C80577
:103DF0004091C9055091CA056C817D818E819F815A
:103E00000F949F264B015C01A7019601609103026C
:103E10007091040280910502909106020F94DC1FBC
:103E2000882309F450C0C0920302D0920402E092A9
:103E30000502F09206022091D2043091D304409101
:103E4000D4045091D504C701B6010F9442202B0130
:103E50003C010F9442286B017C0120E030E0A90175
:103E60000F94DC1F87FD70C020E030E040E450E498
:103E7000C701B6010F94002918162CF4C12CD12CBF
:103E8000C0E4EC2EFE2CA7019601C301B2010F94F1
:103E90009F266093CA047093CB048093CC049093C4
:103EA000CD04C701B6010F940C286093C804062EF8
:103EB000000C770B6F5F7F4F6430710514F064E086
:103EC00070E06093C604D09101021091C804A5016E
:103ED000940160910702709108028091090290910B
:103EE0000A020F94DC1F811133C0D11381C02091CD
:103EF000AE043091AF044091B0045091B104609190
:103F0000CA047091CB048091CC049091CD040F949D
:103F100042202091B2043091B3044091B4045091F6
:103F2000B5040F94A026DF91CF911F910F91FF90C0
:103F3000EF90DF90CF90BF90AF909F908F907F9049
:103F40006F905F904F900895C12CD12C76019BCF3C
:103F50008092070290920802A0920902B0920A028F
:103F60002091D6043091D7044091D8045091D904BF
:103F7000C501B4010F9442204B015C010F9442280B
:103F80006B017C0120E030E0A9010F94DC1F87FD6C
:103F9000F3C020E030E040E450E4C701B6010F94E4
:103FA000002918162CF4C12CD12CB0E4EB2EFE2CD9
:103FB000A7019601C501B4010F949F266093CE041A
:103FC0007093CF048093D0049093D104C701B601BD
:103FD0000F940C286093C904062E000C770B6F5FBA
:103FE0007F4F6430710514F064E070E06093C704A3
:103FF000C091C904D11305C0809102028C1709F445
:1040000070C08091C8049091C9049093020280937B
:1040100001020C2E000CDD0B25E01203C00111245F
:10402000FC01EC0FFD1FEE0FFF1FEE0FFF1FEF5700
:10403000F84F20813181428153812093C204309313
:10404000C3044093C4045093C5040091C704002ED8
:10405000000C110BFC01E00FF11FEE0FFF1FEE0F24
:10406000FF1FEF57F84F60817181828193810F9418
:104070009F266093BE047093BF048093C004909306
:10408000C1042091C60435E02303F0011124CE0FB2
:10409000DF1FCC0FDD1FCC0FDD1FCF57D84F28817E
:1040A00039814A815B812093BA043093BB044093E9
:1040B000BC045093BD04E00FF11FEE0FFF1FEE0F85
:1040C000FF1FEF57F84F60817181828193810F94B8
:1040D0009F266093B6047093B7048093B8049093BE
:1040E000B9048090CE049090CF04A090D004B090FA
:1040F000D1042091BE043091BF044091C00450917E
:10410000C104C501B4010F9442202091C204309132
:10411000C3044091C4045091C5040F94A0266B01C0
:104120007C01C092B204D092B304E092B404F09245
:10413000B5042091B6043091B7044091B804509171
:10414000B904C501B4010F9442202091BA04309102
:10415000BB044091BC045091BD040F94A026A7015C
:1041600096010F949F266093AE047093AF048093E2
:10417000B0049093B104BBCEC12CD12C760118CFE2
:10418000CF92DF92EF92FF92CF93DF93EC010896EC
:104190000E942D1D6B017C0120E030E0A9010F94ED
:1041A000DC1F20E030E0A901882359F0CE010E94F5
:1041B000D31E9B01AC01C701B6010F9442209B01A5
:1041C000AC01688579858A859B850F949F266887D1
:1041D00079878A879B87DF91CF91FF90EF90DF905F
:1041E000CF9008952F923F924F925F926F927F925D
:1041F0008F929F92AF92BF92CF92DF92EF92FF92F7
:104200000F931F93CF93DF93D62FC72FFC0180808E
:104210009180A280B380C501B40120E831E541E07E
:1042200050E00F942026C9016DE671E00F948326BB
:104230006B017C01C501B40120E13EE040E050E0AB
:104240000F942026CA01B90128E130E040E050E097
:104250000F942026362E272E062F172F8CE3482E5C
:10426000512C612C712CC501B401A30192010F9452
:104270002026B62EA72ECA01B901A30192010F94E0
:104280002026CB01C114D10479F1AF92BF927F9364
:104290006F932F923F92FF92EF92DF92CF9288E43A
:1042A00096E19F938F93CF93DF930F94731F8DB7F6
:1042B0009EB70E960FB6F8949EBF0FBE8DBF8D2F82
:1042C0009C2FDF91CF911F910F91FF90EF90DF9086
:1042D000CF90BF90AF909F908F907F906F905F90A6
:1042E0004F903F902F900895E114F104C9F0AF92E0
:1042F000BF927F936F932F923F92FF92EF9288E34A
:1043000096E19F938F93CF93DF930F94731FEDB735
:10431000FEB73C960FB6F894FEBF0FBEEDBFCFCFF1
:10432000012BB9F0AF92BF927F936F932F923F9280
:104330008CE296E19F938F93CF93DF930F94731F3B
:104340008DB79EB70A960FB6F8949EBF0FBE8DBF6D
:10435000B6CF892BA9F0AF92BF927F936F9384E27F
:1043600096E19F938F93CF93DF930F94731FEDB7D5
:10437000FEB738960FB6F894FEBF0FBEEDBF9FCFC5
:10438000AF92BF9280E296E19F938F93CF93DF939A
:104390000F94731F0F900F900F900F900F900F902E
:1043A0008ECFEF92FF920F931F93CF93DF93CDB7F2
:1043B000DEB78C01EDB6FEB60F94291F01962DB71E
:1043C0003EB7281B390B0FB6F8943EBF0FBE2DBF6A
:1043D0008DB79EB70196B8010F94221F0F94ED1070
:1043E0000FB6F894FEBE0FBEEDBEDF91CF911F91C8
:1043F0000F91FF90EF9008958C38910514F08CE8A0
:1044000090E090937511809374110C94AFBAAB0146
:10441000BC014093D3135093D4136093D51370937E
:10442000D6138BE395E10C9467AB2F923F924F929A
:104430005F926F927F928F929F92AF92BF92CF9234
:10444000DF92EF92FF920F931F93CF93DF93CDB73D
:10445000DEB760970FB6F894DEBF0FBECDBF8B8777
:104460006C87042F122F282F30E03E872D87462F90
:1044700050E05A87498785E0982E929EC001939E0E
:10448000900D1124988B8F87FA01E80FF91FEE0F1A
:10449000FF1FEE0FFF1FEF57F84F60817181828180
:1044A00093819B01AC010F949229882309F445C1A3
:1044B0004B85400F6C85610F949EC0011124E985E6
:1044C000FA85E80FF91FEE0FFF1FEE0FFF1FEF57E2
:1044D000F84FC080D180E280F380040F909EA0014D
:1044E0001124E985FA85E40FF51FEE0FFF1FEE0F8B
:1044F000FF1FEF57F84F0081918082807380262F35
:1045000030E0EF85F889E20FF31FEE0FFF1FEE0F8B
:10451000FF1FEF57F84F20807181798372817A8372
:1045200073817B83610F70E0EF85F889E60FF71FD9
:10453000EE0FFF1FEE0FFF1FEF57F84FF88BEF87BF
:10454000F081FC83EF85F889F181FD83EF85F8899F
:10455000F281FE83EF85F889F381FF83FC01E20F8E
:10456000F31FEE0FFF1FEE0FFF1FEF57F84F2081D5
:104570002887A180B2806380FA01E60FF71FEE0F53
:10458000FF1FEE0FFF1FEF57F84F40805180328022
:104590001381202F392D482D572D602F792D882DEF
:1045A000972D0F949229882321F000E0912C812CE3
:1045B000712C9601A701B601C7010F949229882397
:1045C00021F0C02ED92CE82CF72C2C813D814E8176
:1045D0005F816C817D818E819F810F9492298823D8
:1045E00021F01C821D821E821F82222D39814A8168
:1045F0005B81622D79818A819B810F949229882326
:1046000039F02C803D8139834E814A835F815B8301
:104610009201432D512FB201832D912F0F94922996
:10462000882321F0412C512C312C10E028853A2D83
:104630004B2D562D68857A2D8B2D962D0F94922912
:10464000882321F04886A52CB32C612E85E02D858A
:104650003E85829FF001839FF00D112449855A8584
:10466000E40FF51FEE0FFF1FEE0FFF1FEF57F84F80
:10467000FA87E9879601A701B601C7010F94A02622
:10468000202F392D482D572D0F949F266B017C012B
:10469000222D39814A815B81622D79818A819B81BA
:1046A0000F94A0262C813D814E815F810F949F261F
:1046B0009B01AC01C701B6010F94A0266B017C01E0
:1046C00028853A2D4B2D562D68857A2D8B2D962DCC
:1046D0000F94A0269201432D512F0F949F269B01EA
:1046E000AC01C701B6010F94A02620E030E040E401
:1046F00050E40F949A27E985FA8560837183828359
:1047000093836C858B8560960FB6F894DEBF0FBEE1
:10471000CDBFDF91CF911F910F91FF90EF90DF9070
:10472000CF90BF90AF909F908F907F906F905F9051
:104730004F903F902F900D944B0F60960FB6F894CA
:10474000DEBF0FBECDBFDF91CF911F910F91FF90C4
:10475000EF90DF90CF90BF90AF909F908F907F9021
:104760006F905F904F903F902F9008958091FC0440
:104770009091FD04009731F04AE050E070E060E075
:104780000D94F71D60E070E0CB0108958091FC046A
:104790009091FD04009731F04AE050E070E060E055
:1047A0000D94C91C60E070E0CB010895CF93DF93B6
:1047B000EB010E94361E882319F00E94C623EB01EC
:1047C000CE01DF91CF9108950E94C62397FD0CC0C2
:1047D0000E94C6236F3F71058105910509F034F4ED
:1047E0000E94C623862F089580E008958FEF0895D4
:1047F000CF93C62F0E94361E882319F0CF910C94B8
:10480000E4238C2FCF9108958091FC049091FD04B6
:10481000892B41F00E94E42391E0811101C090E0D6
:10482000892F089591E0FCCFCF93DF93C82FD62F27
:104830000E94361E882321F0DF91CF910C9404242E
:104840008C2F0E94E81D811101C08D2FDF91CF9127
:1048500008950E94C623CB010895CF93DF93EB0107
:104860000E94361E882321F0DF91CF910C942924D9
:10487000CE01DF91CF9108950F931F93CF93809135
:10488000FC049091FD040097E9F0FC018F01C191B7
:104890002C2F2F7D81F0C53411F0C536B9F7F80102
:1048A000108270E060E00F946B1BF801C083CF9121
:1048B0001F910F91089570E060E0CF911F910F91CB
:1048C0000D946B1B60E070E0CB01F1CFCF92DF92D3
:1048D000EF92FF926A017B010E94361E882331F01D
:1048E000FF90EF90DF90CF900C943C24C701B6016D
:1048F000FF90EF90DF90CF9008954F925F926F926C
:104900007F928F929F92AF92BF92CF92DF92EF925F
:10491000FF921F93CF93DF9300D01F92CDB7DEB7E6
:1049200019821A821B821C82CE0101964C0188E6F4
:10493000C82E87E0D82E99E1E92E9CE0F92E21ECD3
:10494000A22E28E0B22E10E088E5810F0E94361ECC
:10495000F40181934F01882309F4E0C00E943C24B4
:104960002B013C01812F0E940D1D882309F4CCC02E
:10497000F7012081318142815381C301B2010F943B
:10498000A026F60160837183828393831F5FF4E026
:10499000CF0ED11C84E0E80EF11C94E0A90EB11CEE
:1049A000133091F685E40E94361E8C83882309F427
:1049B000C0C00E943C246B017C0183E00E940D1D5D
:1049C000882371F02091250C3091260C4091270C02
:1049D0005091280CC701B6010F94A0266B017C01F1
:1049E000C0927407D0927507E0927607F09277072D
:1049F0008091C205882359F18091D71382FF27C087
:104A00008C81882321F18981811103C08A818823C7
:104A1000F1F02DEC3CEC4CE45DE360910C087091FE
:104A20000D0880910E0890910F080F94A0269B010D
:104A3000AC016091210C7091220C8091230C90911B
:104A4000240C0F940029181614F40F94910E40E0D2
:104A500050E0BA0186E40E94662420E030E0A9011B
:104A60000F940029181684F40E943C2420E030E0C2
:104A700040E752E40F949A276093410270934202F8
:104A800080934302909344028091D70B83FD28C00A
:104A900080918806882321F12091250C3091260CE5
:104AA0004091270C5091280C609174077091750704
:104AB00080917607909177070F949F262091950615
:104AC0003091960640919706509198060F94A02633
:104AD0006093950670939606809397069093980638
:104AE0000F900F900F900F90DF91CF911F91FF903B
:104AF000EF90DF90CF90BF90AF909F908F907F907E
:104B00006F905F904F900895F5012081318142812F
:104B10005381C301B2010F949F2633CFF7018081E7
:104B20009181A281B381F60180839183A283B383B3
:104B30002DCF8091250C9091260CA091270CB0913F
:104B4000280C8093740790937507A0937607B09311
:104B500077074ECFCF92DF92EF92FF926B017C01ED
:104B600083E3C816D104E104F10470F082E3C81AAB
:104B7000D108E108F10862E370E080E090E00E9473
:104B8000E8A20E9429BEECCFC701B6010E94E8A2AC
:104B9000FF90EF90DF90CF900C9429BE0F931F935E
:104BA000CF93DF930FE31CE0C8E5D1E1F801219139
:104BB0003191419151918F0160E070E080E89FE375
:104BC0000F949A276993799389939993F1E1C83661
:104BD000DF0761F70F94D00CDF91CF911F910F91F8
:104BE0000C94531BCF92DF92EF92FF92CF93DF93FF
:104BF00020912A0C222329F1EC0108960E942D1DF8
:104C00006B017C0120E030E0A9010F94DC1F20E063
:104C100030E0A901882359F0CE010E94D31E9B01E8
:104C2000AC01C701B6010F9442209B01AC0168851D
:104C300079858A859B850F94A026688779878A87DE
:104C40009B87DF91CF91FF90EF90DF90CF900895F9
:104C50002F923F924F925F926F927F928F929F928C
:104C6000AF92BF92CF92DF92EF92FF920F931F937A
:104C7000CF93DF93CDB7DEB76C970FB6F894DEBF56
:104C80000FBECDBF8C015B015A834983FC01EA5BF7
:104C9000FF4F208131814281538129873A874B8799
:104CA0005C87CA01B9010F94E11F6B017C01D5013A
:104CB0002D913D914D915C910F9442200F947E2750
:104CC0002B013C01E981FA812081318142815381AC
:104CD000C701B6010F9442200F947E274B015C015F
:104CE000C301B2010F941328698B7A8B8B8B9C8B39
:104CF000683771058105910540F428E730E040E010
:104D000050E0298B3A8B4B8B5C8BC501B4010F941F
:104D100013286D877E878F87988B6837710581058B
:104D2000910540F448E750E060E070E04D875E8711
:104D30006F87788BF801EE5AFF4F40805180628078
:104D40007380C301B2010F94E31F69837A838B835D
:104D50009C8369897A898B899C890F94E11F6D8B6B
:104D60007E8B8F8B988F20E030E0A90169817A815A
:104D70008B819C810F94DC1F882309F4E1C1A7017A
:104D80009601C701B6010F9442204B015C012D89A9
:104D90003E894F89588DCA01B9010F9442209B0169
:104DA000AC01C501B4010F949F264B015C01298120
:104DB0003A814B815C81CA01B9010F94A0269B0105
:104DC000AC01C501B4010F949A270F947E270F946C
:104DD00013286D837E838F83988766277727CB017F
:104DE00064197509860997090F94E31F4B015C014B
:104DF0006D857E858F8598890F94E11F2B013C017D
:104E000020E030E0A901C501B4010F94DC1F882324
:104E100009F49AC1A3019201C301B2010F94422087
:104E2000698F7A8F8B8F9C8FA7019601C701B6017E
:104E30000F9442209B01AC01698D7A8D8B8D9C8DE6
:104E40000F949F266B017C01A5019401C501B4015B
:104E50000F94A0269B01AC01C701B6010F949A27BD
:104E60000F944228D80195968D909D90AD90BC905E
:104E70009897750164012D813E814F815885C21A32
:104E8000D30AE40AF50A0F941328C61AD70AE80AC7
:104E9000F90AF7FE8EC02D893E894F89588DCA01C7
:104EA000B9010F9442206B017C0129813A814B8129
:104EB0005C81CA01B9010F94A02669877A878B8724
:104EC0009C8720E030E0A90169817A818B819C81F7
:104ED0000F94DC1F882309F43BC1C501B4010F9472
:104EE000E11F29853A854B855C850F944220A701F7
:104EF00096010F949F266D837E838F839887A301ED
:104F00009201C301B2010F9442209B01AC016D815B
:104F10007E818F8198850F94A0262B013C0120E093
:104F200030E040E850E469817A818B819C810F9464
:104F300042209B01AC01C301B2010F949A270F9448
:104F40007E272B013C0120E030E0A9010F940029CD
:104F500018161CF0412C512C3201C301B2010F94E0
:104F600013286D837E838F83988786169706A806FD
:104F7000B90620F48D829E82AF82B8866D817E81D3
:104F80008F8198850F94E11F29853A854B855C8533
:104F90000F944220A70196010F94A0260F944E294A
:104FA0000F94132869877A878B879C87C12CD12C13
:104FB000760169857A858B859C8529893A894B8913
:104FC0005C89621B730B840B950B0F94E11F298185
:104FD0003A814B815C810F949A2720E034E244EFC0
:104FE00059E40F9442200F9413284B015C0169850A
:104FF0007A858B859C852D853E854F855889621BDA
:10500000730B840B950B0F94E11F29813A814B811F
:105010005C810F949A2720E034E244EF59E40F9426
:1050200042200F9413282B013C013FE68316910484
:10503000A104B10408F090C0F401EE0FFF1FEE0FC1
:10504000FF1FEE57F74E85919591A591B4918983F5
:10505000292E3A2EBD8B4FE644165104610471048B
:1050600008F083C0F201EE0FFF1FEE0FFF1FEE5797
:10507000F74E45915591659174919A01CB014D81FF
:105080005E816F817885D80199964D935D936D937C
:105090007C939C974C0D5D1D6E1D7F1DF80145A7EF
:1050A00056A767A770ABE65BFF4F49895A896B89A2
:1050B0007C894083518362837383D5968D929D92C0
:1050C000AD92BC92D897F80141AE52AE63AE74AEC9
:1050D000FD9649814083218232825D8953833496D3
:1050E000208331838283938369857A858B859C8530
:1050F000D1966D937D938D939C93D4973D962D85FA
:105100003E854F85588920833183428353836C9633
:105110000FB6F894DEBF0FBECDBFDF91CF911F91C8
:105120000F91FF90EF90DF90CF90BF90AF909F9046
:105130008F907F906F905F904F903F902F90089549
:1051400060E070E0CB0141CE60E070E0CB0188CE42
:1051500060E070E0CB01F3CEC501B4010E94551AA6
:105160006983272E382E9D8B76CFC301B2010E9412
:10517000551A9B0184CF80912F1290913012891B78
:10518000877019F490E080E0089590912C12992393
:1051900051F0833030F48FEF890F19F080932C1287
:1051A000F1CF10922C12809130122CE5829FC00119
:1051B00011248950974FFC01208120FDE3CF2091DD
:1051C00030122F5F277020932D12309130122091D2
:1051D0002E12321304C020912D1220932E12089506
:1051E00090916F0081E091FD02C080E00895909160
:1051F0006F009D7F90936F00089580FF04C0909191
:10520000930590FD8E7F81FF05C090919305969543
:1052100090FD8D7F82FF06C090919305969596959F
:1052200090FD8B7F08958F929F92AF92BF92CF9205
:10523000DF92EF92FF92CF93DF93209145022223DA
:1052400009F49EC0EC0180919305C82ED12CF12C5D
:10525000E12C80FF2CC08090470290904802A090E3
:105260004902B0904A02288139814A815B81C50197
:10527000B4010F940029181624F488829982AA8216
:10528000BB828090530290905402A0905502B0903F
:105290005602288139814A815B81C501B4010F948E
:1052A000DC1F87FF04C088829982AA82BB82D70153
:1052B000C601B695A7959795879580FF2CC08090DD
:1052C0004B0290904C02A0904D02B0904E022C8167
:1052D0003D814E815F81C501B4010F9400291816EC
:1052E00024F48C829D82AE82BF828090570290907F
:1052F0005802A0905902B0905A022C813D814E81F3
:105300005F81C501B4010F94DC1F87FF04C08C824C
:105310009D82AE82BF8282E0F694E794D794C794D0
:105320008A95D1F7C0FE2CC0C0904F02D090500299
:10533000E0905102F0905202288539854A855B85BC
:10534000C701B6010F940029181624F4C886D9861F
:10535000EA86FB86C0905B02D0905C02E0905D0222
:10536000F0905E02288539854A855B85C701B601C4
:105370000F94DC1F87FF04C0C886D986EA86FB86A7
:10538000DF91CF91FF90EF90DF90CF90BF90AF90E3
:105390009F908F900895CF92DF92EF92FF920F939C
:1053A0001F93C12CD12C76018C0125E23CE041E217
:1053B0005CE06DE17CE089E19CE00E94F5F41F91E6
:1053C0000F91FF90EF90DF90CF9008950D94D00C47
:1053D00080919A06811105C080917907882309F48C
:1053E00063C080918005659B59C081608093800572
:1053F000909103018091800591FF52C0826080935B
:105400008005809180054B9B4DC084608093800512
:105410008091E70580FF10C080919B0680FF0CC043
:105420008091800580FF08C080917807816080931B
:10543000780780E00E94B3C68091E705869580FFDB
:1054400011C080919B06869580FF0CC080918005DD
:1054500081FF08C08091780782608093780781E09F
:105460000E94B3C68091E7058695869580FF1CC093
:1054700080919B068695869580FF16C0809179075E
:10548000882391F08091800582FF0EC0809178077B
:1054900084608093780782E00C94B3C68E7FA6CF99
:1054A0008D7FADCF8B7FB2CF089580919A06811109
:1054B00004C080917907882331F062E070E080E0D9
:1054C00090E00C94AA2508950F931F9380911611D4
:1054D000813019F50E941BA300919C0510919D0538
:1054E00020919E0530919F05601B710B820B930BE1
:1054F00028EE33E040E050E00F9420266091A005B4
:105500007091A1058091A2059091A305620F731F70
:10551000841F951F1F910F9108956091A4057091AC
:10552000A5058091A6059091A705D6CF10921611DA
:1055300010929C0510929D0510929E0510929F0559
:105540001092A4051092A5051092A6051092A70529
:105550001092A0051092A1051092A2051092A30529
:105560000895CF92DF92EF92FF92CF93DF93C62FF1
:10557000FC01C080D180E280F38020E030E0A9010E
:10558000C701B6010F94DC1F20E030E0A90187FDC0
:1055900014C020E030E048EC52E4C701B6010F949B
:1055A000002924E630E040E050E0181634F0C7014E
:1055B000B6010F940C289B01AC01C230A0F4D0E0DE
:1055C000CE50D74FAFEFB0E00F94612624E630E025
:1055D00040E050E00F9442262F3F310519F010F0C3
:1055E0002FEF30E02883DF91CF91FF90EF90DF9095
:1055F000CF9008958091090180FD06C08091D71356
:1056000083FB882780F9089580E00895CF92DF9288
:10561000EF92FF92FC01C080D180E280F38066307F
:1056200019F510920C0610920D0610920E061092AB
:105630000F06109210060E94AFBA20E030E0A901D8
:10564000C701B6010F94DC1F87FF1DC0C12CD12CF0
:105650007601C701B6010F940D29CB01FF90EF90A1
:10566000DF90CF900C94FC210E94CA1E20E030E015
:10567000A901C701B6010F94DC1F87FF15C0C12C1B
:10568000D12C760121C020E030E04CE053E4C7018A
:10569000B6010F9400291816E4F6C12CD12C9CE019
:1056A000E92E93E4F92ED5CF20E030E046E953E42B
:1056B000C701B6010F940029181634F4C12CD12C5F
:1056C00086E9E82E83E4F82EC701B6010F940D2970
:1056D000CB01FF90EF90DF90CF900C94BE1E909185
:1056E000290C977081E0973009F080E008952091AF
:1056F0007E0520FF14C020E83EE3629FA001639F67
:10570000500D729F500D1124CA019695879596955C
:105710008795009731F08A950000E9F708950C9479
:10572000AA250895CF93DF931092D80B1092790C8D
:1057300010927B0C10927A0C10927D0510927C05D1
:10574000CFEFDFEF8091D71385FD07C00E94C8A679
:10575000D0935612C0935512F5CF8FEF9FEF9093D1
:10576000561280935512DF91CF9108958F929F9298
:10577000AF92BF92CF92DF92EF92FF920F931F935F
:10578000CF93DF9310923105109230052FE32093D1
:105790002B0510922A0510922905109228051092C7
:1057A0002C0510922D0510922E0510922F059C01AC
:1057B000F90190812F5F3F4F9032D1F39E34C9F4AD
:1057C000818190ED980F9A3020F08D3211F08B325C
:1057D00081F432969F012F5F3F4F808180538A3042
:1057E00008F47BC09F012F5F3F4F8081803209F416
:1057F00076C0F0937C07E0937B078F010F5F1F4F0C
:10580000C0816AE270E0C8010F94EE29009731F080
:10581000FC01319780818032E1F31182CD3429F08F
:10582000C43519F0C73409F04BC0F80180810F5F0F
:105830001F4F8032D1F380538A3008F041C0C093AB
:105840002B0530E020E04AE0DF011196429FC001C5
:10585000439F900D11249C01205331098081280F12
:10586000311D87FD3A95818190ED980F9A30C8F1EE
:1058700030932A05209329058E3261F4329690E008
:105880004AE0DF0131968C9150ED580F5A3058F1B3
:1058900090932805CD01DC0101964C914032D9F35B
:1058A000CD3489F52E31310539F018F52731310520
:1058B00019F02C31310539F5B0933105A09330053D
:1058C000DF91CF911F910F91FF90EF90DF90CF90DC
:1058D000BF90AF909F908F900895F9017BCFF90111
:1058E00081CFFD01B1CF949F800D112490ED980FD1
:1058F000C8CF2537310538F027373105E8F2203A8F
:1059000083E03807C9F2D0917B0740E050E0BA014C
:1059100010E000E0C12CD12C7601C394FD0131963A
:105920008C91882309F47FC08132E1F4CD34D1F425
:1059300020323105B9F440932C0550932D05609326
:105940002E0570932F05F0933105E093300563E247
:1059500070E0CF010F94EE29009709F4B1CFFC015C
:105960001082AECF81548A3108F058C0DF019D917A
:10597000903291F0A0EDA90FAA30E8F09E3271F4B8
:10598000918190539A30B8F00115110519F48F01E7
:105990000150110990E013C0FD01E8CF9D3211F0D4
:1059A0009B3291F79181A0EDA90FAA3020F09E3291
:1059B00059F79281E6CF9E2F9D1B309759F3A82F60
:1059C000B0E04601570104C0880C991CAA1CBB1CFE
:1059D0008A95D2F7482959296A297B29A25FBA4FAB
:1059E0009C9380818154DF018A3108F497CFDF01D5
:1059F0008191882309F492CF90ED980F9A30B8F3F3
:105A000093ED980F923098F38B3289F3CD01019684
:105A1000EC91E03209F082CFDC01F8CF01151105DD
:105A200001F78D01DECF10933105009330054093CF
:105A30002C0550932D0560932E0570932F0540CFB4
:105A40004F925F926F927F928F929F92AF92BF928E
:105A5000CF92DF92EF92FF92CF93DF9300D000D0EE
:105A60001F921F92CDB7DEB75C01DB01CD90DD90B8
:105A7000ED90FC90E0912A12F0912B12FE83ED83C1
:105A800084819581A681B78189839A83AB83BC8306
:105A90009C01AD01C701B6010F949F262B013C016B
:105AA000F50180809180A280B380AD81BE818D910F
:105AB0009D910D90BC91A02D8D839E83AF83B8875F
:105AC00027E137EB41ED58EBC301B2010F940029F8
:105AD00087FDD1C023E030E04BE953E4C301B201BC
:105AE0000F94DC1F18160CF4C6C02D813E814F8127
:105AF0005885C501B4010F949F262B013C0127E175
:105B000037EB41ED58EB0F94002987FDB4C023E03B
:105B100030E84DE953E4C301B2010F94DC1F1816BD
:105B20000CF4A9C020E030E0A9016D817E818F8155
:105B300098850F94A0262B013C0120E030E040E244
:105B400051E40F94DC1F87FF06C0412C512C30E23A
:105B5000632E31E4732E27E137EB41ED58E3C301A7
:105B6000B2010F949F269B01AC01C501B4010F94B3
:105B7000002987FD80C020E030E84DE953E46D81C5
:105B80007E818F8198850F94A0262B013C0120E017
:105B900030E041E953E40F940029181634F4412C05
:105BA000512C21E9622E23E4722E27E137EB41EDDF
:105BB00058E3C301B2010F94A0269B01AC01C501BB
:105BC000B4010F94DC1F18160CF455C020E030E02F
:105BD000A90169817A818B819C810F94A0264B0158
:105BE0005C0120E030E040EA51E40F94DC1F87FFC5
:105BF00006C0812C912C90EAA92E91E4B92E27E1C0
:105C000037EB41ED58E3C501B4010F949F269B018A
:105C1000AC01C701B6010F94002987FD2CC020E01C
:105C200030E04BE953E469817A818B819C810F9448
:105C3000A0264B015C0120E030E04CE853E40F94D7
:105C40000029181634F4812C912C8CE8A82E83E4BA
:105C5000B82E27E137EB41ED58E3C501B4010F94AD
:105C6000A0269B01AC01B1E0B983C701B6010F9436
:105C7000DC1F18160CF41982898128960FB6F89447
:105C8000DEBF0FBECDBFDF91CF91FF90EF90DF90D1
:105C9000CF90BF90AF909F908F907F906F905F90CC
:105CA0004F900895E3E0F8E082EBDF011D928A95C2
:105CB000E9F708958091C205811104C00E94522E17
:105CC0000C9429B48091D71382FD0D94910E089500
:105CD00080910308882361F09091B408891308C06B
:105CE0008091D71383FF04C081E498E00C94F3B251
:105CF00080E00895FC01238121110C9428AF0895C0
:105D0000EFE6F0E08081826080830895CF92DF9299
:105D1000EF92FF92CF93DF93C82F0E94F02894E078
:105D2000C99FE0011124FE01EB50FA4FC080D180E1
:105D3000E280F38081110E94802EC85ADE4EC70196
:105D4000B6010F94E31F288139814A815B810F944A
:105D50004220DF91CF91FF90EF90DF90CF90089598
:105D60008F929F92AF92BF92CF92DF92EF92FF926B
:105D70001F93CF93DF93CDB7DEB760970FB6F8943C
:105D8000DEBF0FBECDBF182F80E00E94862E4B01D4
:105D90005C018092810590928205A0928305B09269
:105DA000840581E00E94862E6B017C01C0928505EE
:105DB000D0928605E0928705F092880582E00E94E5
:105DC000862E6093890570938A0580938B05909346
:105DD0008C051D861E861F86188A89829A82AB8250
:105DE000BC82CD82DE82EF82F88669877A878B87D4
:105DF0009C8783E00E94862E6D877E878F87988B95
:105E000080912A0C882321F0CE0101960E94C020A7
:105E10001E3FD9F480E1FE013196A9E1BCE001907A
:105E20000D928A95E1F760960FB6F894DEBF0FBE2B
:105E3000CDBFDF91CF911F91FF90EF90DF90CF907A
:105E4000BF90AF909F908F90089584E0189FF001CD
:105E50001124DF01A75EB34F81E090E08C0F9D1FFE
:105E6000E80FF91F40815181628173814D935D93E9
:105E70006D937C931397D7CFCF92DF92EF92FF92DF
:105E8000CF93DF93C82F0E94F02894E0C99FE001D0
:105E90001124FE01E751FA4FC080D180E280F380E7
:105EA00081110E94802EC85ADE4EC701B6010F94A0
:105EB000E31F288139814A815B810F944220DF9161
:105EC000CF91FF90EF90DF90CF9008950E94F0283F
:105ED0009091301290932F1290932E1290932D1236
:105EE00094E690932C1220ED33E03093F608209343
:105EF000F50881110E94802E81E08093E8050895C5
:105F0000CF93DF93CDB7DEB72C970FB6F894DEBFF3
:105F10000FBECDBF0F94AE0D0E94F0289CE0E5EFC0
:105F2000F5E0DE01119601900D929A95E1F781114D
:105F30000E94802ECE0101960E9493C62C960FB629
:105F4000F894DEBF0FBECDBFDF91CF9108952F92A1
:105F50003F924F925F926F927F928F929F92AF92F9
:105F6000BF92CF92DF92EF92FF920F931F93CF9346
:105F7000DF9300D0CDB7DEB78090190C90901A0C4B
:105F8000A0901B0CB0901C0C40901D0C50901E0C4F
:105F900060901F0C7090200CC090210CD090220CAF
:105FA000E090230CF090240C0E94531B0E94A11B34
:105FB00002E61BE187E492E09B838A8386E5282E34
:105FC0008BE1382E198289810E94441CC8010E94ED
:105FD000271DEA81FB816193719381939193FB83E8
:105FE000EA83C1010E94271DEA81FB8160877187D6
:105FF00082879387F981FF5FF9830C5F1F4F84E0ED
:10600000280E311CF330F9F683ED95E00F94130E52
:106010000E94431E0E94CE25A50194016091190C97
:1060200070911A0C80911B0C90911C0C0F94DC1F2A
:1060300081111CC0A301920160911D0C70911E0C76
:1060400080911F0C9091200C0F94DC1F81110EC0C9
:106050002091210C3091220C4091230C5091240C62
:10606000C701B6010F94DC1F8823B9F00F900F9081
:106070000F90DF91CF911F910F91FF90EF90DF90E4
:10608000CF90BF90AF909F908F907F906F905F90D8
:106090004F903F902F900C94802F0F900F900F9067
:1060A000DF91CF911F910F91FF90EF90DF90CF90F4
:1060B000BF90AF909F908F907F906F905F904F9028
:1060C0003F902F90089580916C1190916D11892BC4
:1060D00079F480916C1190916D11892B49F4209184
:1060E0006C1130916D1181E0232B19F480E008953B
:1060F00081E008951092DF048091220290912302A2
:10610000A0912402B09125028093DF059093E005D1
:10611000A093E105B093E205089590918311109248
:106120008311923071F0943079F0913099F481308C
:1061300089F48091DF04882369F0109226020C9480
:106140007A301092180C08958CE697E19093780CB1
:106150008093770C08959091D71393FB882780F94B
:1061600093FF06C081E090913E15911101C080E03F
:106170000895CF93C0917F05CF7739F50E94AB305A
:10618000882319F18091CF139091D013A091D1134E
:10619000B091D2130097A105B105B9F0BC01CD01B2
:1061A0006D597F4F8F4F9F4F24E630E040E050E025
:1061B0000F9420266091D3137091D4138091D5133E
:1061C0009091D6130F942026C22F8C2FCF91089533
:1061D000E2EFF8E010821182089581E008958F9235
:1061E0009F92AF92BF92CF92DF92EF92FF920F9366
:1061F000CF93DF931F92CDB7DEB75C017B014901DE
:106200006B01C40ED51EF501808191810F94FA2592
:106210008983002311F0F7018083BE016F5F7F4FF8
:10622000C4010E947CEDF5018081918101969183EA
:106230008083FFEFEF1AFF0AEC14FD0421F780E0E2
:106240000F90DF91CF910F91FF90EF90DF90CF9063
:10625000BF90AF909F908F9008950F93AB010091E6
:10626000D70521E0022728ED35E0BC0188EB95E059
:106270000E94EF300F9108959091D10095FD0CC0D0
:106280009091D00095FF08C08093D6008091D000F7
:1062900080648093D000089520910E042F5F2F77A3
:1062A0000FB607FC27C090910F04921328C090915D
:1062B000D00095FF1EC090910F0440910E049413DE
:1062C00006C09091D1009F7D9093D10012C0E92F1C
:1062D000F0E0E25FFB4F32819F5F9F773093D60003
:1062E00090930F043091D00030643093D000491760
:1062F00041F3D9CF90910F04921301C0FBCFE091ED
:106300000E04F0E0E25FFB4F828320930E04809145
:10631000D10080628093D10008958F929F92AF92B6
:10632000BF92CF92DF92EF92FF920F931F93CF9382
:10633000DF937C0121E5E20EF11CD7014C914A3537
:1063400009F0A4C06C01B2E5CB0ED11CF60130817E
:10635000353A09F09BC0EC01C05BDF4F2881233048
:1063600008F494C08C0100561F4FD8014C93E15B98
:10637000FF4F308331962083EF54F1093081E05B89
:10638000FF4F30833038B1F43196AC54B1093C91B1
:106390003083E854F109AF5ABF4F50E040E022503B
:1063A000330B42175307CCF4808132968D934F5FA5
:1063B0005F4FF7CF233031F5313809F074C0FC015D
:1063C000EC55FF4FDC01AC5ABF4F2C912083319626
:1063D000885A9F4FDC018C9180834801B12CA12CFD
:1063E000888190E002968A159B050CF43FC0F40169
:1063F00081914F010E943C310E94BFEDFFEFAF1A27
:10640000BF0AEECF323821F5FC01EC5AFF4F308144
:106410004181E05BFF4F408331963083DC01AA5518
:10642000BF4F50E040E02350330B42175307ACF608
:10643000FA01EE7FE45AFF4FE80FF91F6081718186
:106440007C9311966C9311974E5F5F4F1296EDCF30
:10645000243019F6333809F6FC01EC5AFF4F20813D
:106460003181E05BFF4F30833196B0CF80E5DE01B4
:106470001D928A95E9F78AE1F80111928A95E9F768
:106480008AE5D7018C9385EAF6018083DF91CF916D
:106490001F910F91FF90EF90DF90CF90BF90AF9042
:1064A0009F908F900895323809F097CFADCFAF927B
:1064B000BF92CF92DF92EF92FF920F931F93CF93F1
:1064C000DF93EC0184E6C82E80E2D82EE12CF12C7B
:1064D00002E8A12C90E2B92E15E000936413C0925B
:1064E0006513D0926613E0926713F0926813B0922E
:1064F0006E13A0926D131093611381E193E10E94DA
:106500008D318FEFC81AD80AE80AF80A88E7C8164A
:1065100080E2D806E104F10401F724E630E240E02D
:1065200050E0BE0181E193E1DF91CF911F910F9186
:10653000FF90EF90DF90CF90BF90AF900C94C4EDA0
:10654000CF92DF92EF92FF920F931F93CF93DF933F
:10655000CDB7DEB77C01CDB6DEB60F94291F01960C
:106560002DB73EB7281B390B0FB6F8943EBF0FBEB0
:106570002DBF0DB71EB70F5F1F4FB701C8010F9496
:10658000221FC8010E9457320FB6F894DEBE0FBE1C
:10659000CDBEDF91CF911F910F91FF90EF90DF90D3
:1065A000CF9008958F929F92AF92BF92CF92DF9239
:1065B000EF92FF920F931F93CF93DF930E94922B42
:1065C0003AE0C32E30E2D32EE12CF12C15E002E8A4
:1065D00046015701CAE0D0E010926E1310926D137D
:1065E0001093611300936413809265139092661365
:1065F000A0926713B092681381E193E10E948D31FC
:1066000021978FEF881A980AA80AB80A209721F7CD
:106610008AE0C80ED11CE11CF11C82EDC81680E294
:10662000D806E104F104A1F6C12C20E2D22EE12C1F
:10663000F12CD5E0C2E810926E1310926D13D09336
:106640006113C0936413C0926513D0926613E092F5
:106650006713F092681381E193E10E948D311092EB
:106660006E1310926D13D0936113C0936413D7010E
:10667000C6018C529F4FAF4FBF4F809365139093CD
:106680006613A0936713B093681381E193E10E94AE
:106690008D318FEFC81AD80AE80AF80A8AE0C816BE
:1066A00080E2D806E104F10431F69EEDC92E90E2B5
:1066B000D92EE12CF12CD5E0C2E810926E13109285
:1066C0006D13D0936113C0936413C0926513D0927D
:1066D0006613E0926713F092681381E193E10E94E0
:1066E0008D318FEFC81AD80AE80AF80A86EEC81664
:1066F00080E2D806E104F10401F7CC24C39482E1DE
:10670000D82EE12CF12C0AE010E0D5E0C2E810937D
:106710006E1300936D13D0936113C0936413C092F2
:106720006513D0926613E0926713F092681381E1CB
:1067300093E10E948D3110936E1300936D13D093EB
:106740006113C0936413D701C6018096A11DB11DCA
:106750008093651390936613A0936713B0936813A7
:1067600081E193E10E948D318FEFC81AD80AE80ABF
:10677000F80A85E1C81682E1D806E104F10439F689
:1067800082E190E090936E1380936D13D093611328
:10679000C093641384E190E1A0E0B0E080936513BE
:1067A00090936613A0936713B093681381E193E10C
:1067B000DF91CF911F910F91FF90EF90DF90CF90DD
:1067C000BF90AF909F908F900C948D311F920F923D
:1067D0000FB60F9211240BB60F922F938F939F93A6
:1067E000EF93FF9380910F0420910E04821306C053
:1067F0008091D1008F7D8093D10012C0E82FF0E00E
:10680000E25FFB4F92818F5F8F779093D6008093EA
:106810000F049091D00090649093D000281741F31A
:10682000FF91EF919F918F912F910F900BBE0F9041
:106830000FBE0F901F9018951F920F920FB60F92D8
:1068400011240BB60F920F931F932F933F934F93E7
:106850005F936F937F938F939F93AF93BF93CF93E8
:10686000DF93EF93FF93C091D60000913305D09151
:10687000320511E01D0F1F7390910D04913108F046
:106880009FC0E92FF0E08827E75BFB4C8F4F0D940A
:1068900097265A3489349834A734AE34E034B2346D
:1068A000E034B634BA34E034BE34C234C634CD3405
:1068B000E034D834C03229F028F5CA3011F0CD3098
:1068C00031F5011731F0ED2FF0E0EE5CFA4FC283A5
:1068D000D12FD0933205FF91EF91DF91CF91BF91EE
:1068E000AF919F918F917F916F915F914F913F9168
:1068F0002F911F910F910F900BBE0F900FBE0F9015
:106900001F901895CD3481F081E0CE3471F080E194
:106910000CC0CA3338F4C033A0F6C03291F2CD3285
:10692000B1F7CFCFCD3499F782E080930D04C9CF72
:10693000C13359F018F4C03221F2E9CF88E0C433F2
:10694000A1F38BE0C83389F3E2CF83E0EECF84E09C
:10695000C03359F386E0C13341F3D9CF85E0C83362
:10696000B1F6E3CF87E0C23391F6DFCF89E0C133E0
:1069700071F6DBCF8AE0C03351F6D7CF8CE0C73356
:1069800031F6D3CF8DE0C63311F6CFCFC03209F444
:1069900098CF8EE0C33549F2BACF80ED8C0F8A30A4
:1069A00008F08FCF9FE090930D0480930C0489CF63
:1069B000CA3019F0CD3009F084CF10920D0481CF88
:1069C000CA3019F0CD3009F07CCF8091CB138823E9
:1069D000A1F3973089F038F4953079F710923C02A2
:1069E0001092180CEACF9A3059F09F3031F780910D
:1069F0000C040E948D30E1CF81E080930606DDCF4C
:106A000081E080930506D9CF9091C00095FFFCCF1F
:106A10008093C6000895CF93DF93EC01899188237A
:106A200019F00E940435FACF8DE00E9404358AE007
:106A3000DF91CF910C940435CF92DF92EF92FF92C9
:106A4000CF936B017C01C42F4A3069F4F7FE0BC071
:106A5000F094E094D094C094C11CD11CE11CF11CB2
:106A60008DE20E9404354C2FC701B601CF91FF90F3
:106A7000EF90DF90CF900C9461A6CF93DF93EC0161
:106A8000FE0184912196882319F00E940435F8CFE5
:106A9000DF91CF910895CF93DF93D09116118EE3BC
:106AA0009BE10E943D358AE00E9404358091950C5F
:106AB000873009F449C083E08093900C81E0809393
:106AC0006E0280E190E090936E1380936D1385E0E9
:106AD00080936113C2E8C093641384E190E1A0E065
:106AE000B0E08093651390936613A0936713B093FF
:106AF000681381E193E10E948D3161E070E080E0F4
:106B000090E00E94772B81E09AE590936E1380933A
:106B10006D1385E390E09093701380936F1387E07B
:106B200080936113C093641384E890E0A0E0B0E028
:106B30008093651390936613A0936713B0936813C3
:106B400081E193E10E948D3180911611813089F1AC
:106B5000823061F50E94642A6093A0057093A105BC
:106B60008093A2059093A30581E0809316110E9463
:106B70001BA360939C0570939D0580939E05909345
:106B80009F05D23089F08091890690918A060196FE
:106B900090938A06809389061092A8051092A90501
:106BA0001092AA051092AB0581E004C00E94962ABB
:106BB000DBCF80E0DF91CF910895CF93C82FCB0139
:106BC0000E943D3585EB97E10E943D3586EA97E1CD
:106BD000CC2311F08BEA97E10E943D358AE0CF91FA
:106BE0000C94043583ED97E10E943D358CB16DEC3A
:106BF00077E185FB882780F90E94DD3580910301CC
:106C000067EC77E1869581700E94DD3589B161EC92
:106C100077E183FB882780F90E94DD358CB168EB32
:106C200077E1829581700C94DD3580911611813069
:106C3000C1F581E897E10E943D358AE00E94043564
:106C400081E09AE590936E1380936D1387E590E051
:106C50009093701380936F1387E08093611382E8A1
:106C60008093641384E890E0A0E0B0E08093651323
:106C700090936613A0936713B093681381E193E137
:106C80000E948D3182E0809316110E941BA36093B5
:106C9000A4057093A5058093A6059093A70581E0B0
:106CA000089580E008950F931F930E941BA3009105
:106CB000840610918506209186063091870601157D
:106CC00011052105310509F067C0209143122223E7
:106CD00009F45FC0E091411221502093431221E05A
:106CE0002E0F2093411230914412231302C01092B0
:106CF000411224E0E29FF0011124EB5BFD4E008184
:106D000011812281338100938006109381062093A4
:106D1000820630938306600F711F811D911D609361
:106D200084067093850680938606909387068091EB
:106D3000820690918306892B61F11FB7F89480E752
:106D400097E10E943D358AE00E94043584E096E098
:106D500090936E1380936D1380EA90E89093701374
:106D600080936F1387E08093611382E880936413AC
:106D700080EA90E0A0E0B0E0809365139093661302
:106D8000A0936713B093681381E193E10E948D3162
:106D90001FBF1F910F910895601B710B820B930B06
:106DA00097FDF7CF409810928406109285061092B6
:106DB000860610928706EDCF0F931F93CF93DF9334
:106DC0008C01EB019091431220914412921305C063
:106DD0000E9453360E9429BEF5CF8091421234E0C2
:106DE000839FF0011124EB5BFD4E11830083D3835D
:106DF000C2839F5F909343128F5F281739F080936F
:106E00004212DF91CF911F910F910895109242127B
:106E1000F8CFCF92DF92EF92FF921F93CF93DF9341
:106E2000182F662351F01092DE041092DA041092AB
:106E3000DB041092DC041092DD040E941BA36B01A2
:106E40007C018091DA049091DB04A091DC04B09184
:106E5000DD04A7019601281B390B4A0B5B0BDA01F5
:106E6000C901B7FD3DC02091DE0417FD13C0412FBD
:106E7000012E000C550B4C5F5F4F822F022E000C31
:106E8000990B4817590764F184EF91E0A0E0B0E056
:106E9000211724F488EE93E0A0E0B0E08C0D9D1D56
:106EA000AE1DBF1D8093DA049093DB04A093DC0435
:106EB000B093DD042170C22F30E0D32F84E28C9F89
:106EC000B0018D9F700D7C1B112460597C4F82E3B3
:106ED00090E00E94DC368091DE048F5F8093DE04B8
:106EE000DF91CF911F91FF90EF90DF90CF900895A9
:106EF000CF93DF9300D01F92CDB7DEB786EF96E138
:106F00000E943D358AE00E9404358091950C8330C3
:106F1000D9F119821A821B821C8260E0CE0101968F
:106F20000E94B12A19821A821B821C8261E0CE0162
:106F300001960E94B12A81E080936D0210928F0C1D
:106F400080936E0281E09AE590936E1380936D13A7
:106F500083E390E09093701380936F1387E08093A6
:106F6000611382E88093641384E890E0A0E0B0E0CD
:106F70008093651390936613A0936713B09368137F
:106F800081E193E10E948D310F900F900F900F904F
:106F9000DF91CF9108956F927F928F929F92AF92DF
:106FA000BF92CF92DF92EF92FF920F931F93CF93F6
:106FB000DF93CDB7DEB764970FB6F894DEBF0FBE90
:106FC000CDBF1092D0008091D00082608093D0001D
:106FD0001092D50080E18093D4008091D10080612F
:106FE0008093D1008091D10088608093D1008091FE
:106FF000D10080688093D1008091D1008F7D8093F3
:10700000D1008AE5809362138093121385EA8093FE
:10701000631380931313E1EBF3E18AE1DF011D9227
:107020008A95E9F780918E0C882309F473C283E076
:1070300090E090936E1380936D1385E080936113BD
:1070400082E8809364138FE190E1A0E0B0E0809348
:10705000651390936613A0936713B093681381E14F
:1070600093E10E948D3184E690E090936E138093BB
:107070006D1305E00093611312E81093641386E02A
:1070800090E1A0E0B0E08093651390936613A09325
:107090006713B093681381E193E10E948D318BE017
:1070A00090E090936E1380936D130093611310938F
:1070B000641380E092E1A0E0B0E0809365139093C8
:1070C0006613A0936713B093681381E193E10E9464
:1070D0008D3110926E1310926D1300936113109303
:1070E000641384E390E1A0E0B0E080936513909393
:1070F0006613A0936713B093681381E193E10E9434
:107100008D3110926E1310926D13009361131093D2
:1071100064138AE390E1A0E0B0E08093651390935C
:107120006613A0936713B093681381E193E10E9403
:107130008D318091DD119091DE1190936E138093CB
:107140006D13009361131093641386E390E1A0E044
:10715000B0E08093651390936613A0936713B09388
:10716000681381E193E10E948D31809172119091B9
:10717000731190936E1380936D13009361131093AA
:1071800064138CE390E1A0E0B0E0809365139093EA
:107190006613A0936713B093681381E193E10E9493
:1071A0008D3182E090E090936E1380936D13009385
:1071B0006113109364138EE190E1A0E0B0E080933E
:1071C000651390936613A0936713B093681381E1DE
:1071D00093E10E948D3181E080936D0270E6C72EAD
:1071E00070E1D72EE12CF12C10926E1310926D13DA
:1071F0000093611310936413C0926513D0926613C9
:10720000E0926713F092681381E193E10E948D315F
:10721000BFEFCB1ADB0AEB0AFB0AE4E7CE16E0E18C
:10722000DE06E104F10401F7CE0101967C0184E160
:10723000D7011D928A95E9F781E08F9390E99F939A
:107240008F939CE29F938F939F9387E893E09F9304
:107250008F93FF92EF920F94282A20E630E140E0CE
:1072600050E064E973E081E193E10E94C4ED2AE615
:1072700030E140E050E061EA73E081E193E10E9497
:10728000C4ED24E730E140E050E0B70181E193E153
:107290000E94C4ED2EE730E140E050E06FEA73E079
:1072A00081E193E10E94C4ED10926E1310926D1370
:1072B00000936113109364138EE090E1A0E0B0E0BE
:1072C0008093651390936613A0936713B09368132C
:1072D00081E193E10E948D3110926E1310926D1333
:1072E00000936113109364138FE090E1A0E0B0E08D
:1072F0008093651390936613A0936713B0936813FC
:1073000081E193E10E948D310FB6F894DEBF0FBE8C
:10731000CDBF4AE0C42E40E2D42EE12CF12C55E042
:10732000752E62E8662E460157010AE010E01092C1
:107330006E1310926D1370926113609264138092B9
:10734000651390926613A0926713B092681381E15F
:1073500093E10E948D3101501109FFEF8F1A9F0AAE
:10736000AF0ABF0A0115110511F78AE0C80ED11C3A
:10737000E11CF11C92EDC91690E2D906E104F1047A
:1073800091F6C12C30E2D32EE12CF12C05E012E86D
:1073900010926E1310926D13009361131093641387
:1073A000C0926513D0926613E0926713F09268134F
:1073B00081E193E10E948D3110926E1310926D1352
:1073C0000093611310936413D701C6018C529F4F31
:1073D000AF4FBF4F8093651390936613A0936713CD
:1073E000B093681381E193E10E948D31AFEFCA1A27
:1073F000DA0AEA0AFA0ABAE0CB16B0E2DB06E104DE
:10740000F10431F62EEDC22E20E2D22EE12CF12C29
:1074100005E012E810926E1310926D130093611341
:1074200010936413C0926513D0926613E0926713B1
:10743000F092681381E193E10E948D31EFEFCE1A53
:10744000DE0AEE0AFE0AF6EECF16F0E2DF06E104EF
:10745000F10401F7CC24C39482E1D82EE12CF12C65
:107460009AE0A92EB12C05E012E8B0926E13A0921A
:107470006D130093611310936413C0926513D0923F
:107480006613E0926713F092681381E193E10E9422
:107490008D31B0926E13A0926D130093611310930F
:1074A0006413D701C6018096A11DB11D8093651399
:1074B00090936613A0936713B093681381E193E1EF
:1074C0000E948D318FEFC81AD80AE80AF80A95E1B0
:1074D000C91692E1D906E104F10439F68CE596E18A
:1074E0000E943D358AE00E94043564960FB6F894F8
:1074F000DEBF0FBECDBFDF91CF911F910F91FF90E7
:10750000EF90DF90CF90BF90AF909F908F907F9043
:107510006F90089582E090E08CCD0E94CB3710925E
:107520007B0581E080936E028EE097E10E943D35FD
:107530008AE00C9404350F931F93CF938C01C62FD0
:1075400088E093E10E943D35C8010E943D358AE301
:107550000E94043580E38C0F0E9404358AE0CF91AD
:107560001F910F910C9404358BE894E10E943D35F6
:1075700060E08BE794E10E949B3A60E086E694E14C
:107580000E949B3A61E08FE594E10E949B3A61E0A2
:1075900084E594E10E949B3A61E084E494E10E94D6
:1075A0009B3A60E08BE394E10E949B3A61E081E3C7
:1075B00094E10E949B3A61E087E294E10E949B3A49
:1075C00061E080E294E10E949B3A61E088E194E10D
:1075D0000E949B3A61E08AE094E10E949B3A61E05C
:1075E0008CEF93E10E949B3A60E08DEE93E10E9464
:1075F0009B3A60E08FED93E10E949B3A60E089EC5A
:1076000093E10E949B3A61E088EB93E10E949B3AF0
:1076100061E089EA93E10E949B3A61E082EA93E1AA
:107620000E949B3A60E08BE993E10E949B3A61E003
:1076300082E993E10E949B3A61E08DE793E10E9429
:107640009B3A61E08FE693E10E949B3A61E08CE512
:1076500093E10E949B3A60E08FE493E10E949B3AA1
:1076600061E08AE493E10E949B3A61E08DE393E15B
:107670000E949B3A60E089E293E10E949B3A60E0BD
:1076800086E193E10E949B3A60E08AED93E10E94DB
:107690000A1D682F61708DE093E10C949B3A8091F4
:1076A0002C05827149F480912E058C7829F4809103
:1076B0002F05837009F475C082E40E94E81D8823B9
:1076C00051F00E94B62360933B0C70933C0C809366
:1076D0003D0C90933E0C83E50E94E81D882351F0F9
:1076E0000E943C2460936B0C70936C0C80936D0C27
:1076F00090936E0C84E50E94E81D882351F00E944F
:107700003C2460936F0C7093700C8093710C909379
:10771000720C88E50E94E81D882351F00E943C24E9
:107720006093CE087093CF088093D0089093D108CF
:1077300089E50E94E81D882351F00E943C24609353
:10774000D2087093D3088093D4089093D5088AE523
:107750000E94E81D8823B1F00E943C246093D60863
:107760007093D7088093D8089093D9082DEC3CECFF
:107770004CEC5DE30F94DC1F181624F08DE99DE0BE
:107780000E943D3585E40E94E81D882351F00E9447
:107790003C246093DA087093DB088093DC089093B4
:1077A000DD080895AF92BF92CF92DF92EF920F93D0
:1077B0001F93CF93DF935B01EA016901882309F4EA
:1077C00063C086E99DE00E943D35F50160817181CD
:1077D0008281938146E00E9469B6E1100BC08DE87A
:1077E0009DE00E943D35688179818A819B8146E0D8
:1077F0000E9469B686E89DE00E943D35F6016081F1
:1078000071818281938143E00E9469B68FE79DE098
:107810000E943D35F801608171818281938143E04E
:107820000E9469B686E79DE00E943D35F601208101
:10783000318142815381F80160817181828193811C
:107840000F949F2643E00E9469B6EE20F9F08AE08B
:107850000E94043581E69DE00E943D356881798172
:107860008A819B8146E00E9469B68AE00E940435C5
:107870008AE0DF91CF911F910F91EF90DF90CF9031
:10788000BF90AF900C940435E110E4CFDF91CF911D
:107890001F910F91EF90DF90CF90BF90AF90089520
:1078A0000F931F93CF938C01C62F8EE797E00E9412
:1078B0003D35C8010E943D35CC2331F08AE0CF919F
:1078C0001F910F910C940435CF911F910F91089542
:1078D0000E94D4F11092180C10923C020E94AB301E
:1078E000882351F08091D71382FD06C08CE697E182
:1078F0009093780C8093770C61E085E697E10E9485
:10790000503C0C944B350F931F93CF93DF938C0116
:107910006F3F19F41092571160E020915711862F94
:10792000062E000C990B2817190609F08CF56093A8
:10793000571160E08FE297E10E94503CC8010E941D
:107940003D358AE00E940435C8010F94291F800F3D
:10795000911FEC01C01BD10BC034D1053CF0019745
:10796000FC012491207C2038D1F3F3CFDD27AE0138
:10797000B80187E191E10F944A1FC95EDE4E18827B
:1079800087E191E1DF91CF911F910F910C945732D4
:10799000DF91CF911F910F9108951092180C1092C2
:1079A0003C028091D71380648093D71361E08DE30C
:1079B00097E10E94503C42E557E16AE577E185E0B6
:1079C0000E94E2EF60E084E497E10C94833C0F9323
:1079D0001F93CF938C01C62F60E088E897E00E9448
:1079E000503CC8010E943D35CC2331F08AE0CF9154
:1079F0001F910F910C940435CF911F910F91089511
:107A000061E080E997E00C94E73CEF92FF920F93DE
:107A10001F93CF937C018B01C42F60E088E897E02F
:107A20000E94503CC7010E943D3580E20E9404350F
:107A3000C8010E943D35CC2319F08C2F0E940435DB
:107A40008AE0CF911F910F91FF90EF900C94043535
:107A5000DF92EF92FF920F931F93CF93DF93D82E75
:107A60007B018A01E9010E94003DD092831140E030
:107A7000B70189E798E00E94053D0115110531F035
:107A800040E0B80182E798E00E94053D209731F080
:107A900040E0BE0182E798E00E94053D61E08DE68E
:107AA00098E0DF91CF911F910F91FF90EF90DF90C1
:107AB0000C94E73CAF92BF92CF92DF92EF92FF928D
:107AC0000F931F93CF93DF9385E697E00E943D3598
:107AD000C0E0D7E0D15021F080E20E940435FACF17
:107AE0008C2F0E941BEECF5FC53099F78AE00E9471
:107AF000043501E817E0C0E080E20E9404358C2FD5
:107B00000E941BEE5801D5E080E20E940435F50189
:107B1000C080D180E280F380A7019601C701B60141
:107B20000F949229882369F180E20E9404358DE345
:107B30000E9404358DE30E9404358DE30E940435D4
:107B40008DE30E9404358DE30E940435D150F4E1A9
:107B5000AF0EB11CD111D8CF8AE00E940435CF5F9F
:107B60000C5F1F4FC53041F68AE0DF91CF911F9126
:107B70000F91FF90EF90DF90CF90BF90AF900C945B
:107B8000043520E030E0A901C701B6010F940029B7
:107B900087FD03C08BE20E94043543E0C701B601B4
:107BA0000E9469B6D3CF811107C08FEC9DE00E947F
:107BB0003D358AE00C94043583ED9DE0F8CFCF93FA
:107BC000DF93EB010E943D35CE01DF91CF910C9404
:107BD000D9EECF93C62F0E943D358C2FCF910C94B8
:107BE0001BEECF92DF92EF92FF926A017B010E941F
:107BF0003D3542E0C701B601FF90EF90DF90CF9096
:107C00000C9469B6CF92DF92EF92FF926A017B01EA
:107C10000E943D354AE0C701B601FF90EF90DF902A
:107C2000CF900C941C35CF93DF93EB010E943D3530
:107C3000CE01DF91CF910C9422EE4F925F926F9222
:107C40007F928F929F92AF92BF92CF92DF92EF92EC
:107C5000FF920F931F93CF93DF9300D000D01F921A
:107C60001F92CDB7DEB780917A0581110AC4809149
:107C70007805909179059C012F5F3F4F30937905EE
:107C8000209378058E3E924008F4FBC38091DD116D
:107C90009091DE1190936E1380936D1305E0009325
:107CA000611312E81093641386E390E1A0E0B0E062
:107CB0008093651390936613A0936713B093681332
:107CC00081E193E10E948D31809172119091731145
:107CD00090936E1380936D1300936113109364134C
:107CE0008CE390E1A0E0B0E080936513909366137D
:107CF000A0936713B093681381E193E10E948D31E3
:107D00008091DF119091E01190936E1380936D1329
:107D1000009361131093641384E390E1A0E0B0E05A
:107D20008093651390936613A0936713B0936813C1
:107D300081E193E10E948D318091741190917511D0
:107D400090936E1380936D130093611310936413DB
:107D50008AE390E1A0E0B0E080936513909366130E
:107D6000A0936713B093681381E193E10E948D3172
:107D700081E080937A0510927905109278058091C0
:107D8000950C882339F10E949C1C811123C080919D
:107D900077058F5F8093770580917705853620F092
:107DA000109277051092950CE091950CE150E73018
:107DB00008F06AC00E2E000CFF0B8827ED51F14C25
:107DC0008F4F0D949726ED3E3C3F0841344175415D
:107DD000AD41403F10927705DFCF0E946F2B882383
:107DE00009F452C081E080936E0288EE96E10E9411
:107DF0003D358AE00E94043580E190E090936E1357
:107E000080936D1385E08093611312E810936413DF
:107E100084E190E1A0E0B0E0809365139093661355
:107E2000A0936713B093681381E193E10E948D31B1
:107E300081E09AE590936E1380936D1386E390E052
:107E40009093701380936F1387E080936113109366
:107E5000641384E890E0A0E0B0E080936513909311
:107E60006613A0936713B093681381E193E10E94B6
:107E70008D311092950C08C00E946F2B882321F041
:107E80000E949C1C8823A9F380916E02882309F428
:107E900033C780917B058111C0C284E096E0909346
:107EA0006E1380936D1380EA90E890937013809323
:107EB0006F1317E01093611302E80093641380EAD4
:107EC00090E0A0E0B0E08093651390936613A093D8
:107ED0006713B093681381E193E10E948D31809123
:107EE000690290916A02A0916B02B0916C020097B6
:107EF000A105B10509F03FC210926E1310926D13E7
:107F000015E010936113009364138AE890E1A0E0F8
:107F1000B0E08093651390936613A0936713B093BA
:107F2000681381E193E10E948D3189E090E09093A4
:107F30006E1380936D1310936113009364138CE898
:107F400090E1A0E0B0E08093651390936613A09356
:107F50006713B093681381E193E10E948D318091A2
:107F6000690290916A02A0916B02B0916C02009735
:107F7000F1E0AF07B10508F441C2B0936E13A093CE
:107F80006D139093701380936F1387E08093611348
:107F900082E88093641388E890E1A0E0B0E08093E9
:107FA000651390936613A0936713B093681381E1F0
:107FB00093E10E948D318091690290916A02A091B3
:107FC0006B02B0916C02BA2FA92F982F88270097C7
:107FD00021E0A207B10508F417C2B0936E13A09375
:107FE0006D139093701380936F1387E080936113E8
:107FF00012E81093641381EA90E0A0E0B0E080936F
:10800000651390936613A0936713B093681381E18F
:1080100093E10E948D3180912A0C882309F4FAC1E2
:1080200083E090E090936E1380936D1385E08093CE
:1080300061131093641385E490E1A0E0B0E08093B5
:10804000651390936613A0936713B093681381E14F
:1080500093E10E948D3180917B05875E80937B0543
:1080600020917B05822F90E0253608F021C2909365
:108070006E1380936D1385E08093611382E8809383
:10808000641380E090E1A0E0B0E0809365139093EA
:108090006613A0936713B093681381E193E10E9484
:1080A0008D310E949C1C811114C20E94AB30811141
:1080B00005C090917E0591FD0E949C1C90917E05CB
:1080C00080FB91F990937E0591FD03C28091D713B7
:1080D00082FDFFC1809116118150823008F4F9C1F0
:1080E0006091741170917511072E000C880B990B1B
:1080F0000F94E31F6B017C0120E030E0A9010F9495
:10810000DC1F882309F4BBC6609172117091731152
:10811000072E000C880B990B0F94E31F2B013C01D9
:1081200020E030E040E050E4C701B6010F949F2604
:10813000A30192010F94002918160CF4C2C6609195
:10814000DD117091DE11072E000C880B990B0F9436
:10815000E31F6D837E838F8398876091DF11709119
:10816000E011072E000C880B990B0F94E31F4B01B5
:108170005C0120E030E040E251E40F949F262D8125
:108180003E814F8158850F94002918160CF499C62A
:1081900020E030E040E050E4C701B6010F94A02693
:1081A000A30192010F94DC1F87FD10C020E030E096
:1081B00040E251E4C501B4010F94A0262D813E8117
:1081C0004F8158850F94DC1F87FF6AC684E190E0D9
:1081D00090936E1380936D1385E08093611382E812
:1081E0008093641384E190E1A0E0B0E08093651394
:1081F00090936613A0936713B093681381E193E1A2
:108200000E948D318091900C81117CC682E07AC6EB
:108210008AED96E10E943D358AE00E94043581E0B6
:108220009AE590936E1380936D1380E490E09093A1
:10823000701380936F1317E01093611382E880939B
:10824000641384E890E0A0E0B0E08093651390931D
:108250006613A0936713B093681381E193E10E94C2
:108260008D311093950C10CE80917F0C882309F4EA
:108270000BCE0E946F2B882309F406CE0E949C1C13
:10828000811102CE8CEC96E10E943D358AE00E947D
:1082900004358091800C90E0B0E0A0E0895B9F4FB6
:1082A000AE4FB54A21E03AE530936E1320936D133B
:1082B0009093701380936F1387E08093611382E82B
:1082C0008093641384E890E0A0E0B0E080936513AD
:1082D00090936613A0936713B093681381E193E1C1
:1082E0000E948D3110927F0CC4CD0E946F2B882389
:1082F00009F4CACD0E949C1C8111C6CD81E08093F7
:108300006E021092950C8EEB96E10E943D358AE04C
:108310000E94043581E09AE590936E1380936D136B
:108320008EE490E09093701380936F1387E08093B6
:10833000611382E88093641384E890E0A0E0B0E0E9
:108340008093651390936613A0936713B09368139B
:1083500081E193E10E948D3197CD0E949C1C811197
:1083600093CD19821A821B821C8262E0CE01019693
:108370000E9457F57ECD0196A11DB11D35E0B69541
:10838000A795979587953A95D1F70197A109B109D6
:108390000097E1E0AE07B10548F1B0936E13A093EA
:1083A0006D139093701380936F131093611312E801
:1083B000109364138AE890E1A0E0B0E08093651325
:1083C00090936613A0936713B093681381E193E1D0
:1083D0000E948D3188E090E090936E1380936D132E
:1083E00085E08093611310936413A9CD90936E136D
:1083F00080936D1385E080936113D9CF90936E13B2
:1084000080936D1385E0C2CD90936E1380936D13AE
:1084100085E0ECCD82E090E005CE8A3F08F020CEEA
:108420008EEF80937B058DEA96E10E943D358AE0D0
:108430000E94043581E080936E0281E09AE590937A
:108440006E1380936D138DE290E090937013809380
:108450006F1387E08093611382E88093641384E84C
:1084600090E0A0E0B0E08093651390936613A09332
:108470006713B093681381E193E10E948D311092EC
:108480007A0528960FB6F894DEBF0FBECDBFDF91F8
:10849000CF911F910F91FF90EF90DF90CF90BF9001
:1084A000AF909F908F907F906F905F904F900895C6
:1084B0008456910990936E1380936D1385E0809399
:1084C000611382E88093641381E090E1A0E0B0E062
:1084D000DCCD8CE090E090936E1380936D1315E0EB
:1084E0001093611382E88093641384E190E1A0E02B
:1084F000B0E08093651390936613A0936713B093D5
:10850000681381E193E10E948D310E94642A20E189
:108510003EE040E050E00F9420262115310581E037
:108520004807510508F470C050936E1340936D13C3
:108530003093701320936F1387E08093611312E8D8
:108540001093641380E190E1A0E0B0E080936513A4
:1085500090936613A0936713B093681381E193E13E
:108560000E948D310E94642A20E13EE040E050E00C
:108570000F9420262CE330E040E050E00F942026BA
:1085800030936E1320936D1305E0009361131093E5
:10859000641382E190E1A0E0B0E0809365139093D2
:1085A0006613A0936713B093681381E193E10E946F
:1085B0008D310E94B930882309F45CC48F5F8093A9
:1085C0007605E82EF12C833330F5EE0CFF1CF0928B
:1085D0006E13E0926D1300936113109364138EE099
:1085E00090E1A0E0B0E08093651390936613A093B0
:1085F0006713B093681381E193E10E948D3110926B
:108600006E1310926D132BC030936E1320936D1365
:108610001093611394CF84E690E090936E1380934F
:108620006D1300936113109364138EE090E1A0E04A
:10863000B0E08093651390936613A0936713B09393
:10864000681381E193E10E948D31A2E3EA1AA0E868
:10865000FA0AEE0CFF1CF0926E13E0926D13009379
:108660006113109364138FE090E1A0E0B0E0809379
:10867000651390936613A0936713B093681381E119
:1086800093E10E948D310E94B93090E090936E1377
:1086900080936D1385E08093611382E88093641367
:1086A00086E190E1A0E0B0E08093651390936613BB
:1086B000A0936713B093681381E193E10E948D3119
:1086C00020E030E0A901609126127091271280917C
:1086D0002812909129120F94A02620E030E048EC57
:1086E00052E40F9442200F940C2870936E13609301
:1086F0006D1305E00093611312E81093641386E292
:1087000090E1A0E0B0E08093651390936613A0938E
:108710006713B093681381E193E10E948D318091DA
:1087200065029091660290936E1380936D1300938F
:1087300061131093641380E093E1A0E0B0E08093B4
:10874000651390936613A0936713B093681381E148
:1087500093E10E948D3120E030E040E251E46091ED
:108760003F0C7091400C8091410C9091420C0F9401
:1087700042200F94132870936E1360936D1300932F
:1087800061131093641382E492E1A0E0B0E080935F
:10879000651390936613A0936713B093681381E1F8
:1087A00093E10E948D3120E030E040E251E460919D
:1087B000430C7091440C8091450C9091460C0F94A1
:1087C00042200F94132870936E1360936D130093DF
:1087D00061131093641386E492E1A0E0B0E080930B
:1087E000651390936613A0936713B093681381E1A8
:1087F00093E10E948D3120E030E040E251E460914D
:10880000470C7091480C8091490C90914A0C0F9440
:1088100042200F94132870936E1360936D1300938E
:108820006113109364138AE492E1A0E0B0E08093B6
:10883000651390936613A0936713B093681381E157
:1088400093E10E948D3120E030E040E251E46091FC
:108850004B0C70914C0C80914D0C90914E0C0F94E0
:1088600042200F94132870936E1360936D1300933E
:108870006113109364138EE492E1A0E0B0E0809362
:10888000651390936613A0936713B093681381E107
:1088900093E10E948D3120E030E048EC52E4609199
:1088A0001E1270911F1280912012909121120F942C
:1088B00042200F940C2870936E1360936D130093F5
:1088C00061131093641386E392E1A0E0B0E080931B
:1088D000651390936613A0936713B093681381E1B7
:1088E00093E10E948D3120E030E048EC52E4609149
:1088F00022127091231280912412909125120F94CC
:1089000042200F940C2870936E1360936D130093A4
:108910006113109364138AE392E1A0E0B0E08093C6
:10892000651390936613A0936713B093681381E166
:1089300093E10E948D31809175029091760290931F
:108940006E1380936D13009361131093641382E58B
:1089500092E1A0E0B0E08093651390936613A0933A
:108960006713B093681381E193E10E948D31809188
:1089700073029091740290936E1380936D13009321
:1089800061131093641384E592E1A0E0B0E080935A
:10899000651390936613A0936713B093681381E1F6
:1089A00093E10E948D3120E030E040E251E460919B
:1089B000E2117091E3118091E4119091E5110F940F
:1089C00042200F94132870936E1360936D130093DD
:1089D00061131093641386E592E1A0E0B0E0809308
:1089E000651390936613A0936713B093681381E1A6
:1089F00093E10E948D312CEA35EC47E25EE3609111
:108A0000E6117091E7118091E8119091E9110F94AE
:108A10009A2720E030E040E251E40F9442200F9486
:108A2000132870936E1360936D130093611310936A
:108A300064138AE592E1A0E0B0E08093651390931F
:108A40006613A0936713B093681381E193E10E94CA
:108A50008D312CEA35EC47E25EE36091EA117091CA
:108A6000EB118091EC119091ED110F94422020E0D8
:108A700030E040E251E40F9442200F9413287093A9
:108A80006E1360936D1300936113109364138EE55E
:108A900092E1A0E0B0E08093651390936613A093F9
:108AA0006713B093681381E193E10E948D3120E058
:108AB00030E040E251E4609177117091781180913B
:108AC000791190917A110F9442200F94132870938A
:108AD0006E1360936D13009361131093641382E619
:108AE00092E1A0E0B0E08093651390936613A093A9
:108AF0006713B093681381E193E10E948D312CEAF2
:108B000035EC47E25EE360917B1170917C118091BE
:108B10007D1190917E110F949A2720E030E040E281
:108B200051E40F9442200F94132870936E136093B6
:108B30006D13009361131093641386E692E1A0E035
:108B4000B0E08093651390936613A0936713B0937E
:108B5000681381E193E10E948D312CEA35EC47E204
:108B60005EE360917F1170918011809181119091ED
:108B700082110F94422020E030E040E251E40F9453
:108B800042200F94132870936E1360936D1300931B
:108B90006113109364138AE692E1A0E0B0E0809341
:108BA000651390936613A0936713B093681381E1E4
:108BB00093E10E948D318091890C811105C08091D3
:108BC0008B0C882309F46DC06091DD117091DE116A
:108BD000072E000C880B990B0F94E31F20E030E068
:108BE00048EC52E40F9442206B017C016091DF114C
:108BF0007091E011072E000C880B990B0F94E31F66
:108C00009B01AC01C701B6010F949A270F9413285A
:108C10006536710510F064E670E070936E13609332
:108C20006D1305E00093611312E81093641384E25E
:108C300090E1A0E0B0E08093651390936613A09359
:108C40006713B093681381E193E10E948D316091C5
:108C5000DD117091DE11072E000C880B990B0F941B
:108C6000E31F6B017C0120E030E04AE253E40F9403
:108C70000029181624F48091890C811146C1609155
:108C8000DF117091E011072E000C880B990B0F94E7
:108C9000E31F9B01AC01C701B6010F94002987FFB8
:108CA000AFC180917F0C882339F180917E0C91E0D7
:108CB000980F90937E0C90E090936E1380936D13B9
:108CC00085E08093611382E88093641382E490E1ED
:108CD000A0E0B0E08093651390936613A0936713B0
:108CE000B093681381E193E10E948D3180917E0CF5
:108CF0008A3010F010927E0C0E94FA2A882309F420
:108D0000B5C16091930C7091940CEE24E394F12C16
:108D100061157105A9F090E080E00F94E11F20E05B
:108D200030E040E85EE30F9442200F947E2720E07D
:108D300030E040E85FE30F94A0260F9413287B01F6
:108D400001E010E08091790C811102C010E000E098
:108D500080915512909156128F3F980711F40E94FE
:108D6000BEAF9093561280935512080F191FB80189
:108D700090E080E00F94E11F20E030E040E85EE307
:108D80000F9442200F947E274B015C01F0926E13EA
:108D9000E0926D1305E00093611312E810936413E1
:108DA00080E193E1A0E0B0E08093651390936613B7
:108DB000A0936713B093681381E193E10E948D3112
:108DC000C501B4010F94132870936E1360936D1353
:108DD000009361131093641382E193E1A0E0B0E08B
:108DE0008093651390936613A0936713B0936813F1
:108DF00081E193E10E948D3101EB13E1AAE1FA2EAA
:108E0000809132059091330520917405309175055C
:108E1000891B8F7309F449C12A3131050CF0DBC17C
:108E200090913205809133054FEF5FEF981749F02D
:108E3000E82FF0E0EE5CFA4F42818F5F8F738093F2
:108E40003305F901EF54FC4E40838091B1138A350C
:108E500009F0B3C162E070E080E090E00E94772BFF
:108E60008091740590917505019690937505809396
:108E70007405C6CF10926E1310926D13ACCB609137
:108E8000DF117091E011072E000C880B990B0F94E5
:108E9000E31F20E030E0A9010F94DC1F811134C9E9
:108EA0008CE090E090936E1380936D1385E0809337
:108EB000611382E88093641384E190E1A0E0B0E064
:108EC000F3CB8DE090E090936E1380936D1385E06B
:108ED0008093611382E88093641384E190E1A0E0C1
:108EE000B0E08093651390936613A0936713B093DB
:108EF000681381E193E10E948D318091900C811182
:108F000001C081E08093900CDBCB1092890C20E0B3
:108F100030E040E251E46091810C7091820C8091CC
:108F2000830C9091840C0F9442200F940C28709322
:108F30006E1360936D13009361131093641384E5B3
:108F400090E1A0E0B0E08093651390936613A09346
:108F50006713B093681381E193E10E948D3120E0A3
:108F600030E040E251E46091850C7091860C809174
:108F7000870C9091880C0F9442200F940C287093CA
:108F80006E1360936D13009361131093641388E55F
:108F900090E1A0E0B0E08093651390936613A093F6
:108FA0006713B093681381E193E10E948D318CE8DF
:108FB00096E10E943D358AE00E94043581E09AE501
:108FC00090936E1380936D1381E490E090937013EF
:108FD00080936F1387E0809361131093641384E888
:108FE00090E0A0E0B0E08093651390936613A093A7
:108FF0006713B093681381E193E10E948D3151CEE4
:1090000060918B0C662309F44CCE062E000C770B76
:1090100083E796E10E94133E8AE00E940435109295
:109020008B0C84E090E090936E1380936D1385E039
:109030008093611312E8109364138EE890E1A0E02E
:10904000B0E08093651390936613A0936713B09379
:10905000681381E193E10E948D3181E09AE590935C
:109060006E1380936D1383E590E0B0CF10926E1372
:1090700010926D1305E00093611312E810936413CE
:1090800080E193E1A0E0B0E08093651390936613D4
:10909000A0936713B093681381E193E10E948D312F
:1090A00010926E1310926D1393CE121613060CF4D9
:1090B00092C08091151390911613A0911713B0913F
:1090C00018138C34E0E19E07A105B10509F4D7C956
:1090D0008A349041A105B10509F4D1C920E030E0FE
:1090E00040E251E46091190C70911A0C80911B0CB4
:1090F00090911C0C0F9442200F940C2870936E13C7
:1091000060936D1305E00093611312E810936413EC
:1091100088E490E1A0E0B0E080936513909366133B
:10912000A0936713B093681381E193E10E948D319E
:1091300020E030E040E251E460911D0C70911E0C83
:1091400080911F0C9091200C0F9442200F940C28BA
:1091500070936E1360936D130093611310936413F7
:109160008AE490E1A0E0B0E08093651390936613E9
:10917000A0936713B093681381E193E10E948D314E
:1091800020E030E040E251E46091210C7091220C2B
:109190008091230C9091240C0F9442200F940C2862
:1091A00070936E1360936D130093611310936413A7
:1091B0008CE490E1A0E0B0E056C9121613060CF062
:1091C0001FCEF8012F2D11922A95E9F710927505FF
:1091D0001092740515CE909112138091B1139813CB
:1091E00021C0909113138091B21398131BC02330A8
:1091F0003105C4F09091B313909311138091B4137F
:10920000809314139330D1F4982F9D7F9038B1F44C
:109210009091B5139F3409F059C09091B6139B34C7
:1092200009F054C0E1EBF3E18AE1DF011D928A9578
:10923000E9F710927505109274053BCF833809F059
:1092400045C08091B5139091B61398278927982728
:10925000B0E0A0E08093151390931613A09317131A
:10926000B0931813C090B713D12CF12CE12CC092FD
:109270001913D0921A13E0921B13F0921C1328EBCF
:1092800033E140E050E0BA014C155D056E057F0505
:1092900008F04AC0DB01CA01B695A7959795879556
:1092A0000696880F991FFC01EF5EFC4ED9018C9148
:1092B00011969C91892798278927918380834E5FF7
:1092C0005F4F6F4F7F4F2E5F3F4FDECF813861F58D
:1092D0008091B51390E0B0E0A0E0809315139093D7
:1092E0001613A0931713B09318138091B613482F39
:1092F00050E070E060E04093191350931A136093AC
:109300001B1370931C13A7EBB3E1EDE1F3E190E0C5
:1093100030E020E08217930739F04D9150E04193FF
:1093200051932F5F3F4FF6CFE1EBF3E18AE1DF018D
:109330001D928A95E9F710927505109274050E94A6
:10934000F9F5B7CE3F924F925F926F927F928F92D4
:109350009F92AF92BF92CF92DF92EF92FF920F93C4
:109360001F93CF93DF9380912E0587FD38C08091A6
:109370002F058370A1F5C0912A12D0912B1248813C
:1093800059816A817B818DEF95E10E94F13D4C818D
:109390005D816E817F8180E59EE20E94F13D40917A
:1093A00026125091271260912812709129128DE493
:1093B0009EE20E94F13D8AE0DF91CF911F910F91D3
:1093C000FF90EF90DF90CF90BF90AF909F908F90E5
:1093D0007F906F905F904F903F900C940435609019
:1093E0001E1270901F128090201290902112A09057
:1093F0002212B09023120091241210912512C090D5
:109400002612D0902712E0902812F090291288E5B9
:109410000E94361EC82F882309F49AC00E943C245B
:10942000362E472E582ED92F20E030E046E953EC57
:109430000F94002987FD0DC020E030E046E953E499
:10944000632D742D852D9D2F0F94DC1F18160CF0A5
:1094500081C06CE271E08AEE95E10E94133E6CE2FD
:1094600071E085EE95E10E94133E82EE95E10E9447
:109470003D35C0E089E50E94361E882361F10E94D7
:109480003C24362E472E582ED92F20E030E046E9D6
:1094900053EC0F94002987FD0DC020E030E046E931
:1094A00053E4632D742D852D9D2F0F94DC1F18160A
:1094B0000CF055C06CE271E08FEC95E10E94133E18
:1094C0006CE271E08AEC95E10E94133E87EC95E135
:1094D0000E943D35C0E08AE50E94361E882309F4CB
:1094E00043C00E943C246B017C0120E030E040E15D
:1094F00051EC0F94002987FD0AC020E030E040E1E4
:1095000051E4C701B6010F94DC1F18166CF567EF24
:109510007FEF85EB95E10E94133E69E070E080EB00
:1095200095E10E94133E8DEA95E1DF91CF911F9165
:109530000F91FF90EF90DF90CF90BF90AF909F90F2
:109540008F907F906F905F904F903F900C943D353F
:10955000C1E090CF632C742C852C9D2E8BCFA32C37
:10956000B42C052D1D2FB7CFCC23E1F0C301D401BE
:1095700080931E1290931F12A0932012B093211279
:10958000C501D8018093221290932312A093241234
:10959000B0932512C0922612D0922712E092281280
:1095A000F0922912DF91CF911F910F91FF90EF90D0
:1095B000DF90CF90BF90AF909F908F907F906F90F3
:1095C0005F904F903F9008958EE597E00C943D3565
:1095D00088E597E00C943D3584E690E09093B905DA
:1095E0008093B8051092D9051092D8050C94B7DB7A
:1095F000EF92FF920F931F93CF93DF93CDB7DEB718
:1096000062970FB6F894DEBF0FBECDBF0E94FD2853
:10961000882309F43FC04EED53E082FF02C042ECC4
:1096200053E02EED33E081FF02C024EC33E080FDF7
:109630002EC08EED93E05F934F933F932F939F93B4
:109640008F9387E298E19F938F938E010F5F1F4F57
:109650001F930F930F94731F0E94E84AC8010E9442
:109660000B35C8010E949CF10FB6F894DEBF0FBE07
:10967000CDBF81E062960FB6F894DEBF0FBECDBFBE
:10968000DF91CF911F910F91FF90EF90089586EC9D
:1096900093E0D1CF80E0EECFCF92DF92EF92FF92B6
:1096A0008AE50E94361E882309F45AC00E943C2491
:1096B00020E030E040E050EC0F94DC1FC12CD12CB6
:1096C000E12C90ECF92E87FD0FC00E943C2420E095
:1096D00030E040E050E40F94002918160CF462C00A
:1096E0000E943C246B017C012091470C3091480C76
:1096F0004091490C50914A0CC701B6010F94422089
:109700000F940C28CB010E9425F180E50E94E81DF2
:1097100081114EC0A7019601609126127091271207
:1097200080912812909129120F94A02660932612FE
:109730007093271280932812909329120E94E84A6E
:10974000409126125091271260912812709129128F
:109750008EE995E10E94F13D8AE00E94043505C042
:1097600083E50E94361E8111A1CF80912E0587FDD1
:1097700024C080912F05837001F50E94E84A409132
:1097800026125091271260912812709129128FE8A9
:1097900095E10E94F13D8AE0FF90EF90DF90CF903D
:1097A0000C940435C12CD12CE12C80E4F82E9CCFF4
:1097B0000E9404248111AECFD8CF82E50E94E81D1B
:1097C0008111DBCFFF90EF90DF90CF900895CF9382
:1097D00084E50E94361EC0E08823D9F00E94E4236D
:1097E000C82F1816B4F40E94E84A8DE40E9404358C
:1097F0008091290590912A050E94D9EE6C2FCC0FFB
:10980000770B8DEA9EE00E94133E8AE00E940435A9
:10981000CFEF8C2FCF9108954F925F926F927F92EE
:109820008F929F92AF92BF92CF92DF92EF92FF9270
:10983000CF93DF93CDB7DEB72C970FB6F894DEBF8A
:109840000FBECDBF4090C1085090C2086090C308C1
:109850007090C4082091470230914802409149021B
:1098600050914A02C301B2010F94A02669837A8302
:109870008B839C838090C5089090C608A090C708F1
:10988000B090C80820914B0230914C0240914D029B
:1098900050914E02C501B4010F94A0266D837E83C2
:1098A0008F839887C090C908D090CA08E090CB08F1
:1098B000F090CC0820914F0230915002409151021B
:1098C00050915202C701B6010F94A02669877A878A
:1098D0008B879C872091530230915402409155020E
:1098E00050915602C301B2010F94A0262B013C01F6
:1098F00020915702309158024091590250915A02DA
:10990000C501B4010F94A0264B015C0120915B02BC
:1099100030915C0240915D0250915E02C701B60138
:109920000F94A0266B017C010E94E84A88EE9DE01E
:109930000E943D3583E50E94E81D882321F00E94A6
:1099400004248093450280914502811151C08FEC1F
:109950009DE00E943D3580EE9DE00E943D354981AD
:109960005A816B817C8182EF9CE10E94F13D4D81A7
:109970005E816F81788580E59EE20E94F13D498598
:109980005A856B857C858DE49EE20E94F13D8EEDCB
:109990009DE00E943D3586ED9DE00E943D35B3017E
:1099A000A20182EF9CE10E94F13DB501A40180E596
:1099B0009EE20E94F13DB701A6018DE49EE20E9465
:1099C000F13D8AE02C960FB6F894DEBF0FBECDBFF6
:1099D000DF91CF91FF90EF90DF90CF90BF90AF904D
:1099E0009F908F907F906F905F904F900C94043574
:1099F00083ED9DE0AECF5F926F927F928F929F92A8
:109A0000AF92BF92CF92DF92EF92FF920F931F938C
:109A1000CF93DF931F92CDB7DEB77C0139018B0165
:109A20005B01A40EB51ED12CC12CA016B10609F401
:109A300050C0F70180809180F80151908F015982C8
:109A4000C4010F94FA255816B9F1652DC4010F947D
:109A50000226FFEFCF1ADF0AC6018F779927892BDD
:109A600021F162E070E080E090E00E94E8A2C40191
:109A70000F94FA2599818917F9F00E94E84A8FE638
:109A800094E00E943D3581E00F90DF91CF911F91CE
:109A90000F91FF90EF90DF90CF90BF90AF909F908D
:109AA0008F907F906F905F90089562E070E080E00B
:109AB00090E00E94AA25DBCFBE016F5F7F4FC301FC
:109AC0000E947CEDF70180819181019691838083D2
:109AD000ACCF80E0D9CFCF92DF92EF92FF920F937D
:109AE0001F93CF93DF93CDB7DEB7CA5AD1090FB614
:109AF000F894DEBF0FBECDBFCF55DF4F188219825D
:109B00001A821B82C15AD0408091C8039091C90328
:109B1000A091CA03B091CB03CB55DF4F88839983C3
:109B2000AA83BB83C55AD04084E690E09093B905E0
:109B30008093B8051092D9051092D8051092DA05D5
:109B400028ED35E044E050E0BE016B557F4F88EBD7
:109B500095E00E94FB4C8091B8059091B905029662
:109B60009093B9058093B8051092D9051092D80545
:109B700081E0C655DF4F8883CA5AD040CE01865552
:109B80009F4F0E94FFD128ED35E048E450E06BE2A2
:109B90007CE088EB95E00E94FB4C28ED35E040E14D
:109BA00050E06EEC78E088EB95E00E94FB4C8AE098
:109BB00097EDA3EABCE3CF55DF4F88839983AA834F
:109BC000BB83C15AD040CE018F559F4F0E94F6D122
:109BD00087EF97E00E9411D286E292E00E9408D2BD
:109BE00082E292E00E94F6D18091BD089091BE0879
:109BF000A091BF08B091C00889839A83AB83BC83CE
:109C00008E010F5F1F4FC8010E94F6D1CF55DF4F65
:109C1000188219821A821B82C15AD0407E018DE6B9
:109C2000E80EF11C83E0D7018C938983CE018F5518
:109C30009F4F0E94F6D1C7010E94FFD1C8010E9428
:109C4000FFD14AE0D42EDA94DD2031F0CE018F55D9
:109C50009F4F0E94F6D1F7CF8EE192E10E9411D280
:109C6000CF55DF4F188219821A821B82C15AD04009
:109C70003AE0D32EDA94DD2031F0CE018F559F4F9C
:109C80000E94F6D1F7CF85E0C82EC982F701C082C5
:109C9000C8010E94FFD1C7010E94FFD128ED35E025
:109CA00048E050E06BEC75E088EB95E00E94FB4CDF
:109CB00028ED35E048E050E063EC75E088EB95E096
:109CC0000E94FB4C28ED35E044E650E061E877E087
:109CD00088EB95E00E94FB4C19828FEFD7018C93A3
:109CE000C8010E9408D2C7010E94FFD190E1D92E7D
:109CF000F8018D2D11928A95E9F728ED35E040E1C4
:109D000050E0B80188EB95E00E94FB4C1982C80135
:109D10000E9408D2198A1A8A1B8A1C8A80E090E065
:109D2000A0E8BFE38D879E87AF87B88B8091E21153
:109D30009091E311A091E411B091E51189839A8388
:109D4000AB83BC832CEA35EC47E25EE36091E6111D
:109D50007091E7118091E8119091E9110F949A2781
:109D60006D837E838F8398872CEA35EC47E25EE330
:109D70006091EA117091EB118091EC119091ED11CD
:109D80000F94422069877A878B879C8728ED35E07E
:109D900044E150E0B80188EB95E00E94FB4C84E17F
:109DA00090E09A838983C8010E94E4D18091771161
:109DB00090917811A0917911B0917A1189839A8349
:109DC000AB83BC832CEA35EC47E25EE360917B1108
:109DD00070917C1180917D1190917E110F949A2742
:109DE0006D837E838F8398872CEA35EC47E25EE3B0
:109DF00060917F11709180118091811190918211F9
:109E00000F94422069877A878B879C87C8010E94BC
:109E1000EDD18CE0EBE7F2E0D80101900D928A954C
:109E2000E1F7C8010E94EDD11982C8010E94FFD15B
:109E30008FE790E09A838983C8010E94E4D1E7E824
:109E4000F2E0D80101900D92CA94E1F728ED35E0D7
:109E500045E050E0B80188EB95E00E94FB4C809112
:109E6000C2058983C8010E9408D280E2ECE8F2E0D2
:109E7000D80101900D928A95E1F728ED35E040E296
:109E800050E0B80188EB95E00E94FB4CD7011C9292
:109E9000C7010E9408D28AEE97E00E9408D286EE9F
:109EA00097E00E94F6D1CF55DF4F188219821A82AF
:109EB0001B82C15AD040CE018F559F4F0E94F6D1D0
:109EC00080E2F80111928A95E9F728ED35E040E249
:109ED00050E0B80188EB95E00E94FB4CFE01F9963A
:109EE00088E0DF011D928A95E9F744E650E060E0E2
:109EF00070E049835A836B837C834D835E836F83D9
:109F0000788783E090E0A0E0B0E089879A87AB870C
:109F1000BC874D875E876F87788B498B5A8B6B8B9D
:109F20007C8B8D8B9E8BAF8BB88F898F9A8FAB8FED
:109F3000BC8F8D8F9E8FAF8FB8A38EE190E0A0E095
:109F4000B0E089A39AA3ABA3BCA38DA39EA3AFA3A8
:109F5000B8A789A79AA7ABA7BCA78DA79EA7AFA7AD
:109F6000B8AB89AB9AABABABBCAB8DAB9EABAFAB7D
:109F7000B8AF28ED35E040E450E0B80188EB95E05B
:109F80000E94FB4CF8018D2D11928A95E9F728ED7E
:109F900035E040E150E0B80188EB95E00E94FB4CD1
:109FA000D8011D92DA94E9F728ED35E040E150E060
:109FB000B80188EB95E00E94FB4CCF55DF4F18822B
:109FC00019821A821B82C15AD040CE018F559F4FF1
:109FD0000E94F6D12CE0D22EF8018D2D11928A9597
:109FE000E9F728ED35E04CE050E0B80188EB95E06A
:109FF0000E94FB4C8CE6D8011D928A95E9F728ED6A
:10A0000035E04CE650E0B80188EB95E00E94FB4C4F
:10A010008CEA95E00E94EDD128ED35E048E050E073
:10A020006AEB75E088EB95E00E94FB4CF70111921A
:10A03000DA94E9F7C755DF4F1882C95AD04080E05B
:10A0400090E0A0E4B0E4C356DF4F88839983AA83ED
:10A05000BB83CD59D040C7010E9411D2CE01875594
:10A060009F4F0E94FFD1CE0183569F4F0E94F6D191
:10A0700080E3D7011D928A95E9F78EE69BE10E9465
:10A080003D358AE00E94043528ED35E040E350E09C
:10A09000B70188EB95E00E94FB4C8091DA058111B5
:10A0A00028C00091B8051091B9058091D80590910C
:10A0B000D905F7019183808384E690E09093B905F8
:10A0C0008093B80528ED35E044E050E064EE72E09E
:10A0D00088EB95E00E94FB4CC7010E94E4D191E01F
:10A0E0000137134009F490E08091DA05892B8093C1
:10A0F000DA058091DA05811105C060E082EA9BE112
:10A100000E94833C82E89BE10E943D358AE00E94E8
:10A1100004359091DA0581E08927C655DF4F0FB6E7
:10A12000F894DEBF0FBECDBFDF91CF911F910F918D
:10A13000FF90EF90DF90CF900895CF93DF9300D002
:10A140001F92CDB7DEB7809188068823C1F083E3E4
:10A1500090E09C838B831A8219829E012F5F3F4F70
:10A1600040E150E069E876E0CE0103960E94FB4CA6
:10A1700082E89BE10E943D358AE00E9404350F9001
:10A180000F900F900F90DF91CF910895CF92DF92B3
:10A19000EF92FF92CF93C82F809116118150823099
:10A1A00008F069C00E947837109216110E941BA314
:10A1B0006093A4057093A5058093A6059093A705C9
:10A1C000C090A805D090A905E090AA05F090AB0535
:10A1D0000E94642AAB01BC014093A8055093A905D5
:10A1E0006093AA057093AB0580918D0690918E06C1
:10A1F000A0918F06B09190068C199D09AE09BF09F8
:10A20000840F951FA61FB71F80938D0690938E060F
:10A21000A0938F06B0939006C1110AC0C1E00E94BE
:10A220009D508C2FCF91FF90EF90DF90CF900895AD
:10A2300080918B0690918C06019690938C0680936A
:10A240008B060E94642AC0909106D0909206E090FE
:10A250009306F0909406C616D706E806F906F0F6BF
:10A260000E94642A609391067093920680939306ED
:10A2700090939406D3CFC0E0D2CFCF93DF9300D09A
:10A280001F921F92CDB7DEB781E08093880680E1F0
:10A29000E9E8F6E0DF011D928A95E9F70E949D50FA
:10A2A00086E18D8382E390E09C838B831A821982FE
:10A2B0009E012F5F3F4F41E050E0BE016B5F7F4F3B
:10A2C000CE0103960E94FB4C0F900F900F900F90C1
:10A2D0000F90DF91CF910895CF93DF93CDB7DEB785
:10A2E000A8970FB6F894DEBF0FBECDBF8C01F42E39
:10A2F0000E94DCBA0E94E44A88E397E00E943D3560
:10A300000115110511F40FE217E080917E0580FD23
:10A3100079C0816080937E058BE197E00E943D3596
:10A320008AE00E940435CC24C3948AE5D82ED092CA
:10A330006E13C0926D138FE090E090937013809332
:10A340006F1397E0792E7092611322E8E22EE0926B
:10A35000641334E8832E912CA12CB12C80926513C8
:10A3600090926613A0926713B092681381E193E113
:10A370000E948D31D0926E13C0926D1388E590E0EB
:10A380009093701380936F1370926113E092641333
:10A390008092651390926613A0926713B09268132F
:10A3A00081E193E10E948D318AE289838A838B83E4
:10A3B0008C83F801DE011596BE016F5F7F4FCD01E2
:10A3C000861B970B2491319621110CC0FB01E80FDD
:10A3D000F91F8AE29F01261B370B2832310524F42E
:10A3E0008193F8CF2D93EBCF20E630E140E050E0B1
:10A3F00081E193E10E94C4ED6AE070E080E090E0CA
:10A400000E94772B61E086E297E00E94503C89EE43
:10A4100093E030E6019729F0232F2A950000E9F711
:10A42000F9CFF89489EE93E038EE019729F0232FC5
:10A430002A950000E9F7F9CF0E94DCBAFF2031F03D
:10A440000E94A21E0E94BB1EA895FECF0E94A01EC5
:10A45000F9CF80917807882319F010927807089532
:10A4600040E070E060E088E997E10E946C518091E3
:10A47000960C9091970C2FEF3FEF981751F0E92F22
:10A48000F0E0EA56F34F228130E09F5F9F77909390
:10A49000970CC90108951F920F920FB60F921124C5
:10A4A0000F900FBE0F901F9018951F920F920FB62E
:10A4B0000F9211240BB60F920F931F932F933F937C
:10A4C0004F935F936F937F938F939F93AF93BF93BC
:10A4D000CF93DF93EF93FF93C091C6000091970C49
:10A4E000D091960C11E01D0F1F7790910B049131C4
:10A4F00008F09FC0E92FF0E08827EE57FD4A8F4F04
:10A500000D9497269352C252D152E052E7521953FA
:10A51000EB521953EF52F3521953F752FB52FF52B9
:10A52000065319531153C03229F028F5CA3011F0DF
:10A53000CD3031F5011731F0ED2FF0E0EA56F34F51
:10A54000C283D12FD093960CFF91EF91DF91CF91E1
:10A55000BF91AF919F918F917F916F915F914F913B
:10A560003F912F911F910F910F900BBE0F900FBE37
:10A570000F901F901895CD3481F081E0CE3471F0AA
:10A5800080E10CC0CA3338F4C033A0F6C03291F277
:10A59000CD32B1F7CFCFCD3499F782E080930B0461
:10A5A000C9CFC13359F018F4C03221F2E9CF88E0A5
:10A5B000C433A1F38BE0C83389F3E2CF83E0EECF5D
:10A5C00084E0C03359F386E0C13341F3D9CF85E04D
:10A5D000C833B1F6E3CF87E0C23391F6DFCF89E02D
:10A5E000C13371F6DBCF8AE0C03351F6D7CF8CE0B0
:10A5F000C73331F6D3CF8DE0C63311F6CFCFC0329B
:10A6000009F498CF8EE0C33549F2BACF80ED8C0FB4
:10A610008A3008F08FCF9FE090930B0480930C0456
:10A6200089CFCA3019F0CD3009F084CF10920B04D5
:10A6300081CFCA3019F0CD3009F07CCF8091CB1397
:10A640008823A1F3973089F038F4953079F7109288
:10A650003C021092180CEACF9A3059F09F3031F733
:10A6600080910C040E948D30E1CF81E0809306063A
:10A67000DDCF81E080930506D9CF8EBD0DB407FEF6
:10A68000FDCF08958FEF8EBD0DB407FEFDCF8EB5C3
:10A690000895909164009B7F90936400982F906A36
:10A6A00096959CBD80FD03C091E0863009F490E052
:10A6B0009DBD0895CF93DF93EB010E943D35CE0100
:10A6C000DF91CF910C9426AB2F923F924F925F92E5
:10A6D0006F927F928F929F92AF92BF92CF92DF92B2
:10A6E000EF92FF920F931F93CF93DF93009709F0A0
:10A6F000AAC110927B0C10927A0C90937D058093E6
:10A700007C05BAE0CB2EB0E2DB2EE12CF12C15E07B
:10A7100002E846015701C4E1D0E01092B412109251
:10A72000B3121093A7120093AA128092AB129092C8
:10A73000AC12A092AD12B092AE1287E592E10E94E7
:10A740008D3121972FEF821A920AA20AB20A20971E
:10A7500021F744E1C40ED11CE11CF11C8AE5C816A6
:10A7600080E2D806E104F104A1F6C12CA0E2DA2EC1
:10A77000E12CF12CD5E0C2E81092B4121092B31281
:10A78000D093A712C093AA12C092AB12D092AC126F
:10A79000E092AD12F092AE1287E592E10E948D3107
:10A7A0001092B4121092B312D093A712C093AA12AF
:10A7B000D701C6018C529F4FAF4FBF4F8093AB1252
:10A7C0009093AC12A093AD12B093AE1287E592E1D4
:10A7D0000E948D31EFEFCE1ADE0AEE0AFE0AFAE091
:10A7E000CF16F0E2DF06E104F10431F6FEEDCF2EE4
:10A7F000F0E2DF2EE12CF12CD5E0C2E81092B41289
:10A800001092B312D093A712C093AA12C092AB12A7
:10A81000D092AC12E092AD12F092AE1287E592E1C6
:10A820000E948D312FEFC21AD20AE20AF20A46EED6
:10A83000C41640E2D406E104F10401F7CC24C39429
:10A84000E2E1DE2EE12CF12C0AE010E0D5E0C2E8D6
:10A850001093B4120093B312D093A712C093AA120C
:10A86000C092AB12D092AC12E092AD12F092AE1246
:10A8700087E592E10E948D311093B4120093B312D8
:10A88000D093A712C093AA12D701C6018096A11D2A
:10A89000B11D8093AB129093AC12A093AD12B09304
:10A8A000AE1287E592E10E948D318FEFC81AD80A67
:10A8B000E80AF80AE5E0CE16E2E1DE06E104F1047A
:10A8C00039F600917A0C10917B0C0115110509F0F5
:10A8D000D6C08091790C882309F4E1C02AE030E2E7
:10A8E00040E050E06CEC73E087E592E10E94C4ED3B
:10A8F000C1E0D0E003E010E0E0907A0CF0907B0C37
:10A9000035E0332E42E8242E44244A94542C64E04B
:10A91000662E712C7FE1C72E74E0D72E80917A0CC1
:10A9200090917B0C800F911FE816F90608F0D5C0B6
:10A93000C7010E94DFEE882309F481C08091911144
:10A9400064E871E1882311F061E971E1FB01019094
:10A950000020E9F7CF010197861B970BF4E1FC9FDC
:10A960009001FD9F300D1124265F3F4D50E040E0E7
:10A97000459710F0FB01128A87E592E10E94C4ED31
:10A98000CE018F5F9D4EB0E0A0E021964E0124E005
:10A99000880C991C2A95E1F7FDEF8F1AFFE99F0AB1
:10A9A000B12CA12C2091D71324FF7EC07092B41239
:10A9B0006092B3123092A7122092AA128093AB1227
:10A9C0009093AC12A093AD12B093AE1287E592E1D2
:10A9D0000E948D31D092B412C092B3123092A7125D
:10A9E0002092AA128092AB129092AC12A092AD1259
:10A9F000B092AE1287E592E10E948D31B7018DE2EF
:10AA000097E10E94DF3D8091911161E971E181112F
:10AA100002C064E871E18AE297E10E945A5368ED4E
:10AA20007BE086E297E10E945A5364E871E185E297
:10AA300097E10E945A5381E297E10E943D352FEF42
:10AA4000E21AF20A6BCF20917A0C30917B0CA901AB
:10AA50004150510960917C0570917D056817790717
:10AA600038F42C5F3F4F30937B0C20937A0C45CE0B
:10AA70004430510508F43DCE24503109F4CF043060
:10AA8000110569F48091790C882331F083E090E01E
:10AA900090937B0C80937A0CD0E0C0E02DCFD0E077
:10AAA000C0E004E010E028CF1092B4121092B3126C
:10AAB0003092A7122092AA128093AB129093AC12FC
:10AAC000A093AD12B093AE1287E592E10E948D3152
:10AAD0005092B4124092B31281CFDF91CF911F9167
:10AAE0000F91FF90EF90DF90CF90BF90AF909F902D
:10AAF0008F907F906F905F904F903F902F90089530
:10AB0000AF92BF92CF92DF92EF92FF920F931F937B
:10AB1000CF93DF93CDB7DEB7E6970FB6F894DEBFDD
:10AB20000FBECDBF0091300510913105F8010190A5
:10AB30000020E9F731976F01C01AD10AF801CF015F
:10AB4000801B910B8C159D053CF481918F32B9F7D8
:10AB5000DF0111971C92F3CF8BE1E7EFF3E1DE0108
:10AB60005C9601900D928A95E1F7F12CE12CEC14A2
:10AB7000FD040CF05DC0F801EE0DFF1D8081811118
:10AB800003C08FEFE81AF80A5801AE0CBF1CF5019C
:10AB90008081882309F44CC0FFEFEF1AFF0AF80107
:10ABA000EE0DFF1D7F01E01AF10A81918111FACFAC
:10ABB000CE014C960E94B9AF8BE1FE017C96DE017E
:10ABC000119601900D928A95E1F7B501CE0101969B
:10ABD0000E94C7A7CE0101960E947A2E8FE20E94A2
:10ABE00004358091911181113BC089ED93E00E9461
:10ABF00026AB8091D71384FF1BC019821C8221E0F1
:10AC0000A501BE01645E7F4FCE0101960E94FBB19B
:10AC1000811129C08AE00E9404350E94E84AB501EA
:10AC20008CE096E10E945A53CE0101960E947A2E42
:10AC30008AE00E940435CE014C960E947A2EE69658
:10AC40000FB6F894DEBF0FBECDBFDF91CF911F913D
:10AC50000F91FF90EF90DF90CF90BF90AF9008954D
:10AC600081E991E1C4CFCE014C960E9428AF8BE1DF
:10AC7000FE013196DE015C9601900D928A95E1F716
:10AC8000CE0101960E947A2E72CF2F923F924F9260
:10AC90005F926F927F928F929F92AF92BF92CF926C
:10ACA000DF92EF92FF920F931F93CF93DF9300D029
:10ACB00000D000D01F921F92CDB7DEB7B82E809182
:10ACC000830D843008F0D1C10E941BA36B017C016D
:10ACD0008091830D811108C08091960C9091970C02
:10ACE000891B8F7709F4A4C681E6A82E13C08A3089
:10ACF00019F08D3009F0F6C010927E0D80911C0D78
:10AD000090911D0DFC01E85EF24F1682892BF1F443
:10AD10000E9429BE8091830D843008F0ECC08091A0
:10AD2000960C9091970C891B8F7709F4E4C00E94D0
:10AD3000375297FFDCCF0E94E44A85EB95E00E94F2
:10AD40003D358091960C8093970CE4CF10921D0DA9
:10AD500010921C0D0EE11DE0F8018191803209F482
:10AD600046C08E3409F0A9C060EB75E0C8010F94AD
:10AD7000591F4C01892B41F06EE470E0C801049624
:10AD80000F94EE29009709F4C8014AE050E070E002
:10AD900060E001960F94C91C2B013C018091180DB5
:10ADA0009091190DA0911A0DB0911B0D0196A11D46
:10ADB000B11D481659066A067B0629F060E08DE74A
:10ADC00095E0892851F16AE270E0C8010F941D2ACC
:10ADD0009C01009729F1982F901B912C992349F001
:10ADE0009150F801E90FF11D80819826F7CF8F016E
:10ADF000B3CF4AE050E070E060E0C90101960F94E3
:10AE0000C91C292D30E050E040E062177307840729
:10AE1000950751F060E08EE595E00E94D1F47ACF7D
:10AE200060E084E395E0F9CF4092180D5092190D3F
:10AE300060921A0D70921B0D8091DD068130E1F059
:10AE400067E470E0C8010F94EE290097A9F04AE08A
:10AE500050E070E060E001960F94C91C6430710509
:10AE60008105910548F483E994E00E943D3560E056
:10AE700089E894E00E94833CC0927D07D0927E07CF
:10AE8000E0927F07F092800780911E0D8B3309F4CA
:10AE900041CF8091830D843008F03CCF8091850DA7
:10AEA0008A9DC00111246EE17DE08A57924F0F9474
:10AEB000F92980E00E948BF42DCF8091D71380FF79
:10AEC000BBCF60E77CE2C8010F94591F009731F0B7
:10AED000FC01838180538A3008F0AECF60E08AE0C5
:10AEE00095E09BCF2CE13DE04EE15DE06EE77DE03B
:10AEF0000E94B61C0FCF8091D71382FFB6C01A8272
:10AF0000198271E6F72EE0E1EE2EF9E6DF2E809150
:10AF1000830D843008F0A9C00E94EE1C8111A5C0E9
:10AF200041E050E0BE016B5F7F4F8BE395E10E94F3
:10AF30007BAD0D8110E0019711F00FEF1FEF8091B5
:10AF4000431590914415A0914515B09146158093F5
:10AF5000D3139093D413A093D513B093D6130E9418
:10AF6000EE1C0F3F100749F4811107C00E94E44A0C
:10AF700083ED95E00E943D35CACF4091850D242F89
:10AF800030E00A3061F00D3051F0882309F45FC0E1
:10AF900089819A81009719F001969A83898310928A
:10AFA000900489819A81F29EF001F39EF00D1124A4
:10AFB000ED57F24FE80FF91F1382892B69F50E94B4
:10AFC00029BE0E94EE1C882309F4A1CF0E94AF5D28
:10AFD0008BE395E10E9428AF8091CE13882391F1F5
:10AFE00081508093CE138D9DC001112462E08A5E52
:10AFF000994F0E947DB4E091CE1324E0E29FF001CE
:10B000001124EE5EF94F60817181828193810E94EB
:10B0100007220E9430A77BCF1A82198281E00E940A
:10B020008BF48091D3139091D413A091D513B09148
:10B03000D61380937F0D9093800DA093810DB093D4
:10B04000820DBFCF0E9431AFE092DD0660CF4F9DF1
:10B05000A00111244A57524F9E012F5F3F4F60E9D4
:10B0600074E0802F0E94B61C52CF0E941BA36B017C
:10B070007C01B11004C080911511882351F0C09259
:10B080006811D0926911E0926A11F0926B11BB24A1
:10B09000B3948091080590910905A0910A05B0919B
:10B0A0000B050097A105B105B1F0409168115091D1
:10B0B000691160916A1170916B11840F951FA61F21
:10B0C000B71FA7019601281B390B4A0B5B0BDA014E
:10B0D000C901B7FF92C18091140290911502A0910D
:10B0E0001602B0911702892B8A2B8B2B09F099C17C
:10B0F0000E941BA34B015C018091180C811108C0B8
:10B1000020912F129091301281E0291301C080E02C
:10B110002091DD113091DE1191E089272A3A310525
:10B120000CF480E091E04091950450919604609178
:10B13000970470919804452B462B472B09F490E017
:10B14000981789F0882309F4BDC1D501C401805640
:10B150009444A24FBF4F8093950490939604A0937C
:10B160009704B09398044090250C5090260C609062
:10B17000270C7090280C20919104309192044091FA
:10B18000930450919404C301B2010F94DC1F8823EF
:10B1900019F18091950490919604A0919704B09133
:10B1A0009804409291045092920460929304709299
:10B1B0009404892B8A2B8B2B09F449C0D501C40137
:10B1C00080569444A24FBF4F809395049093960469
:10B1D000A0939704B093980480919504909196045D
:10B1E000A0919704B09198040097A105B10579F159
:10B1F000881A990AAA0ABB0AB7FC29C010929504BA
:10B2000010929604109297041092980483E396E0AB
:10B210000E943D3560E08FE196E00E94833C809182
:10B22000DF119091E0111816190624F490E080E0E7
:10B230000E94BE1E80917411909175111816190606
:10B2400034F410927511109274110E94AFBA80916B
:10B250009D0490919E04A0919F04B091A00446018A
:10B260005701881A990AAA0ABB0AD501C401B7FD79
:10B27000B9C120912F129091301240912D028091EE
:10B280002C02291323C19091F208899FC001112437
:10B29000880F892F881F990B91958D838091F308D2
:10B2A000489FC0011124880F892F881F990B919501
:10B2B0008E830E941BA369837A838B839C8340E0E7
:10B2C000BE016F5F7F4FCE0105960E94081C6D8105
:10B2D00070E089E00E9412A241E0BE016F5F7F4FE3
:10B2E000CE0105960E94081C6E8170E087E00E94E6
:10B2F00012A280911106882309F467C100912002EF
:10B3000010912102C80102972091DF113091E011C4
:10B31000281739070CF459C1809030128F82188693
:10B3200019861A861B8680912F129F80891509F431
:10B33000E7C0892D90E03CE5A32EA89EF001A99ED0
:10B34000F00D1124E950F74F458956896789708DB2
:10B35000452B462B472B81F4418D528D638D748D87
:10B36000452B462B472B41F4458D568D678D70A19B
:10B37000452B462B472BE1F12CE5B22EB89E9001D0
:10B38000B99E300D1124A9014950574F1A01FA01F5
:10B3900061817281838194810F944E294B015C01FC
:10B3A000F10161A172A183A194A10F94E11F2B016E
:10B3B0003C01F10165A176A187A190A50F94E11F41
:10B3C0009B01AC01C301B2010F949A27A50194011E
:10B3D0000F9442204B015C01288539854A855B85A5
:10B3E0000F940029181624F488869986AA86BB86AD
:10B3F0008F818F5F87708F8396CF0E94E44A609120
:10B400007B0770917C0782EE95E00E945A538AE098
:10B410000E94043540E070E060E090E080E00E942F
:10B420006C5190912F1280913012981749F0C09270
:10B430006811D0926911E0926A11F0926B1158CEA6
:10B44000BB2019F01092A10453CE0E941BA30091BF
:10B4500068111091691120916A1130916B118090DF
:10B46000140290901502A0901602B0901702080DD9
:10B47000191D2A1D3B1D601B710B820B930B97FD41
:10B48000E1CF8091A104811133CE81E08093A104AA
:10B490005F9A8091290C8E7F8093290C8A9A8091E3
:10B4A000290C8D7F8093290C8091080180958170F3
:10B4B000809306018091290C8B7F8093290C0E9438
:10B4C000A01E16CE80E090E0DC0145CE2091301227
:10B4D0005CE5259F900111242950374FF901EA5A64
:10B4E000FF4F9081899FC0011124880F892F881FE9
:10B4F000990B91958D83295A3F4FF9018081D0CEC8
:10B5000020911A0230911B0240911C0250911D02A1
:10B51000688579858A859B850F9442204B015C0163
:10B52000B801012E000C880B990B0F94E31F9B01AF
:10B53000AC01C501B4010F94A02669837A838B8383
:10B540009C8340911E0250911F02B801CE010196CA
:10B550000E94E7BD89809A80AB80BC8040909904AE
:10B5600050909A0460909B0470909C04A3019201F7
:10B57000C501B4010F94DC1F87FF16C028E431EE2B
:10B580004AE75FE3C301B2010F94422020E037EDA8
:10B5900043EA5CE30F94A026A50194010F94422096
:10B5A00069837A838B839C8369817A818B819C8177
:10B5B0006093990470939A0480939B0490939C04E5
:10B5C0000F940C28CB010E94BE1EF4E6CF0ED11CB6
:10B5D000E11CF11CC0929D04D0929E04E0929F0455
:10B5E000F092A0040E9429BE8091DD06882309F410
:10B5F000E0C180912602882309F4A3C08091DF0472
:10B6000081119FC080911511811108C08091161180
:10B61000813021F08091D71382FF93C0F894649B0E
:10B6200010C08091220290912302A0912402B09137
:10B6300025028093DF059093E005A093E105B09388
:10B64000E2056091DF057091E0058091E105909140
:10B65000E205789420E030E0A9010F94DC1F87FF19
:10B6600070C001E00093DF0480911511811167C063
:10B6700088E496E00E943D358AE00E94043584E02B
:10B680008093900C82E080937C0C81E09AE590930B
:10B690006E1380936D138EE490E0909370138093FB
:10B6A0006F1387E08093611382E88093641384E8CA
:10B6B00090E0A0E0B0E08093651390936613A093B0
:10B6C0006713B093681381E193E10E948D310E946A
:10B6D000003D0093831140E36CE876E089E798E051
:10B6E0000E94053D61E08DE698E00E94E73C1091E4
:10B6F0000C0560E0102781E498E069F48AE796E0A1
:10B700000E94503C80E30E9404358AE00E94043588
:10B7100060E08DE596E00E94503C88E696E00E944D
:10B720003D3580E30E9404358AE00E9404351123F0
:10B7300031F083E696E09093780C8093770C0E942A
:10B74000AF5D90910901892F809581701091000261
:10B750001817C9F02091D71320622093D713809334
:10B76000000290FD3FC164EF71E080E090E00E9434
:10B77000AA250E9453AF8091D71383FD7CC111117C
:10B7800033C10E94D2320E941BA36B017C01109135
:10B7900013021123F1F080910D058823D1F040911F
:10B7A000A2045091A3046091A4047091A5044601E1
:10B7B0005701841A950AA60AB70AB501A40177FDB4
:10B7C0001AC0833009F42FC10CF01EC181300CF077
:10B7D00023C1212F30E0A8EEB3E00F947426C60EEB
:10B7E000D71EE81EF91EC092A204D092A304E092D4
:10B7F000A404F092A50480911611813009F073C061
:10B800000E941BA36B017C018091AA049091AB0460
:10B81000A091AC04B091AD04A7019601281B390B8F
:10B820004A0B5B0BDA01C901B7FD3AC0D701C6016B
:10B83000805F984DAF4FBF4F8093AA049093AB04A5
:10B84000A093AC04B093AD048090A8059090A90596
:10B85000A090AA05B090AB050E94642AAB01BC0180
:10B860004093A8055093A9056093AA057093AB0572
:10B8700080918D0690918E06A0918F06B0919006D2
:10B8800088199909AA09BB09840F951FA61FB71F1C
:10B8900080938D0690938E06A0938F06B0939006AA
:10B8A0008091A6049091A704A091A804B091A90446
:10B8B00046015701881A990AAA0ABB0AD501C40190
:10B8C000B7FD11C020E8C20E2EEED21E26E3E21E06
:10B8D000F11CC092A604D092A704E092A804F092B2
:10B8E000A9040E949D500E9453360E941D3E8091E3
:10B8F0000705882379F10E941BA36B017C018091CD
:10B90000030590910405A0910505B0910605460137
:10B910005701881A990AAA0ABB0AD501C401B7FDC2
:10B9200019C02091070530E0A8EEB3E00F9474260B
:10B93000C60ED71EE81EF91EC0920305D09204055C
:10B94000E0920505F092060580E00E940DB78AE0BE
:10B950000E94043580910205882359F10E941BA39F
:10B960006B017C018091FE049091FF04A091000581
:10B97000B0910105A7019601281B390B4A0B5B0BFF
:10B98000DA01C901B7FD15C02091020530E0A8EE2B
:10B99000B3E00F947426C60ED71EE81EF91EC0929F
:10B9A000FE04D092FF04E0920005F09201050E948F
:10B9B000EEA62B960FB6F894DEBF0FBECDBFDF917B
:10B9C000CF911F910F91FF90EF90DF90CF90BF909C
:10B9D000AF909F908F907F906F905F904F903F902F
:10B9E0002F9008950E9442AF123008F0CCCE0E94F2
:10B9F000D23260E085EC96E056C083ED96E09093FD
:10BA0000780C8093770CBFCE843009F0E2CE0E9490
:10BA1000E84A8AED96E004C00E94E84A89E097E08F
:10BA20000E943D35D6CE0E94E84A82EF96E0F8CFDC
:10BA300080917D0790917E07A0917F07B09180074C
:10BA4000A7019601281B390B4A0B5B0BDA01C901D0
:10BA5000885E9340A109B109B7FD46C98DEC95E018
:10BA60000E943D35C0927D07D0927E07E0927F070D
:10BA7000F092800739C91230C8F48DE996E00E942F
:10BA80003D358AE00E9404350E94922B90E080E0D0
:10BA90000E9464531092940C1092930C1092920C8A
:10BAA00060E086EB96E00E94833C6DCE123009F098
:10BAB0006ACE0E94ADB3882379F081E00E9483B3FF
:10BAC00042EB50E063E078E08CED93E10E947BADC7
:10BAD0008CED93E10E9428AF0E94682E81118DCFDA
:10BAE0000E94522E0E9429B40E947EB34CCECF9366
:10BAF000DF9380912F1290913012891B809587706F
:10BB000019F40E944556F5CF80912F128F5F8770F0
:10BB1000A0912F129CE5A99FD0011124FD01E950AD
:10BB2000F74FEF0119929A95E9F798E09083A45F97
:10BB3000B64F90E1E1E3F2E101900D929A95E1F7C1
:10BB400020912F1290913012291303C094E6909304
:10BB50002C1280932F12DF91CF910C94802E909114
:10BB60002F1280913012981306C08091F5089091A1
:10BB7000F608892B21F080E00E944556F0CF089509
:10BB8000FC01208131814281538160914B0C709185
:10BB90004C0C80914D0C90914E0C0F9442200F94C0
:10BBA0000D2960933D1270933E1280933F12909343
:10BBB000401290912F128091301298130C94775D5F
:10BBC0000E94AF5D0E94F02840913D1250913E12BC
:10BBD00060913F127091401240930106509302060B
:10BBE000609303067093040681110C94802E0895CF
:10BBF0004F925F926F927F928F929F92AF92BF927D
:10BC0000CF92DF92EF92FF920F931F93CF93DF9328
:10BC1000EC018B015A01F90120914B0C30914C0C35
:10BC200040914D0C50914E0C6081718182819381C5
:10BC30000F9442200F940D296B017C012091470C39
:10BC40003091480C4091490C50914A0CF5016081AB
:10BC50007181828193810F9442200F940D294B01B1
:10BC60005C012091430C3091440C4091450C509163
:10BC7000460CF80160817181828193810F9442208A
:10BC80000F940D292B013C0120913F0C3091400C69
:10BC90004091410C5091420C688179818A819B814D
:10BCA0000F9442200F940D29609331127093321239
:10BCB0008093331290933412409235125092361280
:10BCC00060923712709238128092391290923A1222
:10BCD000A0923B12B0923C12C0923D12D0923E1202
:10BCE000E0923F12F092401290912F128091301208
:10BCF000981791F0DF91CF911F910F91FF90EF90E6
:10BD0000DF90CF90BF90AF909F908F907F906F907B
:10BD10005F904F900C94775D0E94AF5D0E94F02879
:10BD20004091391250913A1260913B1270913C123D
:10BD3000009135121091361220913712309138123D
:10BD4000C0903112D0903212E0903312F090341241
:10BD5000C092F505D092F605E092F705F092F8054D
:10BD60000093F9051093FA052093FB053093FC0529
:10BD70004093FD055093FE056093FF057093000608
:10BD800040913D1250913E1260913F1270914012CD
:10BD900040930106509302066093030670930406D5
:10BDA000882391F0DF91CF911F910F91FF90EF9039
:10BDB000DF90CF90BF90AF909F908F907F906F90CB
:10BDC0005F904F900C94802EDF91CF911F910F9137
:10BDD000FF90EF90DF90CF90BF90AF909F908F90AB
:10BDE0007F906F905F904F9008954F925F926F9207
:10BDF0007F928F929F92AF92BF92CF92DF92EF92FB
:10BE0000FF920F931F93CF93DF93CDB7DEB72C979D
:10BE10000FB6F894DEBF0FBECDBF2B013C012987C2
:10BE20003A874B875C8747015801F601E080F18033
:10BE30000281138120E030E0A901B701C8010F940D
:10BE4000DC1F882309F488C05E2D4F2D302F212F51
:10BE5000852F942FA32FB22F89839A83AB83BC8322
:10BE600020E030E0A901B701C8010F94DC1F811167
:10BE700008C0E0903D02F0903E0200913F02109118
:10BE80004002C701D8018D839E83AF83B887A50187
:10BE900094016091210C7091220C8091230C90915F
:10BEA000240C0F94DC1F87FF0CC08092210C909211
:10BEB000220CA092230CB092240CCE0101960E9479
:10BEC000CB294092190C50921A0C60921B0C709264
:10BED0001C0C89859A85AB85BC8580931D0C90933D
:10BEE0001E0CA0931F0CB093200CCE0105960E944F
:10BEF000CB29A50194016091210C7091220C8091B5
:10BF0000230C9091240C0F940029181664F480924D
:10BF1000210C9092220CA092230CB092240CCE0102
:10BF200001960E94CB290E94AF5D2C960FB6F89423
:10BF3000DEBF0FBECDBFDF91CF911F910F91FF905C
:10BF4000EF90DF90CF90BF90AF909F908F907F90B9
:10BF50006F905F904F90089550E040E030E820E40B
:10BF600077CFCF92DF92EF92FF920F931F936A01E8
:10BF7000E090210CF090220C0091230C1091240CE5
:10BF8000FB012081318142815381FC0160817181FB
:10BF9000828193810E94F55E1F910F91FF90EF9037
:10BFA000DF90CF900895CF92DF92EF92FF920F93A0
:10BFB0001F936B01FC01E080F18002811381E9E1B4
:10BFC000FCE02481358146815781608171818281C5
:10BFD00093810E94F55E1F910F91FF90EF90DF908B
:10BFE000CF900895AF92BF92CF92DF92EF92FF92DF
:10BFF0000F931F93CF93DF9300D01F92CDB7DEB77F
:10C00000FC01E080F18002811381611112C0A090D7
:10C01000210CB090220CC090230CD090240C9501E0
:10C02000A601B701C8010F94DC1F87FF02C075018C
:10C03000860120E030E048EC53E4B701C8010F94DA
:10C04000DC1F87FD04C0E12CF12C08EC13E4C701D0
:10C05000D80189839A83AB83BC8360EE72E0CE0102
:10C0600001960E94D35F0F900F900F900F90DF9179
:10C07000CF911F910F91FF90EF90DF90CF90BF90E5
:10C08000AF900895BF92CF92DF92EF92FF920F93FD
:10C090001F93CF93DF9300D01F92CDB7DEB7B82E9A
:10C0A000882351F180E090E0A0E2B1E489839A8393
:10C0B000AB83BC83C0902612D0902712E090281248
:10C0C000F090291220E030E0A901C701B6010F94D9
:10C0D000DC1F87FF0CC0A701960160E070E080E2E2
:10C0E00091E40F949F2669837A838B839C8360E01D
:10C0F000CE0101960E94F25F6091190C70911A0CAA
:10C1000080911B0C90911C0C20911D0C30911E0CE9
:10C1100040911F0C5091200C19821A821B821C82A4
:10C12000E090210CF090220C0091230C1091240C33
:10C13000FE0131966F010E94F55EB09279070E9470
:10C14000552A0F900F900F900F90DF91CF911F9174
:10C150000F91FF90EF90DF90CF90BF900895809166
:10C160007907882319F080E00E94426080E00895FA
:10C170002F923F924F925F926F927F928F929F92F7
:10C18000AF92BF92CF92DF92FF920F931F93CF9304
:10C19000DF93CDB7DEB760970FB6F894DEBF0FBE62
:10C1A000CDBFF82E282E312CF101E351F24D4490F1
:10C1B000042C000C5508660877086101CC0CDD1CC6
:10C1C000CC0CDD1C82E0F81609F407C1C301B201F2
:10C1D0000F94E31F2B013C01C6018A58974E0E9421
:10C1E000271D4B015C01A3019201C501B4010F940D
:10C1F00042204B015C01C6018659974E0E94271DC3
:10C2000020E030E040EC5FE30F944220A301920174
:10C210000F944220AB01BC0100E010E098018F2D8B
:10C220000F94151320E030E0A901C501B4010F946B
:10C23000DC1F882309F440C092E000E010E020E415
:10C2400031E4F91619F000E010E09801B501A401FD
:10C2500070588F2D0F941513A5019401C501B401D9
:10C260000F94A0264B015C01E2E000E010E020EC1E
:10C2700030E4FE16E1F0F101E55AF74E64916111E8
:10C2800007C00E94E84A89E398E10E943D356AE0D0
:10C2900070E090E080E00F94E11F9B01AC0160E052
:10C2A00070E088E492E40F949A278B019C01B50119
:10C2B000A4018F2D0F94151381E090E0A0E0B0E071
:10C2C0000F2C04C0880F991FAA1FBB1F0A94D2F716
:10C2D0002091290C282B2093290C20919305822B47
:10C2E00080939305C601825A974E0E94271DF6013E
:10C2F000E75EF34F6083718382839383F2E0FF12E2
:10C300001AC0209126123091271240912812509184
:10C3100029126091210C7091220C8091230C909134
:10C32000240C0F949F266093210C7093220C809311
:10C33000230C9093240CF601E551F84F10821182E2
:10C34000128213828F2D0E94441C0E94E629F6015E
:10C35000E75EF34F80819181A281B381F601E859B4
:10C36000F84F80839183A283B38382E0F81609F4A7
:10C3700062C08CE0ECEAF2E0DE01119601900D92D1
:10C380008A95E1F7E1E0F0E0EC0FFD1FEC0DFD1DFB
:10C3900080809180A280B38020E030E0A901C501B7
:10C3A000B4010F94DC1F81114BC060960FB6F89456
:10C3B000DEBF0FBECDBFDF91CF911F910F91FF90D8
:10C3C000DF90CF90BF90AF909F908F907F906F90B5
:10C3D0005F904F903F902F90089580917907811141
:10C3E00003C081E00E9442608EE798E10E94271D11
:10C3F00020E030E0A9010F94DC1F882309F4E6CE89
:10C40000C301B2010F94E31F2B013C018EE798E1B9
:10C410000E94271D4B015C0120E030E040EA50E41F
:10C420000F94DC1F87FFDFCE812C912C80EAA82E91
:10C4300080E4B82ED8CE0E94AF608111B6CF99CFDC
:10C4400020E030E0A901C501B4010F94002987FF65
:10C4500004C0B7FAB094B7F8B094F601E75EF34FB2
:10C460006F01A5019401C301B2010F9442209B0109
:10C47000AC01F60160817181828193810F949F26C6
:10C48000F6016083718382839383F2E080E090E021
:10C49000A0E4B1E4FF1621F080E090E0A8E4B2E46B
:10C4A0008D879E87AF87B88BCE010D960E94CB29D2
:10C4B0007CCFCF93DF9300D01F92CDB7DEB780E063
:10C4C00090E0A0EAB0E489839A83AB83BC8361E007
:10C4D000CE0101960E94F25F0F900F900F900F9087
:10C4E000DF91CF9108958F929F92AF92BF92CF929A
:10C4F000DF92EF92FF920F931F93CF93DF93CDB70D
:10C50000DEB72C970FB6F894DEBF0FBECDBF8B0100
:10C5100040E050E068E472E44D835E836F83788787
:10C5200040E050E060EA70E449875A876B877C8777
:10C530008130B9F1823009F459C020E030E040E0A8
:10C5400050E46091210C7091220C8091230C909109
:10C55000240C0F94A0264B017C0120E030E048EC35
:10C5600053E40F940029181634F4812C912C88EC94
:10C57000E82E93E4F92EF801A084B184C284D38418
:10C580009401A701B501C6010F940029181614F0F3
:10C5900054016701C501D60189839A83AB83BC83AB
:10C5A00048C0BE01675F7F4FC80108960E94D35FF5
:10C5B000B8016C5F7F4FAE014B5F5F4FC8010E94B7
:10C5C000B15F0E94802F2C960FB6F894DEBF0FBE8D
:10C5D000CDBFDF91CF911F910F91FF90EF90DF9032
:10C5E000CF90BF90AF909F908F900895F8012085D5
:10C5F0003185428553856091210C7091220C809188
:10C60000230C9091240C0F94A0266B017C0120E058
:10C6100030E048EC53E40F94DC1F87FD06C0C12CCA
:10C62000D12C28ECE22E23E4F22EC982DA82EB82AE
:10C63000FC82BE01675F7F4FCE010196B7CFEF92BC
:10C64000FF920F931F93CF93DF937C018B010E9486
:10C650007A30C9E1DCE020916102309162024091C0
:10C66000630250916402F70160817181828193813C
:10C670000F949A272C853D854E855F850F94A026C3
:10C680006C877D878E879F87C8010E94CB29DF91A9
:10C69000CF911F910F91FF90EF900C94AF5D4F924F
:10C6A0005F926F927F92AF92BF92CF92DF92EF92A2
:10C6B000FF920F931F93CF93DF9300D000D01F9270
:10C6C0001F92CDB7DEB75C0180E090E0A0E7B2E456
:10C6D00089839A83AB83BC8380E090E0A0E8B0ECD0
:10C6E0008D839E83AF83B887BE016F5F7F4FCE017E
:10C6F00005960E941F6368E873E180E090E00E9465
:10C70000AA25C12CD12C88ECE82E81E4F82EC98210
:10C71000DA82EB82FC8280E090E0A0E8B0E48D83D6
:10C720009E83AF83B887BE016F5F7F4FCE010596B2
:10C730000E941F630BE21CE0F80140AC51AC62ACFC
:10C7400073ACC0AED1AEE2AEF3AE80E090E0A0EA52
:10C75000B1E489839A83AB83BC83F50180819181A5
:10C76000A281B3818D839E83AF83B887BE016F5F43
:10C770007F4FCE0105960E941F63F80140AE51AE77
:10C7800062AE73AE129A64E670E080E090E00E94C0
:10C79000AA2581E028960FB6F894DEBF0FBECDBF64
:10C7A000DF91CF911F910F91FF90EF90DF90CF908D
:10C7B000BF90AF907F906F905F904F9008951F93C0
:10C7C000CF93DF93CDB7DEB72C970FB6F894DEBFCB
:10C7D0000FBECDBF182F882379F020E030E0A901EB
:10C7E0006091CB057091CC058091CD059091CE05DF
:10C7F0000F94DC1F8823F9F080912A0C8117D9F05F
:10C800000E94AF5D8CE0E8EBF2E0DE011196019052
:10C810000D928A95E1F7CE0101960E94D31E809178
:10C820002A0C882391F089E19CE00E94F225109265
:10C830002A0C0E94E6292C960FB6F894DEBF0FBE94
:10C84000CDBFDF91CF911F91089581E080932A0C95
:10C8500089E19CE00E94C020ECCF2F923F924F9242
:10C860005F926F927F928F929F92AF92BF92CF9280
:10C87000DF92EF92FF920F931F93CF93DF93CDB789
:10C88000DEB7CB54D1090FB6F894DEBF0FBECDBFD3
:10C890002DB73EB739AF28AF87E00E94F84A811123
:10C8A0000BC061E086E50E94F8238DA3853060F01F
:10C8B0008CE39DE00E943D35A8ADB9AD0FB6F8946C
:10C8C000BEBF0FBEADBF40C33DA1332321F08CE1FD
:10C8D0009DE00E943D356AE080E50E94F823182F14
:10C8E0008CEF810F8F3218F088EF9CE0E3CF60E08F
:10C8F00085E40E941424882309F448C081E08FABAA
:10C90000E0902A12F0902B12D7012D913D914D917C
:10C910005C916091190C70911A0C80911B0C909194
:10C920001C0C0F94A026AB01BC0188E50E94662474
:10C9300069877A878B879C87F701248135814681B7
:10C94000578160911D0C70911E0C80911F0C90916D
:10C95000200C0F94A026AB01BC0189E50E9466243F
:10C960006D877E878F87988BBE01635F7F4FCE0177
:10C9700009960E94202D382E81110BC063E684EEAB
:10C980009CE00E94833C8CEC9CE094CF92E09FABB7
:10C99000B7CF8CE40E94E81D082F882309F431C129
:10C9A0000E94E4238EA3803118F085EA9CE082CFB8
:10C9B000FEA1F13009F427C160E083E50E94142450
:10C9C0008AAF882321F0011102C037E03EA38DA178
:10C9D000833020F08BE89CE00E943D3590912A0C3A
:10C9E0009DAF80E00E94DF630E947D1C1D8A1E8A2D
:10C9F0001F8A188E198E1A8E1B8E1C8E83EF9FE451
:10CA0000A3ECB7E48D8F9E8FAF8FB8A383EF9FE425
:10CA1000A3ECB7EC89A39AA3ABA3BCA3A12FB0E06E
:10CA2000BCA7ABA7EDB7FEB724E0129FE019F10950
:10CA300011240FB6F894FEBF0FBEEDBF8DB79EB7A1
:10CA400001969CAF8BAF2DA14FA9BE01635F7F4FB5
:10CA5000CE0109960F941C119B01AC010F949229F1
:10CA6000811162C20E941BA36115710581059105A8
:10CA700011F00F94621B212C1BAA1CAA1DAA1EAA2E
:10CA8000AEA1A150BB0B2C96BFAFAEAF2C97E22D41
:10CA9000F0E0F8A7EFA32BA53CA5E217F3070CF0F5
:10CAA00074C23196FEA7EDA73F932F93FF93EF93A8
:10CAB00087E79CE09F938F9381E89CE09F938F93FF
:10CAC0001F920F9458108DB79EB709960FB6F89421
:10CAD0009EBF0FBE8DBF9EA1992309F458C10F942C
:10CAE000131B2AE030E040E050E00F9442260F9400
:10CAF000E31F20E030E040EA50E40F9400290FEFFC
:10CB00001FEF181614F001E010E00F94131B28E635
:10CB100031E040E050E00F9442260F94E31F2B01D8
:10CB20003C010F94131B20E230E040E050E00F94F2
:10CB300042266B5F7F4F8F4F9F4F0F94E31F4B0138
:10CB40005C01ADA1A430D1F4BC01A40189E69CE054
:10CB50000E94F13DB301A20181E69CE00E94F13DFB
:10CB60008BE59CE00E943D350130110519F483E40A
:10CB70000E94043587E59CE00E943D35312CC801B8
:10CB8000110FAA0BBB0B2A968CAF9DAFAEAFBFAFF8
:10CB90002A972C96AEADBFAD2C973A161B060CF01B
:10CBA000F6C02A966CAD7DAD8EAD9FAD2A970F94E1
:10CBB000E31F6B017C01BAADBB2341F1AC019B01CA
:10CBC0000F94A02620E030E040E952E40F94422088
:10CBD0009B01AC01C301B2010F94A0262B013C01C3
:10CBE00020E030E044EB53E40F9400291816FCF4E5
:10CBF00020E030E044EB53E4C301B2010F949F26E0
:10CC0000EDCF1EA2D9CE22E02EA3D6CE0F94131BB9
:10CC100024E130E040E050E00F944226675E7F4F11
:10CC20008F4F9F4F0F94E31FA7019601CFCF20E0B6
:10CC300030E0A901C301B2010F94DC1F87FF0BC0D4
:10CC400020E030E044EB53E4C301B2010F94A0268E
:10CC50002B013C01ECCF00912A1210912B12F8010C
:10CC600024813581468157816D857E858F859889A0
:10CC70000F949F2622966CAF7DAF8EAF9FAF229709
:10CC80002BED3FE049E450E4C301B2010F94422090
:10CC900020E030E044E353E40F949A276B017C01D9
:10CCA0000F9495276FA778AB89AB9AABD8012D91DC
:10CCB0003D914D915C9169857A858B859C850F941A
:10CCC0009F2626966CAF7DAF8EAF9FAF2697A501AE
:10CCD00094016FA578A989A99AA90F9442209B0174
:10CCE000AC0126966CAD7DAD8EAD9FAD26970F94B1
:10CCF000A02669837A838B839C83C701B6010F9436
:10CD00004029A50194010F94422022962CAD3DADFF
:10CD10004EAD5FAD22970F94A0266D837E838F83E7
:10CD200098874BE351E070E060E0CE0101960E94ED
:10CD3000E7BD46E351E070E060E0CE0105960E9459
:10CD4000E7BDBDA1B43099F449815A816B817C81E2
:10CD50008BE49CE00E94F13D4D815E816F8178857E
:10CD600080E59EE20E94F13D8AE00E940435198A26
:10CD70001A8A1B8A1C8AAE014F5E5F4FBE016B5F31
:10CD80007F4FCE0101960E94B15F339402CF20E025
:10CD90004FA9BE01635F7F4FCE0109960F941C110E
:10CDA0004B015C01312CAC019B010F949229811144
:10CDB00002C033243394A5019401C501B4010F943A
:10CDC00092298111E2C0EFA1F8A5EE0FFF1FEE0F2F
:10CDD000FF1F2BAD3CADE20FF31F80829182A28238
:10CDE000B382A50194016D8D7E8D8F8D98A10F94D6
:10CDF0000029181624F48D8E9E8EAF8EB8A2A50140
:10CE0000940169A17AA18BA19CA10F94DC1F87FFDB
:10CE100004C089A29AA2ABA2BCA2A50194016BA9ED
:10CE20007CA98DA99EA90F94A0266BAB7CAB8DAB82
:10CE30009EABADA5BEA5BD01BB0F880B990B0F9492
:10CE4000E31F6FA378A789A79AA79B01AC016BA9E1
:10CE50007CA98DA99EA90F949A272B013C014D8A8C
:10CE60005E8A6F8A788EEBADFCADF8ABEFA710E071
:10CE7000C12CD12C7601AFA5B8A96D917D918D9172
:10CE80009D91B8ABAFA7A30192010F949F269B0180
:10CE9000AC010F9442209B01AC01C701B6010F9475
:10CEA000A0266B017C011F5F211628F72FA138A552
:10CEB00049A55AA50F949A270F944E29698F7A8F06
:10CEC0008B8F9C8FBDA1B23068F18DA59EA50E946D
:10CED00022EE6BA57CA586E49CE00E94133E80E4D4
:10CEE0009CE00E943D3543E0C501B4010E9469B653
:10CEF00080E20E94043581E0EDA1E3300CF480E093
:10CF0000E12C8E010F5D1F4F9E01235E3F4FAE014E
:10CF1000475E5F4FBE016B5E7F4F0E94D23B8AE04F
:10CF20000E9404352394B3CD0E94AF600E94641C1C
:10CF30008DAD0E94DF630E94802F88AD99AD0FB642
:10CF4000F8949EBF0FBE8DBFE8ADF9AD0FB6F89453
:10CF5000FEBF0FBEEDBFC55BDF4F0FB6F894DEBF5F
:10CF60000FBECDBFDF91CF911F910F91FF90EF903A
:10CF7000DF90CF90BF90AF909F908F907F906F90F9
:10CF80005F904F903F902F9008950E94AF603320A4
:10CF900069F285E39CE00E943D3581E0FDA11F160A
:10CFA0000CF080E0EE24E3948E010F5D1F4F9E0194
:10CFB000235E3F4FAE01475E5F4FBE016B5E7F4F0A
:10CFC0000E94D23B698D7A8D8B8D9C8D0052110908
:10CFD00026E042E00F94A91A9F938F9384E29CE08D
:10CFE0009F938F938EE29CE09F938F931F920F9459
:10CFF00058102DB73EB7295F3F4F0FB6F8943EBF8C
:10D000000FBE2DBF93CF2F923F924F925F926F92A0
:10D010007F928F929F92AF92BF92CF92DF92EF92C8
:10D02000FF920F931F93CF93DF93CDB7DEB76A972D
:10D030000FB6F894DEBF0FBECDBF83E50E94E81D9A
:10D04000182F30902A0C882319F00E940424382EBF
:10D050004090190C50901A0C60901B0C70901C0C96
:10D0600080911D0C90911E0CA0911F0CB091200C72
:10D070008B8B9C8BAD8BBE8B8091210C9091220C65
:10D08000A091230CB091240C8F8B988FA98FBA8F0D
:10D09000112329F0311003C080E00E94DF6386E590
:10D0A0000E94E81D8A8B20E030E0A9016091CB0549
:10D0B0007091CC058091CD059091CE050F94DC1F29
:10D0C000882309F4C9C083E40E94E81D882309F479
:10D0D0009DC00E943C246B017C01A1E8B7E0B987A8
:10D0E000A887BF83AE83F5E0FD831D861E8628ECEE
:10D0F0002F8702EC1A86212C88EC8B8792E49C8780
:10D10000AE81BF81B98BA88B15E0E889F989819040
:10D110009190A190B190F98BE88B2A85322D4B85A7
:10D120005C85C501B4010F94DC1F87FF04C08A86AB
:10D13000292CAB86BC862D853E854F85502FC50199
:10D14000B4010F940029181624F48D869E86AF86AC
:10D150000B2D1150D1F6FD81F150FD838E819F8101
:10D1600044969F838E83F111CBCF2D853E854F85CD
:10D17000502F6A85722D8B859C850F94A02620E008
:10D1800030E040E05FE30F944220A70196010F9446
:10D19000A0264B015C012DEB37E346E855EB0F94DD
:10D1A000002987FD0AC02DEB37E346E855E3C501AA
:10D1B000B4010F94DC1F18164CF580E00E94DF6369
:10D1C00010E0E884F98400E0D7016D917D918D91A4
:10D1D0009D917D016D01B4E0CB1AD108A5019401A8
:10D1E0000F949F26F6016083718382839383602F5F
:10D1F000812F0F944B0F0F5F053031F71F5F88852C
:10D2000099854496998788871530D9F6AA89AA23E3
:10D2100081F020E030E0A9016091CB057091CC0550
:10D220008091CD059091CE050F94DC1F81110E9455
:10D230005A3D8AE50E94E81D882351F00E943C2453
:10D2400069837A838B839C83CE0101960F94130E9E
:10D25000832D0E94DF630BC0311003C09A8999238C
:10D2600041F30E94E84A85E69BE00E943D35332069
:10D2700051F080912A0C811106C00E94E44A86E494
:10D280009BE00E943D350E94E84A88E39BE00E94B3
:10D290003D3580912A0C0E94D33D0E94E84A8BE2E2
:10D2A0009BE00E943D35C090BD08D090BE08E09044
:10D2B000BF08F090C00820E030E0A901C701B60126
:10D2C0000F94002918160CF053C042E0C701B601B4
:10D2D0000E9469B68DE00E9404358AE00E94043500
:10D2E000A30192016091190C70911A0C80911B0C92
:10D2F00090911C0C0F94DC1F81111FC02B893C895D
:10D300004D895E8960911D0C70911E0C80911F0CDF
:10D310009091200C0F94DC1F81110FC02F89388D44
:10D32000498D5A8D6091210C7091220C8091230CB3
:10D330009091240C0F94DC1F81110E94802F6A961B
:10D340000FB6F894DEBF0FBECDBFDF91CF911F9116
:10D350000F91FF90EF90DF90CF90BF90AF909F9094
:10D360008F907F906F905F904F903F902F90089597
:10D3700086E29BE00E943D35B3CF8F929F92AF92A1
:10D38000BF92EF92FF920F931F93CF93DF9380E0B2
:10D390000E94DF631092C7051092C8051092C9055C
:10D3A0001092CA051092C3051092C4051092C505CB
:10D3B0001092C6051092CF051092D0051092D1059B
:10D3C0001092D2051092CB051092CC051092CD058B
:10D3D0001092CE0501E817E0C0E0812C912C80EC82
:10D3E000A82E8FE7B82E7801D0E0F70181929192B4
:10D3F000A192B1927F016D2F8C2F0F944B0FDF5FA5
:10D40000D53099F7CF5F0C5E1F4FC53061F7DF91C4
:10D41000CF911F910F91FF90EF90BF90AF909F9091
:10D420008F90089590912F1280913012981308C018
:10D430008091F5089091F608892B11F40C94A21EA6
:10D4400080E00E944556EECF2F923F924F925F921E
:10D450006F927F928F929F92AF92BF92CF92DF9204
:10D46000EF92FF920F931F93CF93DF93CDB7DEB769
:10D47000A6970FB6F894DEBF0FBECDBF88E697E043
:10D480000E9413298091D70B83FD7EC02091250C2B
:10D490003091260C4091270C5091280C6091740714
:10D4A0007091750780917607909177070F94DC1F34
:10D4B000882309F469C01091F408111161C08091AA
:10D4C0005F029091600201972091DD113091DE1191
:10D4D000281739073CF40E94E84A8CE098E10E9442
:10D4E0003D3511E02091250C3091260C4091270C00
:10D4F0005091280C609174077091750780917607A0
:10D50000909177070F949F266B017C0120E030E01B
:10D51000A9010F94002987FF04C0F7FAF094F7F8E7
:10D52000F094209161023091620240916302509127
:10D530006402C701B6010F94422020E030E84BE3BB
:10D5400054E40F9400291816ECF40E94E84A8DEE7A
:10D5500097E10E943D358091740790917507A091E5
:10D560007607B09177078093250C9093260CA093B3
:10D57000270CB093280C84E797E00E94C05D04C09C
:10D5800010E0B0CF1111E7CF2AE037ED43E25CE3C2
:10D590006091410270914202809143029091440255
:10D5A0000F9442206B017C016091670270916802C8
:10D5B000072E000C880B990B0F94E31F9B01AC0105
:10D5C000C701B6010F944220698B7A8B8B8B9C8BA1
:10D5D00080912A0C882309F18090BD089090BE08A4
:10D5E000A090BF08B090C008C0907007D09071079D
:10D5F000E0907207F090730720E030E0A901C501C8
:10D60000B4010F94DC1F8823D1F1A7019601C50155
:10D61000B4010F940029181694F1C12CD12C760175
:10D620008E010F5E1F4F24E737E040E757E06CE6BE
:10D6300077E088E697E00E94F5F480E1E8E6F7E01D
:10D64000A9E1BCE001900D928A95E1F7A6960FB68C
:10D65000F894DEBF0FBECDBFDF91CF911F910F9128
:10D66000FF90EF90DF90CF90BF90AF909F908F9002
:10D670007F906F905F904F903F902F9008952091F2
:10D68000190C30911A0C40911B0C50911C0C60919C
:10D6900068077091690780916A0790916B070F94F2
:10D6A0009F266D8B7E8B8F8B988F20911D0C3091D8
:10D6B0001E0C40911F0C5091200C60916C077091D2
:10D6C0006D0780916E0790916F070F949F26698F69
:10D6D0007A8F8B8F9C8F2091210C3091220C40915E
:10D6E000230C5091240CC701B6010F949F266D8F17
:10D6F0007E8F8F8F98A32091250C3091260C40911E
:10D70000270C5091280C60917407709175078091D7
:10D710007607909177070F949F266B017C0120E09C
:10D7200030E0A9016D897E898F89988D0F94DC1F67
:10D7300081110CC020E030E0A901698D7A8D8B8DBC
:10D740009C8D0F94DC1F882309F467CF2D893E89B7
:10D750004F89588DCA01B9010F9442204B015C01D9
:10D76000298D3A8D4B8D5C8DCA01B9010F944220F1
:10D770009B01AC01C501B4010F94A0264B015C01D3
:10D780002D8D3E8D4F8D58A1CA01B9010F944220B5
:10D790009B01AC01C501B4010F94A0264B015C01B3
:10D7A000A7019601C701B6010F9442209B01AC016D
:10D7B000C501B4010F94A0260F944E294B015C01C2
:10D7C0002DEB37E346E855E30F94DC1F87FF0FC0CE
:10D7D00020E030E0A901C701B6010F9400294601FD
:10D7E000570187FF04C0B7FAB094B7F8B0942DEB97
:10D7F00037E346E855E3C501B4010F94DC1F87FD0C
:10D800001CCF20E030E040EA51E4C501B4010F94A0
:10D810009A270F9413281B01672B19F422242394B1
:10D82000312CB10190E080E00F94E11F9B01AC012D
:10D8300060E070E080E89FE30F949A272B013C01A1
:10D84000AC019B01C501B4010F9442204B015C0166
:10D85000A30192016D897E898F89988D0F94422052
:10D860006D8B7E8B8F8B988FA3019201698D7A8D42
:10D870008B8D9C8D0F944220698F7A8F8B8F9C8F1C
:10D88000A30192016D8D7E8D8F8D98A10F94422002
:10D890006D8F7E8F8F8F98A3A3019201C701B60170
:10D8A0000F94422069A37AA38BA39CA380E1E9E1B2
:10D8B000FCE08E010F5F1F4FD80101900D928A95F9
:10D8C000E1F70E941BA32B013C0128EC420E511CE6
:10D8D000611C711C0DA31EA381E0281A310809F4F4
:10D8E00060C00E941BA38B019C0104191509260925
:10D8F000370937FD59C02B013C0128EC420E511C61
:10D90000611C711C80E00E9445562D893E894F891B
:10D91000588D69817A818B819C810F94A0266983BF
:10D920007A838B839C83298D3A8D4B8D5C8D6D81A1
:10D930007E818F8198850F94A0266D837E838F834F
:10D9400098872D8D3E8D4F8D58A169857A858B8561
:10D950009C850F94A02669877A878B879C8729A14D
:10D960003AA14BA15CA16D857E858F8598890F9426
:10D97000A0266D877E878F87988B750164018E0145
:10D980000F5E1F4F9E01235F3F4FAE01475F5F4F0A
:10D99000BE016B5F7F4F8DA19EA10E94F5F48111A6
:10D9A0009BCF750164013CCE0E9429BEAECF8F9201
:10D9B0009F92AF92BF92CF92DF92EF92FF92CF935E
:10D9C000DF938090410290904202A0904302B09079
:10D9D0004402FC01C080D180E280F38020E030E08E
:10D9E000A901C701B6010F94DC1F882341F0C09242
:10D9F0004102D0924202E0924302F0924402C0916E
:10DA00006702D091680284E690E090936802809368
:10DA10006702C0906102D0906202E0906302F090D1
:10DA2000640280E090E0A0E8BFE3809361029093FD
:10DA30006202A0936302B09364020E94246A8092FF
:10DA4000410290924202A0924302B0924402D093CB
:10DA50006802C0936702C0926102D0926202E092B3
:10DA60006302F0926402DF91CF91FF90EF90DF901C
:10DA7000CF90BF90AF909F908F9008950F931F937A
:10DA8000CF93DF9300D01F92CDB7DEB79C0108E69D
:10DA900017E090E1E9E1FCE0D80101900D929A9540
:10DAA000E1F7F9012081318142815381F8016085DC
:10DAB0007185828593850F94A026F8016087718710
:10DAC0008287938780E090E0A0EAB0E489839A831C
:10DAD000AB83BC83CE0101960E94D76C0F900F9050
:10DAE0000F900F90DF91CF911F910F9108952F927A
:10DAF0003F924F925F926F927F928F929F92AF92DE
:10DB0000BF92CF92DF92EF92FF921F93CF93DF935A
:10DB1000CDB7DEB72C970FB6F894DEBF0FBECDBFE2
:10DB20007A011901DC012D913D914D915C912D837C
:10DB30003E834F835887FB01408051806280738011
:10DB40008090190C90901A0CA0901B0CB0901C0C9B
:10DB5000A50194016D817E818F8198850F94DC1FD2
:10DB600081110EC011E0A301920160911D0C709112
:10DB70001E0C80911F0C9091200C0F94DC1F8111C2
:10DB800010E0D1012D913D914D915C9129873A870B
:10DB90004B875C87F701C080D180E280F3802091C1
:10DBA0000B0230910C0240910D0250910E02C70100
:10DBB000B6010F94DC1F882309F44EC0C0920B02FB
:10DBC000D0920C02E0920D02F0920E028091250C90
:10DBD0009091260CA091270CB091280C40911D0C1F
:10DBE00050911E0C60911F0C7091200C8092680760
:10DBF00090926907A0926A07B0926B0740936C07F6
:10DC000050936D0760936E0770936F07C092700713
:10DC1000D0927107E0927207F092730780937407B5
:10DC200090937507A0937607B093770720E030E0D4
:10DC300040E05FE36091570C7091580C8091590C53
:10DC400090915A0C0F94422069837A838B839C8332
:10DC5000CE0101960E94D76C2D813E814F8158855F
:10DC6000209368073093690740936A0750936B07C6
:10DC700040926C0750926D0760926E0770926F072A
:10DC8000D1012D913D914D915C91609174077091FE
:10DC9000750780917607909177070F94A02660937F
:10DCA0007407709375078093760790937707111127
:10DCB0002FC020E030E0A90169857A858B859C859D
:10DCC0000F94DC1F811133C060E070E088EC92E4B7
:10DCD00069837A838B839C83CE0101960E94D76CE3
:10DCE0002C960FB6F894DEBF0FBECDBFDF91CF915B
:10DCF0001F91FF90EF90DF90CF90BF90AF909F90DB
:10DD00008F907F906F905F904F903F902F900895ED
:10DD10002AEF3EE74AE25FE360915B0C70915C0C96
:10DD200080915D0C90915E0C0F944220D1CF60E009
:10DD300070E080EA91E4CCCF0F931F93CF93DF93F1
:10DD400000D000D01F921F92CDB7DEB78B01FC012F
:10DD500023A5211102C00F94DA131D821E821F8297
:10DD6000188620E030E040E05FE36091210C709184
:10DD7000220C8091230C9091240C0F94A02669838F
:10DD80007A838B839C839E012B5F3F4FAE014F5F55
:10DD90005F4F6DE17CE089E19CE00E94776D1D8220
:10DDA0001E821F82188620E030E040E05FE3F80129
:10DDB00060857185828593850F94A02669837A8317
:10DDC0008B839C83B8016C5F7F4F9E012B5F3F4F1D
:10DDD000AE014F5F5F4FC8010E94776D28960FB666
:10DDE000F894DEBF0FBECDBFDF91CF911F910F9191
:10DDF00008959B01AC01485F5F4FBC016C5F7F4F92
:10DE00000C94776D2F923F924F925F926F927F9218
:10DE10008F929F92AF92BF92CF92DF92EF92FF923A
:10DE20000F931F93CF93DF93CDB7DEB7A6970FB6AF
:10DE3000F894DEBF0FBECDBF8C011B015A87498706
:10DE40004090190C50901A0C60901B0C70901C0C98
:10DE500080901D0C90901E0CA0901F0CB090200C78
:10DE6000DB018D919D910D90BC91A02D8B8B9C8B96
:10DE7000AD8BBE8B9C01AD01C301B2010F949F26F7
:10DE80006B017C01D10114968D919D910D90BC91F7
:10DE9000A02D8F8B988FA98FBA8F9C01AD01C501E2
:10DEA000B4010F949F266B8F7C8F8D8F9E8FA985D9
:10DEB000BA858D919D910D90BC91A02D8B879C87EB
:10DEC000AD87BE879C01AD01C301B2010F949F26AF
:10DED0006F8F78A389A39AA3A985BA8514968D918B
:10DEE0009D910D90BC91A02D8F87988BA98BBA8B9B
:10DEF0009C01AD01C501B4010F949F266BA37CA3C7
:10DF00008DA39EA3A7019601C701B6010F944220DD
:10DF10006B017C012B8D3C8D4D8D5E8DCA01B9014D
:10DF20000F9442209B01AC01C701B6010F94A026BB
:10DF30004B015C012B893C894D895E896B857C8511
:10DF40008D859E850F949F262B013C012F89388D4E
:10DF5000498D5A8D6F85788989899A890F949F2672
:10DF60006B017C01A3019201C301B2010F94422015
:10DF70002B013C01A7019601C701B6010F94422075
:10DF80009B01AC01C301B2010F94A0260F944E294E
:10DF90006B017C012F8D38A149A15AA1CA01B90199
:10DFA0000F9442202B013C012BA13CA14DA15EA16D
:10DFB000CA01B9010F9442209B01AC01C301B20117
:10DFC0000F94A0269B01AC01C501B4010F94002958
:10DFD0001816B4F520E030E0A901C701B6010F948E
:10DFE000002987FF2AC0C701B601905820E030E021
:10DFF00040EA50E40F940029181614F5A101698530
:10E000007A85C8010E94026FA6960FB6F894DEBF0B
:10E010000FBECDBFDF91CF911F910F91FF90EF9079
:10E02000DF90CF90BF90AF909F908F907F906F9038
:10E030005F904F903F902F900895C701B601D6CFC3
:10E0400020E030E040E050E4C501B4010F94002925
:10E05000181624F4B101C8010E949C6E19821A821C
:10E060001B821C82BE016F5F7F4FC1010E94F96E4F
:10E070002DEC3CEC4CEC5CE3C701B6010F94422064
:10E080009B01AC01F80160817181828193810F94C1
:10E0900042206D837E838F839887D8019B968C91D5
:10E0A0009B978823C9F02AE939E949E95FE3149687
:10E0B0006D917D918D919C9117970F94422069836A
:10E0C0007A838B839C83BE016F5F7F4F88E697E0E6
:10E0D0000E94F96EF80113A6BE016B5F7F4F898520
:10E0E0009A850E94F96E90CF3F924F925F926F9205
:10E0F0007F928F929F92AF92BF92CF92DF92EF92D8
:10E10000FF920F931F93CF93DF93CDB7DEB76C973A
:10E110000FB6F894DEBF0FBECDBFDB010C91142FFC
:10E12000100F153008F067C11196DC90C22ECD0C8F
:10E13000B4E0BC1508F45FC1ED2DF0E0ED50FB4FED
:10E140008080912CB12CA12C002E04C0B694A794F1
:10E15000979487940A94D2F780FE4DC1EC2DF0E09D
:10E16000ED50FB4F8080912CB12CA12C012E04C0CE
:10E17000B694A794979487940A94D2F780FE3BC1F3
:10E18000322E642F7C014090C3055090C4056090EE
:10E19000C5057090C6058091CB059091CC05A091E6
:10E1A000CD05B091CE05898F9A8FAB8FBC8F660F4E
:10E1B000770B072E000C880B990B0F94E31F4B0174
:10E1C0005C01602F000F770B880B990B0F94E31FF6
:10E1D000298D3A8D4B8D5C8D0F944220A3019201C5
:10E1E0000F94A026A50194010F94A0266D877E8729
:10E1F0008F87988B612F110F770B880B990B0F94DA
:10E20000E31F298D3A8D4B8D5C8D0F944220A30125
:10E2100092010F94A026A50194010F949F26698373
:10E220007A838B839C834090C7055090C80560908B
:10E23000C9057090CA058091CF059091D005A09135
:10E24000D105B091D205898F9A8FAB8FBC8F632D8A
:10E25000660F770B072E000C880B990B0F94E31FAA
:10E260004B015C016D2DDD0C770B880B990B0F9426
:10E27000E31F298D3A8D4B8D5C8D0F944220A301B5
:10E2800092010F94A026A50194010F94A026698BFA
:10E290007A8B8B8B9C8B6C2DCC0C770B880B990B12
:10E2A0000F94E31F298D3A8D4B8D5C8D0F94422086
:10E2B000A30192010F94A026A50194010F949F261B
:10E2C0006D837E838F839887F70180859185A285F2
:10E2D000B38589879A87AB87BC878D8B9E8BAF8BE5
:10E2E000B88F45E351E061E070E0CE0141960E94B5
:10E2F000E7BD45E351E061E070E0CE0105960E9484
:10E30000E7BD4AE351E061E070E0CE010D960E9466
:10E31000E7BD4AE351E061E070E0CE0101960E9462
:10E32000E7BD89889A88AB88BC8827E137EB41ED47
:10E3300058EBC501B4010F94002987FD5CC023E0B0
:10E3400030E04BE953E4C501B4010F94DC1F18160B
:10E350000CF451C08D849E84AF84B88827E137EBDC
:10E3600041ED58EBC501B4010F94002987FD43C06E
:10E3700023E030E84DE953E4C501B4010F94DC1FFC
:10E380001816CCF18D809E80AF80B88427E137EBE2
:10E3900041ED58EBC501B4010F94002987FD2BC056
:10E3A00023E030E04BE953E4C501B4010F94DC1FD6
:10E3B00018160CF189809A80AB80BC8027E137EB7E
:10E3C00041ED58EBC501B4010F94002987FD13C03E
:10E3D00023E030E84DE953E4C501B4010F94DC1F9C
:10E3E00018164CF0AE014F5F5F4FBE01635F7F4F69
:10E3F000C7010E94026F6C960FB6F894DEBF0FBE85
:10E40000CDBFDF91CF911F910F91FF90EF90DF90E3
:10E41000CF90BF90AF909F908F907F906F905F90C4
:10E420004F903F9008952F923F924F925F926F923C
:10E430007F928F929F92AF92BF92CF92DF92EF9294
:10E44000FF920F931F93CF93DF93CDB7DEB7CC58D6
:10E45000D1090FB6F894DEBF0FBECDBF85E19BE0BA
:10E460000E943D3587E00E94F84A81116EC084E524
:10E470000E94361E882329F00E94292481110E94BF
:10E4800057B680E090E0A0E8BFE389839A83AB832E
:10E49000BC838D839E83AF83B8878DEC9CECACE40A
:10E4A000BEE389879A87AB87BC8780E090E0A0E2D3
:10E4B000B1E48D879E87AF87B88B8CE390E09A8B11
:10E4C000898B8DEC90E09C8B8B8B8DEC9CECACEC79
:10E4D000BEE38D8B9E8BAF8BB88F80E090E0A0EE7B
:10E4E000BFE3898F9A8FAB8FBC8F1BA61CA64AE90E
:10E4F00059E969E97EE38FE40E9466246D8F7E8F7F
:10E500008F8F98A360E083E40E94142489A360E0C5
:10E510008BE40E9414248AA382E40E94361E88237E
:10E5200081F10E942924009761F19C012852310950
:10E530002536310520F16CE870E087EE9AE00E9404
:10E54000133E82EE9AE00E943D35C457DF4F0FB66E
:10E55000F894DEBF0FBECDBFDF91CF911F910F9119
:10E56000FF90EF90DF90CF90BF90AF909F908F90F3
:10E570007F906F905F904F903F902F9008959A8B6F
:10E58000898B8CE40E94361E8823E1F00E943C2493
:10E590006B017C01C986DA86EB86FC8620E030E0E0
:10E5A000A9010F94002987FD0AC020E030E040E077
:10E5B00050E4C701B6010F94DC1F18161CF48AEB57
:10E5C0009AE0C1CF81E50E94E81D882331F1809156
:10E5D000FC049091FD04892BE9F00E943C246B011E
:10E5E0007C01CD82DE82EF82F8862DEC3CEC4CE49F
:10E5F0005DE30F94002987FD0AC020E030E040E78A
:10E6000051E4C701B6010F94DC1F181634F489E8F1
:10E610009AE099CF8EE59AE096CF83E50E94361E68
:10E620008823E9F00E943C246B017C01CD8ADE8ABC
:10E63000EF8AF88E2DEC3CEC4CEC5DE30F94002956
:10E6400087FD0AC020E030E040E050E4C701B60199
:10E650000F94DC1F18161CF487E39AE074CF80E552
:10E660000E94E81D882341F18091FC049091FD04F3
:10E67000892B19F48FEF99E066CF8BA58F5F8BA75D
:10E680000E943C246B017C01CD86DE86EF86F88AF1
:10E6900020E030E0A9010F94002987FD0AC020E0A6
:10E6A00030E048EC51E4C701B6010F94DC1F1816A6
:10E6B0001CF487ED99E047CF86E40E94361E88233C
:10E6C000E9F00E943C246B017C01C98EDA8EEB8E4E
:10E6D000FC8E20E030E040E85FE30F94002987FDE6
:10E6E0000AC020E030E040E850E4C701B6010F94D2
:10E6F000DC1F18161CF48EEA99E025CFC98CDA8C41
:10E70000EB8CFC8C8D889E88AF88B88CA701960115
:10E71000C701B6010F9442209B01AC0160E070E09C
:10E7200084E490E40F949A2729813A814B815C819B
:10E730000F9442202B013C01A5019401C501B401B5
:10E740000F944220A70196010F9442202CEE31E550
:10E7500048EB5DE30F949A279B01AC01C301B20122
:10E760000F94422069837A838B839C8388E40E9480
:10E77000361E882379F00E942924009759F09C01C5
:10E78000255A31092838310518F080E899E0DBCEA8
:10E790009C8B8B8B85E50E94E81D8823C9F00E9425
:10E7A0001BA3611571058105910511F00F94621B82
:10E7B0008091FC049091FD04892B91F00E943C24EF
:10E7C0006093F8047093F9048093FA049093FB0427
:10E7D00082E50E94E81D811108C08CE499E0B3CE67
:10E7E00060E070E088E492E4EBCF8091FC049091CB
:10E7F000FD04892B61F00E942924AD969FAF8EAF56
:10E80000AD97181619064CF088E199E09CCE2AE1E4
:10E8100030E0AD963FAF2EAFAD9789E50E94361E32
:10E82000882381F10E943C242091C5083091C608BC
:10E830004091C7085091C8080F949F266B017C0136
:10E8400088E50E94361E882331F10E943C242091E5
:10E85000C1083091C2084091C3085091C4080F9478
:10E860009F266BA37CA38DA39EA3CFA2D8A6E9A6C7
:10E87000FAA6CE0183960E94A71D811115C08EEEC7
:10E8800098E061CEC0901D0CD0901E0CE0901F0C43
:10E89000F090200CD5CF6091190C70911A0C8091DA
:10E8A0001B0C90911C0CDDCF84E40E94E81D91E0CC
:10E8B00089270E94DF6380E090E0A0EAB0E48DA7A2
:10E8C0009EA7AFA7B8AB60E0CE018D960E94F25F25
:10E8D0003091EA07CD57DF4F3883C358D0401092AC
:10E8E000EA070E94A11B8DEC98E00E943D358989C2
:10E8F0009A898A3191050CF044C08B899C890E94C9
:10E90000BE1E61E080E00E94F7B8811142C06FEF47
:10E9100082EE98E00E94833C8CA5811104C0CE0158
:10E9200001960F94DA1380E090E0A0EAB0E48093BF
:10E93000700790937107A0937207B09373071DA699
:10E940001EA61FA618AABE01635D7F4F88E697E04A
:10E950000E94F96ECD57DF4F5881C358D040509375
:10E96000EA070E94A11B8AA18111EFCD10927511B7
:10E97000109274110E94AFBA90E080E00E94BE1E17
:10E98000E4CD0E94FC2181E00E9480B78111B5CFC7
:10E99000BECF1092250C1092260C1092270C1092CC
:10E9A000280C85E29CE00E94C05D8BA5882309F4B9
:10E9B00052C020E030E040E751E460915B0C709180
:10E9C0005C0C80915D0C90915E0C0F949A276DA762
:10E9D0007EA78FA798AB80E1E9E1FCE0A8E6B7E06D
:10E9E00001900D928A95E1F72D853E854F855889D6
:10E9F0006091740770917507809176079091770701
:10EA00000F94A02660937407709375078093760720
:10EA100090937707CE018D960E94D76C2D853E8509
:10EA20004F855889609174077091750780917607BA
:10EA3000909177070F949F266093740770937507E2
:10EA400080937607909377078CA5811104C0CE013F
:10EA500001960F94DA13E3EFF4E085E0DF011D92F5
:10EA60008A95E9F780E1E9E1FCE0A8E6B7E00190EA
:10EA70000D928A95E1F789859A85AB85BC8580934F
:10EA8000700790937107A0937207B09373071DA648
:10EA90001EA61FA618AABE01635D7F4F88E697E0F9
:10EAA0000E94F96EBE01635E7F4F88E697E00E9488
:10EAB000F96E89A1882309F41CC42091190C3091A6
:10EAC0001A0C40911B0C50911C0CE5962CAF3DAFDD
:10EAD0004EAF5FAFE59780911D0C90911E0CA091F9
:10EAE0001F0CB091200CE1968CAF9DAFAEAFBFAFC5
:10EAF000E197312C212C9FEFA4969FAFA497AFEF05
:10EB0000A896AFAFA897BFEFC158DF4FB883CF57D4
:10EB1000D040EFE4C058DF4FE883C058D040F3EC5A
:10EB2000CF57DF4FF883C158D04027E4CE57DF4F8F
:10EB30002883C258D04081E090E0A0E0B0E0022CF1
:10EB400004C0880F991FAA1FBB1F0A94D2F7CC5785
:10EB5000DF4F88839983AA83BB83C458D040A3EF37
:10EB6000B4E0E796BFAFAEAFE79710E000E09101E9
:10EB7000032C000C440B550BC857DF4F28833983F7
:10EB80004A835B83C858D040C457DF4F2882CC5893
:10EB9000D040E796AEADBFADE7978D91E796BFAF9A
:10EBA000AEAFE79790E0B0E0A0E0CC57DF4F288110
:10EBB00039814A815B81C458D04082239323A423A6
:10EBC000B523892B8A2B8B2B09F024C1C857DF4F23
:10EBD000688179818A819B81C858D0400F94E31F56
:10EBE0002091CB053091CC054091CD055091CE05BB
:10EBF0000F9442202091C3053091C4054091C50572
:10EC00005091C6050F94A026EB966CAF7DAF8EAFEA
:10EC10009FAFEB97B801012E000C880B990B0F9456
:10EC2000E31F2091CF053091D0054091D10550913F
:10EC3000D2050F9442202091C7053091C80540911C
:10EC4000C9055091CA050F94A0266B017C01EB9673
:10EC50002CAD3DAD4EAD5FADEB97E5966CAD7DADAA
:10EC60008EAD9FADE5970F949F262B013C01A70128
:10EC70009601E1966CAD7DAD8EAD9FADE1970F94A1
:10EC80009F264B015C01A3019201C301B2010F94C5
:10EC900042202B013C01A5019401C501B4010F9450
:10ECA00042209B01AC01C301B2010F94A0260F9436
:10ECB0004E294B015C01EB962CAD3DAD4EAD5FADE9
:10ECC000EB976BA17CA18DA19EA10F949F262B0198
:10ECD0003C01A70196016FA178A589A59AA50F947B
:10ECE0009F266B017C01A3019201C301B2010F9425
:10ECF00042202B013C01A7019601C701B6010F94E8
:10ED000042209B01AC01C301B2010F94A0260F94D5
:10ED10004E2920E030E040E751E40F949A27A50106
:10ED200094010F94A0266B017C018090F8049090D0
:10ED3000F904A090FA04B090FB0420E030E040E831
:10ED40005FE3C501B4010F9400291816F4F4C5015E
:10ED5000B4010F940C284B015C0160E070E0CB0122
:10ED6000181419041A041B0434F40F94131BA5017E
:10ED700094010F9442260F94E31F9B01AC01B6014E
:10ED8000C7010F94A0266B017C01C158DF4F288179
:10ED9000CF57D040C058DF4F3881C058D040CF57F0
:10EDA000DF4F4881C158D040CE57DF4F5881C258FD
:10EDB000D040B601C7010F94DC1F87FF2BC0A4967B
:10EDC0000FAFA497C457DF4F3881CC58D040A896D6
:10EDD0003FAFA897EC96CFAEEC97ED96DFAEED97F0
:10EDE000EE96EFAEEE97EF96FFAEEF97C158DF4F7E
:10EDF000C882CF57D040C058DF4FD882C058D040CB
:10EE0000CF57DF4FE882C158D040CE57DF4FF8824E
:10EE1000C258D0400F5F1F4F0530110509F0B9CE21
:10EE20004FEF241A340A55E02516310409F083CE39
:10EE3000A4968FADA497E82FF0E0ED50FB4F208112
:10EE400081E090E0A0E0B0E0A8960FACA89704C0E5
:10EE5000880F991FAA1FBB1F0A94D2F7822B8083A9
:10EE6000A8969FADA8976A969FAF6A97A496AFADF4
:10EE7000A4976B96AFAF6B97EC968FADEC97ED9632
:10EE80009FADED97EE96AFADEE97EF96BFADEF97D6
:10EE90006F968CAF9DAFAEAFBFAF6F97A896BFAD6B
:10EEA000A897BF3F09F409C2A496EFADA497EF3F1E
:10EEB00009F403C26B2FBB0F770B880B990B0F94D0
:10EEC000E31F2091CB053091CC054091CD055091A9
:10EED000CE050F9442202091C3053091C405409186
:10EEE000C5055091C6050F94A026162F072F382E62
:10EEF000292E862F902FA32DB22D65968CAF9DAF16
:10EF0000AEAFBFAF6597A496FFADA4976F2FFF0F6D
:10EF1000770B880B990B0F94E31F2091CF0530914D
:10EF2000D0054091D1055091D2050F9442202091F7
:10EF3000C7053091C8054091C9055091CA050F9485
:10EF4000A0266B017C016996CCAEDDAEEEAEFFAEC5
:10EF50006997CE018F5A9F4F0E94A71D882309F4FD
:10EF6000B0C120E030E040EA50E4612F702F832DE3
:10EF7000922D0F94A0264B015C01CB01D501219667
:10EF80008CAF9DAFAEAFBFAF21972596CCAEDDAEB7
:10EF9000EEAEFFAE2597A8962FADA8972111E3C13D
:10EFA000A4963FADA4973111B3C120E030E040EA10
:10EFB00050E4C701B6010F94A0266B017C01A49612
:10EFC0004FADA497442309F4C5C1A4968FADA4976F
:10EFD00084300CF0BFC122ED422E23E5522E2BE7E8
:10EFE000622E21E4722E21968CAC9DACAEACBFACEF
:10EFF000219725968CAD9DADAEADBFAD2597A7965B
:10F000008CAF9DAFAEAFBFAFA7979C01AD01699626
:10F010006CAD7DAD8EAD9FAD69970F949F26AB967D
:10F020006CAF7DAF8EAF9FAFAB97A5019401659696
:10F030006CAD7DAD8EAD9FAD65970F949F262D96DF
:10F040006CAF7DAF8EAF9FAF2D97AB962CAD3DAD26
:10F050004EAD5FADAB9761962CAF3DAF4EAF5FAF9E
:10F060006197A50194016091190C70911A0C80911F
:10F070001B0C90911C0C0F949F264B015C01A796D2
:10F080002CAD3DAD4EAD5FADA79760911D0C70915D
:10F090001E0C80911F0C9091200C0F949F26A79618
:10F0A0006CAF7DAF8EAF9FAFA797812F902FA32D11
:10F0B000B22D8DA79EA7AFA7B8ABC9AADAAAEBAAB3
:10F0C000FCAAC984DA84EB84FC84CDAADEAAEFAA68
:10F0D000F8AE2DEC3CEC4CEC5CE3C301B2010F94B8
:10F0E000422029813A814B815C810F9442202091FA
:10F0F000250C3091260C4091270C5091280C0F9430
:10F10000A02669AF7AAF8BAF9CAFA5019401C50172
:10F11000B4010F9442204B015C01A7962CAD3DAD8C
:10F120004EAD5FADA797CA01B9010F9442209B0174
:10F13000AC01C501B4010F94A02620E030E040E00E
:10F1400050E40F9400291816ACF420E030E040E0C1
:10F150005FE3C701B6010F94A02629966CAF7DAF7F
:10F160008EAF9FAF2997BE01635C7F4FCE010196A2
:10F170000E949C6E89859A85AB85BC8529968CAF4B
:10F180009DAFAEAFBFAF2997A3961CAE1DAE1EAE0E
:10F190001FAEA397BE01615A7F4FCE01CD960E944C
:10F1A000F96E8CA58823C1F02AE939E949E95FE3C2
:10F1B0006D817E818F8198850F944220A3966CAFDC
:10F1C0007DAF8EAF9FAFA397BE01615A7F4F88E698
:10F1D00097E00E94F96E1CA6E090530CF090540C3E
:10F1E0000091550C1091560CA0904F0CB090500C03
:10F1F000C090510CD090520C9501A601B701C801E6
:10F200000F940029181614F47501860180904102AC
:10F2100090904202A0904302B09044022DEC3CEC4E
:10F220004CEC5DE3B701C8010F94422060934102AA
:10F2300070934202809343029093440240E0BE01E7
:10F24000675B7F4FCE018D960E9469C280E1E9E144
:10F25000FCE0A8E6B7E001900D928A95E1F7809274
:10F26000410290924202A0924302B092440220E0F6
:10F270004FEFBE01675A7F4FCE0101960E94747016
:10F2800020E041E0BE01675A7F4FCE0101960E9407
:10F2900074702FEF40E0BE01675A7F4FCE01019698
:10F2A0000E94747021E040E0BE01675A7F4FCE019A
:10F2B00001960E9474700E94AF5D8091960C8093BD
:10F2C000970CAD964EAD5FADAD9741505109AD96DF
:10F2D0005FAF4EAFAD97452B09F419CB6A968FAD52
:10F2E0006A9787FD14CB6B968FAD6B9787FFE1CB49
:10F2F0000ECB2BA13CA14DA15EA1E5962CAF3DAF5D
:10F300004EAF5FAFE5978FA198A5A9A5BAA5EBCBA6
:10F31000812F902FA32DB22D21968CAF9DAFAEAF34
:10F32000BFAF219720E030E040EA50E4C701B601CA
:10F330000F949F2625966CAF7DAF8EAF9FAF25971C
:10F34000A4965FADA49754300CF42FCE182D092D40
:10F350003A2C2B2C92ED492E93E5592E9BEF692EDA
:10F3600090E4792E40CEA8969FADA89794300CF4E7
:10F3700052C0A496AFADA497A4300CF120E030E0C9
:10F3800040EA50E4612F702F832D922D0F949F2619
:10F3900021966CAF7DAF8EAF9FAF219720E030E01C
:10F3A00040EA50E4C701B6010F949F266B017C012F
:10F3B000A496EFADA497E4300CF40DCECBCF812F03
:10F3C000902FA32DB22D21968CAF9DAFAEAFBFAFC6
:10F3D000219720E030E040EA50E4C701B6010F94E5
:10F3E000A02625966CAF7DAF8EAF9FAF2597A496D4
:10F3F000BFADA497B111D2CF20E030E040EA50E495
:10F40000612F702F832D922D0F949F26162F072F7B
:10F41000382E292E9FCFA496FFADA497F1110DC0D1
:10F4200020E030E040E251E4B401C5010F949F2692
:10F43000162F072F382E292ECECDA4962FADA497A8
:10F4400024309CF020E030E040E251E4B401C501FA
:10F450000F949F2621966CAF7DAF8EAF9FAF219703
:10F46000182D092D3A2C2B2CB6CD182D092D3A2C00
:10F470002B2C82ED482E83E5582E8BEF682E81E4ED
:10F48000782EB1CD2F923F924F925F926F927F92E2
:10F490008F929F92AF92BF92CF92DF92EF92FF92A4
:10F4A0000F931F93CF93DF93CDB7DEB7EA970FB6D5
:10F4B000F894DEBF0FBECDBF80912A0C888B87E504
:10F4C0000E94E81D882309F423C120E030E0A9014F
:10F4D0006091CB057091CC058091CD059091CE05C2
:10F4E0000F94DC1F811108C00E94E44A82E19CE075
:10F4F0000E943D3510E01FC18AE50E94361E882318
:10F5000039F10E943C242091C9083091CA084091E9
:10F51000CB085091CC080F949F266B017C0120E012
:10F5200030E040E251ECC701B6010F94002987FD9D
:10F530000AC020E030E040E251E4C701B6010F9478
:10F54000DC1F181674F40E94E44A85E09CE0D0CFDA
:10F55000C090210CD090220CE090230CF090240C51
:10F56000DECF40E050E060EC7FE788E50E94662453
:10F570002091C1083091C2084091C3085091C4083D
:10F580000F949F262B013C0140E050E060EC7FE7A8
:10F5900089E50E9466242091C5083091C6084091F3
:10F5A000C7085091C8080F949F264B015C016FEF6C
:10F5B00089E40E94F823182F6FEF8AE40E94F82351
:10F5C000082FA3019201C301B2010F949229811166
:10F5D0006EC0A5019401C501B4010F949229811157
:10F5E00066C08BA19CA1ADA1BEA18FA798ABA9AB12
:10F5F000BAAB2091C3053091C4054091C505509127
:10F60000C605C301B2010F949F262B013C0120E0E7
:10F6100030E040E05FE36FA578A989A99AA90F942B
:10F6200042209B01AC01C301B2010F94A0262FA57B
:10F6300038A949A95AA90F949A270F940C28162F74
:10F640004FA058A469A47AA42091C7053091C80599
:10F650004091C9055091CA05C501B4010F949F2678
:10F660004B015C0120E030E040E05FE3C301B20108
:10F670000F9442209B01AC01C501B4010F94A02658
:10F68000A30192010F949A270F940C28062F812F23
:10F69000012E000C990B97FD33C005979CF5802F28
:10F6A000002E000C990B97FD2FC005977CF51530A7
:10F6B00008F020CF053008F01DCF80E00E94DF6306
:10F6C00095E01902F0011124E00FF11D07FDFA95F4
:10F6D000EE0FFF1FEE0FFF1FEF57F84FC082D182D2
:10F6E000E282F382602F812F0F944B0F88890E9452
:10F6F000DF638889882309F4FDCE0E94802FFACE2B
:10F7000010E0CDCF14E0CBCF00E0D1CF04E0CFCFDD
:10F710008AE40E94E81D182F811127C070E060E084
:10F7200086E50E942D249A838983059708F180EE4F
:10F730009BE00E943D35812FEA960FB6F894DEBF1C
:10F740000FBECDBFDF91CF911F910F91FF90EF9032
:10F75000DF90CF90BF90AF909F908F907F906F90F1
:10F760005F904F903F902F9008950E94BD69C2CE48
:10F7700060E084E40E9414248F8740E050E0BA01E6
:10F780008AE50E9466246BA77CA78DA79EA740E010
:10F7900050E86BE376E483E50E94662420E030E0E5
:10F7A00040E752E40F949A2760933D0270933E0223
:10F7B00080933F0290934002E0902A12F0902B1227
:10F7C000D7018D909D90AD90BC9020E030E0A901D4
:10F7D000C501B4010F94A0266FAB78AF89AF9AAF83
:10F7E00020E030E040E251E40F94DC1F87FF06C0C8
:10F7F0001FAA18AEB0E2B9AFE1E4EAAF20E030E80A
:10F800004DE953E4C501B4010F94A0266FA7672EFC
:10F810008BAB9CAB20E030E041E953E40F9400292E
:10F82000181634F41FA6612CF1E9FBAB23E42CABD2
:10F83000D70114968D909D90AD90BC90179720E0C5
:10F8400030E0A901C501B4010F94A026D62EE72E01
:10F85000F82E092F20E030E040EA51E40F94DC1F3D
:10F8600087FF05C0D12CE12CF0EAFF2E01E420E057
:10F8700030E04BE953E4C501B4010F94A026B62E45
:10F88000C72E8DAB9EAB20E030E04CE853E40F94E4
:10F890000029181634F4B12CC12CBCE8BDABE3E44C
:10F8A000EEAB88E40E94E81D882309F410C20E9490
:10F8B0003C240F940C281B0177FF02C06F5F7F4F21
:10F8C000759567957195619571096A567F4F072EF9
:10F8D000000C880B990B0F94E31F762E872E982E21
:10F8E000A92E2D2D3E2D4F2D502F0F940029181687
:10F8F0001CF4D72C74010A2D2FA938AD49AD5AAD8F
:10F90000672D782D892D9A2D0F940029181624F033
:10F910007FA888AC99ACAAAC872D982DA92DBA2DBB
:10F920008B8B9C8BAD8BBE8B8D2D9E2DAF2DB02FD9
:10F930008F8B988FA98FBA8FB101330C880B990BDD
:10F940000F94E31F1B012C01AC019B016D2D7E2D3B
:10F950008F2D902F0F94A026D62EE72EF82E092F4C
:10F960002B2D3C2D4DA95EA90F94DC1F87FF04C0F1
:10F97000BD2CCE2CFDAA0EABA2019101672D782DD6
:10F98000892D9A2D0F94A026D62EE72EF82E092F1A
:10F990002FA5362D4BA95CA90F94DC1F87FF04C04F
:10F9A000DFA66E2CFBAA0CAB8FA5962DABA9BCA92C
:10F9B0008B8F9C8FAD8FBE8F8B2D9C2DADA9BEA93B
:10F9C0008F8F98A3A9A3BAA3BE01695E7F4FCE0112
:10F9D00043960E94202D882309F4AAC1BE01615ECE
:10F9E0007F4FCE014B960E94202DE82E882309F4EC
:10F9F0009FC12F89388D498D5A8D6F8D78A189A12E
:10FA00009AA10F949F2620E030E040E85EE30F9437
:10FA100042204B015C012B893C894D895E896B8DAD
:10FA20007C8D8D8D9E8D0F949F2620E030E040E8E8
:10FA30005EE30F9442206BA37CA38DA39EA38FA2B1
:10FA400098A6A9A6BAA689819A811816190674F4EF
:10FA50008EEA9BE00E943D358F85882321F084EA61
:10FA60009BE00E943D358AE00E9404350E94AF5D14
:10FA70000E947D1C80E00E94DF63809179078111E4
:10FA800003C081E00E9442602091CB053091CC05FB
:10FA90004091CD055091CE056BA17CA18DA19EA179
:10FAA0000F94DC1F811130C02091CF053091D0051B
:10FAB0004091D1055091D2056FA178A589A59AA54D
:10FAC0000F94DC1F811120C02091C3053091C40523
:10FAD0004091C5055091C6056B897C898D899E89A9
:10FAE0000F94DC1F811110C02091C7053091C8050B
:10FAF0004091C9055091CA056F89788D898D9A8D7D
:10FB00000F94DC1F8823A9F00E94BD6988E0FE01E4
:10FB1000B396ABECB5E001900D928A95E1F788E0E1
:10FB2000FE017396A3ECB5E001900D928A95E1F782
:10FB3000188A60E085E40E941424882309F4FBC03D
:10FB4000F1E0FFA71B861C861D861E861A8A9E2C46
:10FB500044E7C42E4BE0D42E52E8A52E5BE0B52E30
:10FB60001A8915300CF0F7C06B857C858D859E85D4
:10FB70009B01AC010F9492298111EDC0992009F4E9
:10FB8000DDC031E03BAB35E0232E91E09926F12E2C
:10FB9000FF0CFF0CF10EF394898B19896A891215F9
:10FBA00009F4D5C0062E000C770B880B990B0F9427
:10FBB000E31F2FA138A549A55AA50F9442202F89EC
:10FBC000388D498D5A8D0F94A0262B013C01612F51
:10FBD000110F770B880B990B0F94E31F2BA13CA1FE
:10FBE0004DA15EA10F9442202B893C894D895E89ED
:10FBF0000F94A0266B837C838D839E834F825886CF
:10FC000069867A8689819A81892B79F06F2D80E9BE
:10FC10009BE00E94E93D69E170E08EE89BE00E9474
:10FC2000133E8BE89BE00E943D351F9299E19F9324
:10FC30001F92FF92DF92CF92BF92AF921F920F94CA
:10FC4000581029814FA5BE01695F7F4FCE010396F1
:10FC50000F941C112B013C014B865C866D867E86C1
:10FC60000FB6F894DEBF0FBECDBFAC019B010F9461
:10FC70009229811169C089883A8825E0382D32039C
:10FC800080011124030D111D37FC1A95000F111F5F
:10FC9000000F111F0F57184FA30192016BA57CA5F0
:10FCA0008DA59EA50F94A026D8016D937D938D936D
:10FCB0009C931397632D882D0F944B0F188A81E026
:10FCC0000E944556F3948989BBA98B0F65CF4D2DB2
:10FCD0005E2D6F2D702F86E40E9466241B012C017F
:10FCE0004FA958AD69AD7AAD8CE40E9466246B8B48
:10FCF0007C8B8D8B9E8B2F8A388E498E5A8E4B2D06
:10FD00005C2D6DA97EA982E40E9466246B017C01B2
:10FD10004FA5562D6BA97CA982E50E9466246B8FA6
:10FD20007C8F8D8F9E8FCF8ED8A2E9A2FAA24CCE67
:10FD300084EC9BE0FECC22E02FA704CF8FEF8BABAF
:10FD400022242A9484E021CF88890E94DF638A8953
:10FD50008F5F8A8B05CF0E94D4F10E94AF60882309
:10FD600059F088890E94DF6380E090E0A0ECBFE753
:10FD70008B879C87AD87BE876B857C858D859E85AF
:10FD80009B01AC010F949229811159C08F8581117B
:10FD900026C082E0F82E02E094E0C92E12E0DC2CAE
:10FDA000D11A21E041E0612F802F0E94152221E02D
:10FDB0004FEF612F8F2D0E9415222FEF41E06D2D07
:10FDC000802F0E9415222FEF4FEF6D2D8F2D0E9457
:10FDD0001522115020F70150F3940F3FF9F60E94BD
:10FDE0005A3D0E94431E8F85811124C081E29CE010
:10FDF0000E942D1D4B015C0189E19CE00E94D31EF5
:10FE00009B01AC01C501B4010F9442209B01AC01E0
:10FE10006091210C7091220C8091230C9091240C04
:10FE20000F949F266093210C7093220C8093230CD7
:10FE30009093240C8F858111E888E0922A0C0E940F
:10FE4000641C80912A0C81110E94E6290E9459624B
:10FE50000E94802F6B857C858D859E8511E09B019E
:10FE6000AC010F949229811166CC44CB8F929F9262
:10FE7000AF92BF92CF92DF92EF92FF920F931F93B8
:10FE8000CF93DF9300D01F92CDB7DEB75C016B013B
:10FE90007A01122F0023E1F10E94E84A8DE998E0EF
:10FEA0000E943D3561E0812F0E94093790900D0539
:10FEB00083E080930D0581E08093180C0E94003D43
:10FEC00082E08093831140E36DE878E089E798E071
:10FED0000E94053D40E06EE170E182E798E00E94FB
:10FEE000053D61E08DE698E00E94E73C8FE798E0F1
:10FEF0000E94D1218091180C882341F060E0812F6D
:10FF00000E94093781E00E944556F4CF90920D057A
:10FF100020E030E0A901F501608171818281938147
:10FF20000F94DC1F882371F080E090E0A0ECB0E437
:10FF300089839A83AB83BC83BE016F5F7F4FC5010A
:10FF40000E941F6320E030E0A901F6016081718109
:10FF5000828193810F94DC1F882351F18090630C80
:10FF60009090640CA090650CB090660C80E090E0DE
:10FF7000A0E7B1E48093630C9093640CA093650CAC
:10FF8000B093660C80E090E0A0EAB1E489839A83A4
:10FF9000AB83BC83BE016F5F7F4FC6010E941F63AE
:10FFA0008092630C9092640CA092650CB092660CE7
:10FFB00020E030E0A901F7016081718182819381A5
:10FFC0000F940029181674F480E090E0A0E4B0E4E7
:10FFD00089839A83AB83BC83BE016F5F7F4FC70168
:10FFE0000E941F638091DF042EE130E1882311F02D
:10FFF0002EE438E04CE558E066E678E081E00E94C7
:020000021000EC
:10000000283D0E94003D81E00F900F900F900F90CF
:10001000DF91CF911F910F91FF90EF90DF90CF90E4
:10002000BF90AF909F908F900895CF93C82F8091ED
:10003000D70B83FD14C08091F408811110C080910A
:100040005F02909160029C01215031094091DF11C3
:100050005091E0114217530714F40E94BE1ECC23A6
:1000600029F061E080E0CF910C94F7B88091F4081A
:1000700091E0892780933C0280913C02882389F09B
:100080008091DD119091DE112091DF113091E0110E
:10009000821B930B97FF03C091958195910902975D
:1000A00044F410923C028091D70B83FF06C0C1E05C
:1000B0001AC080E00E944556DFCFC091F408C111FC
:1000C00012C080915F029091600201972091DF1130
:1000D0003091E0112817390754F70E94E84A80E36D
:1000E00098E00E943D358C2FCF910895AF92BF923A
:1000F000CF92DF92EF92FF920F931F93CF93DF93F4
:10010000CDB7DEB764970FB6F894DEBF0FBECDBF94
:100110000E94E74B87FDAFC08AE50E94361E882308
:1001200009F4BAC040E050E0BA018AE50E946624B2
:100130007B018C012091210C3091220C4091230CE9
:100140005091240C60E070E088EC93E40F949F26BB
:100150005B016C019701A8010F940029181614F097
:100160007501860120E030E0A901B701C8010F94B4
:100170000029181624F4E12CF12C00E010E0B7015E
:10018000C8010F940C28072E000C880B990B0F94B4
:10019000E31F698B7A8B8B8B9C8B20E030E0A9016D
:1001A0000F94DC1F882321F0CE0141960E943E6D02
:1001B00080E090E0A0EAB1E48D879E87AF87B88B9E
:1001C00019861A861B861C868CE40E94E81D8823EB
:1001D00009F467C00E943C246B017C0120E030E000
:1001E000A901C701B6010F94002987FF04C0F7FADF
:1001F000F094F7F8F094CD82DE82EF82F8862091B9
:10020000DF113091E0112430310574F08091DD115F
:100210009091DE11821B930B97FF03C091958195FE
:10022000910901E004970CF400E080E00E94158041
:10023000882359F022E0AE01435F5F4FBE016B5F40
:100240007F4FCE0109960E94367F69897A898B8912
:100250009C898B019C01305809831A832B833C8332
:1002600020E030E0A9010F94DC1F882321F0CE01AB
:1002700001960E943E6D64960FB6F894DEBF0FBEE5
:10028000CDBFDF91CF911F910F91FF90EF90DF9045
:10029000CF90BF90AF900895E12CF12C00E211E4D3
:1002A00049CFC090BE05D090BF05E090C005F0904A
:1002B000C10594CF7F928F929F92AF92BF92CF92BF
:1002C000DF92EF92FF920F931F93CF93DF9300D0B3
:1002D00000D01F921F92CDB7DEB76C015B014A01BF
:1002E000722E780100910B060E94CA1E8091DF11C8
:1002F0009091E0118E159F051CF4C7010E94BE1E4F
:1003000080E00E941580882331F0272DA401B501DB
:10031000C6010E94367F1E141F043CF4C7010E94D0
:10032000BE1E60E080E00E94F7B881E00E94158068
:1003300080E090E0A0E7B2E489839A83AB83BC833A
:1003400080E090E0A0E8B0EC8D839E83AF83B88717
:10035000BE016F5F7F4FCE0105960E941F6387E04D
:100360000E94FD28811158C08091210C9091220C8F
:10037000A091230CB091240C4091E7045091E80423
:100380006091E9047091EA04C090E304D090E40421
:10039000E090E504F090E604C0926807D092690707
:1003A000E0926A07F0926B0740936C0750936D07D9
:1003B00060936E0770936F07809370079093710737
:1003C000A0937207B093730780E090E0A8E4B2E4D2
:1003D00089839A83AB83BC83CE0101960E94D76C3C
:1003E0008091EB049091EC04A091ED04B091EE04A7
:1003F0008093700790937107A0937207B09373076F
:1004000080E090E0A0EAB0E489839A83AB83BC8368
:10041000CE0101960E94D76CC12CD12C80E7E82E2A
:1004200082E4F82EC982DA82EB82FC8280E090E0DE
:10043000A0E8B0E48D839E83AF83B887BE016F5F71
:100440007F4FCE0105960E941F6320E030E0A90196
:100450006091EF047091F0048091F1049091F204A6
:100460000F94DC1F87FF0BC0C982DA82EB82FC820B
:10047000BE016F5F7F4F8FEE94E00E941F638091FB
:10048000EF049091F004A091F104B091F2048093F4
:10049000250C9093260CA093270CB093280C8093E6
:1004A000740790937507A0937607B093770784E756
:1004B00097E00E94C05D8091C20581110F94910E5A
:1004C00061E08CEB98E00E94503C809115118150C6
:1004D0008093151142E557E164EC78E085E00E94D5
:1004E000E2EF80911511882339F00E9430A78091A6
:1004F00015118150809315118091E204882351F0E9
:100500001092E2048091E0048093F2088091E1046B
:100510008093F3080E947A3080911611823011F492
:100520000E944B350E94D4F128960FB6F894DEBF96
:100530000FBECDBFDF91CF911F910F91FF90EF9034
:10054000DF90CF90BF90AF909F908F907F90089555
:10055000CF92DF92EF92FF920F931F93CF93DF938F
:1005600000D01F92CDB7DEB77C016B018A0161E03C
:1005700081E498E00E94503C42E557E168E478E06D
:1005800085E00E94E2EF9091151181E0890F809340
:1005900015118091D71382FF06C08B7F8093D713EC
:1005A0009E5F909315110E94153680E1E9E1FCE011
:1005B000A3EEB4E001900D928A95E1F70E94AF5D41
:1005C0008091E20481110FC081E08093E204809168
:1005D000F2088093E0041092F2088091F30880936F
:1005E000E1041092F30820E030E0A901F7016081F6
:1005F0007181828193810F94DC1F8823F1F08091B7
:10060000F40881110CC080915F0290916002019703
:100610002091DD113091DE112817390774F080E048
:1006200090E0A0E7B2E489839A83AB83BC83BE01E8
:100630006F5F7F4FC7010E941F6387E00E94FD2804
:10064000811103C0B6010E94736220E030E0A9016D
:10065000F80160817181828193810F94DC1F88236E
:1006600041F080E00E941580882319F0C8010E94A3
:100670004F63129A64E670E080E090E00E94AA2541
:1006800081E00F900F900F900F90DF91CF911F910D
:100690000F91FF90EF90DF90CF900895CF92DF926F
:1006A000EF92FF92CF93DF936B017C01D42FC09127
:1006B0000D0583E080930D0581E08093180CC11433
:1006C000D104E104F10431F00E941BA3C60ED71E31
:1006D000E81EF91E8091180C882389F0C114D104FA
:1006E000E104F10421F48D2F0E944556F3CF0E94BE
:1006F0001BA36C197D098E099F0997FDF4CF1092F9
:10070000180CC0930D05DF91CF91FF90EF90DF9013
:10071000CF9008950F931F93CF93DF93C82F162F79
:100720000E94E84AC11194C0C4E9D7E0CE010E94FA
:100730003D3561E0812F0E9409370E941BA3685359
:1007400070458F4F9F4F6093070670930806809304
:10075000090690930A0610920B0600910D0583E09E
:1007600080930D0530E020E04EE150E162E278E058
:1007700082E00E94283D82E298E00E94D12181E03F
:100780008093180C8091180C882309F464C060E0F1
:10079000812F0E94093780910B06882309F454C0E9
:1007A0000E94E84A88E098E00E943D3530E020E071
:1007B00042EF57E069EF77E082E00E94283D89EF41
:1007C00097E00E94D12141E060E070E0CB010E94FF
:1007D0004E8330E020E050E040E065EE77E085E0D9
:1007E0000E94283D85EE97E00E94A0320E94CA1E1A
:1007F00080E00E9415800E94E84ACE010E943D35AB
:100800000E941BA3685370458F4F9F4F609307064C
:10081000709308068093090690930A0610920B06BF
:1008200030E020E04EE150E169ED77E082E00E94A7
:10083000283D88EC97E00E94D12181E08093180C3C
:1008400061E0812F0E94093781E00E9445569ACFCE
:10085000C9EAD7E06BCF00930D05DF91CF911F91CF
:100860000F910895CF92DF92EF92FF920F931F9313
:10087000CF93DF93CDB7DEB7A0970FB6F894DEBF66
:100880000FBECDBF0E94E74B87FDCCC085E40E9420
:10089000E81D882309F4D5C00E943C246B017C012B
:1008A00020E030E0A9010F94002987FF04C0F7FA87
:1008B000F094F7F8F094F7FAF094F7F8F094CD8EFE
:1008C000DE8EEF8EF8A28CE0E4ECF2E0DE01119611
:1008D00001900D928A95E1F78AE50E94361E8823E1
:1008E00051F040E050E0BA018AE50E946624698731
:1008F0007A878B879C8788E50E94361E882351F073
:1009000040E050E0BA0188E50E94662469837A835A
:100910008B839C8389E50E94361E882351F040E03A
:1009200050E0BA0189E50E9466246D837E838F833F
:10093000988785E50E94E81D882309F489C00E94F4
:100940003C246B017C0120E030E0A901C701B60125
:100950000F94002987FF04C0F7FAF094F7F8F09499
:10096000F7FAF094F7F8F094C98EDA8EEB8EFC8EDD
:100970001D8A1E8A1F8A188E8CE40E94E81D882317
:1009800009F46FC00E943C246B017C0120E030E040
:10099000A901C701B6010F94002987FF04C0F7FA27
:1009A000F094F7F8F094C98ADA8AEB8AFC8A62E05C
:1009B00070E082E40E942D24F82E8091151181119F
:1009C00031C021E0AE01475E5F4FBE016F5F7F4FD8
:1009D000CE014D960E94A882882321F16F2D81E0DF
:1009E0000E948A8382E50E94361E882309F442C051
:1009F0000E94292440E050E060EA71E44D875E8760
:100A00006F87788B20911511222361F08C012F2D97
:100A1000AE01435F5F4FBE016F5E7F4FCE014596D3
:100A20000E945A81A0960FB6F894DEBF0FBECDBFCC
:100A3000DF91CF911F910F91FF90EF90DF90CF90BA
:100A40000895C12CD12C80E8E82E80E4F82E33CF15
:100A5000C090BA05D090BB05E090BC05F090BD05F4
:100A600072CFC090BE05D090BF05E090C005F09059
:100A7000C1058CCF90E080E0BDCFCF92DF92EF92A6
:100A8000FF920F931F93CF93DF93CDB7DEB76C9791
:100A90000FB6F894DEBF0FBECDBF8CE40E94E81DF8
:100AA000882309F4B0C00E943C246B017C0120E043
:100AB00030E0A9010F94002987FF04C0F7FAF094F1
:100AC000F7F8F094F7FAF094F7F8F094C98EDA8E0C
:100AD000EB8EFC8E8CE0E4ECF2E0DE0111960190EE
:100AE0000D928A95E1F788E50E94361E8823A1F0D1
:100AF00040E050E0BA0188E50E9466242091C108D8
:100B00003091C2084091C3085091C4080F949F26A9
:100B100069837A838B839C8389E50E94361E8823B0
:100B2000A1F040E050E0BA0189E50E9466242091DE
:100B3000C1083091C2084091C3085091C4080F9475
:100B40009F266D837E838F8398878AE50E94361E59
:100B5000882351F040E050E0BA018AE50E94662403
:100B600069877A878B879C871D861E861F86188AD1
:100B700080911511811138C020E0AE01435F5F4FB5
:100B8000BE016F5F7F4FCE0149960E94A8828823E5
:100B900059F18091C20581110F94910E60E080E0BF
:100BA0000E948A83898D9A8DAB8DBC8DB0588D8BB8
:100BB0009E8BAF8BB88F198A1A8A1B8A1C8A1D8656
:100BC0001E861F86188A80911511882369F010E00F
:100BD00000E020E0AE014B5E5F4FBE016F5E7F4FD5
:100BE000CE010D960E945A816C960FB6F894DEBF26
:100BF0000FBECDBFDF91CF911F910F91FF90EF906E
:100C0000DF90CF900895C12CD12C80E8E82E80E4AD
:100C1000F82E58CF2F923F924F925F926F927F9211
:100C20008F929F92AF92BF92CF92DF92EF92FF92FC
:100C30000F931F93CF93DF93CDB7DEB7E5970FB632
:100C4000F894DEBF0FBECDBF8DAB20910D052CAB50
:100C500021E020930D0580912B058D3409F401C608
:100C6000843511F40C94199B873409F091C180915B
:100C7000290590912A058B31910509F4DDC108F011
:100C800079C18430910508F030C12091DD068230B1
:100C9000910508F48EC1213009F091C111E002974D
:100CA00009F010E00E947D2419821A821B821C82A6
:100CB0001D821E821F82188682E50E94361E8823AE
:100CC00009F490C10E943C246B017C0120E030E0DB
:100CD000A9010F94DC1F882309F4EAC04090190C85
:100CE00050901A0C60901B0C70901C0C80911D0C85
:100CF00090911E0CA0911F0CB091200C8CA79DA769
:100D0000AEA7BFA78090680790906907A0906A0778
:100D1000B0906B0780916C0790916D07A0916E0762
:100D2000B0916F0788AB99ABAAABBBABA50194019F
:100D3000C301B2010F94DC1F81110DC028A939A98C
:100D40004AA95BA96CA57DA58EA59FA50F94DC1F64
:100D5000882309F4ADC0A3019201C501B4010F9429
:100D60009F2620E030E040E05FE30F94422068A738
:100D700079A78AA79BA72CA53DA54EA55FA568A925
:100D800079A98AA99BA90F949F2620E030E040E032
:100D90005FE30F9442202B013C0120E030E0A901E9
:100DA000C701B6010F94DC1F881F8827881F1817FA
:100DB00009F40FC180E090E0A0E8BFEB8CA79DA7ED
:100DC000AEA7BFA728A539A54AA55BA5CA01B90149
:100DD0000F9442204B015C01A3019201C301B201B7
:100DE0000F9442209B01AC01C501B4010F94A026D1
:100DF0000F944E294B015C01AC019B01C701B60168
:100E00000F949F2668AB79AB8AAB9BABA50194018D
:100E1000C701B6010F94A0269B01AC0168A979A96E
:100E20008AA99BA90F9442206B017C0120E030E04D
:100E3000A9010F94002987FDD1C0C701B6010F9405
:100E40004E296B017C01C301B2019058A5019401A8
:100E50000F949A272CA53DA54EA55FA50F9442207F
:100E6000A70196010F94422028A539A54AA55BA5A4
:100E70000F94A02669837A838B839C83A5019401B8
:100E800068A579A58AA59BA50F949A272CA53DA5B1
:100E90004EA55FA50F944220A70196010F94422012
:100EA000A30192010F94A0266D837E838F83988780
:100EB00020E030E0A90169817A818B819C810F94C7
:100EC000DC1F8111A3C020E030E0A9016D817E818B
:100ED0008F8198850F94DC1F811198C00E94E44A8D
:100EE00080EC9EE00E943D356AC08531910509F491
:100EF00066C08A31910509F49CC0049709F048C086
:100F000080E50E94361EC12CD12C7601882321F069
:100F10000E94B6236B017C0183E50E94361E882364
:100F200061F00E943C2420E030E04AE754E40F9452
:100F300042200F9413286B017C010E94AF5D8091C9
:100F40001711811105C060E086ED9EE00E94833C90
:100F50000E941BA3C60ED71EE81EF91E0E941BA3EB
:100F60006C197D098E099F0997FF29C080E00E94B6
:100F70004556F4CF8A32910509F4E8C260F48D3108
:100F8000910509F411C208F470C04E9709F464C2C7
:100F90000F94DF1014C08B35910509F4BAC38C355A
:100FA000910509F4BAC38A35910591F71092E507C6
:100FB00006C0213021F40E947D240E94246A3DA9AC
:100FC000311102C00F948C108CA980930D050C94E4
:100FD000DF9380E090E0A0E8BFE3F0CEC12CD12CFD
:100FE000760131CF89E40E94361E882331F00E94B9
:100FF0003C2469837A838B839C838AE40E94361E17
:10100000882309F455CF0E943C244ECF412FBE01C6
:101010006F5F7F4F88E697E00E9469C20E941BA322
:10102000609368117093691180936A1190936B11AA
:10103000C6CF0E941372C3CF87E00E94F84A811185
:10104000BECF8CE0E0EDF2E0DE01119601900D9252
:101050008A95E1F770E060E080E50E94D623BE014A
:101060006F5F7F4F0E947362AACF87E00E94FD28C6
:10107000811106C060E08FE40E94142481119FCF8B
:101080000E94AF5D1092460260912A0C8CE40E948F
:101090001424E82E80E00E94DF630E941BA360936B
:1010A00068117093691180936A1190936B110E947B
:1010B0007D1C81E080939A060E94552A8AE50E9451
:1010C000E81DF82E882369F081E00E94FD28182F82
:1010D00082E00E94FD2811110C943C9B11E08111CB
:1010E00001C010E088E50E94E81D81110C942E9B40
:1010F000111141C189E50E94E81D082F811307C025
:10110000012FF11204C011E001E0FF24F39482E505
:101110000E94361E882309F431C10E943C246CA32E
:101120007DA38EA39FA320E030E0A9010F94DC1FD4
:10113000882361F0111105C0011103C0FF2009F4DB
:101140000CC160E0CE0184960E94F25F112309F485
:101150007FC0002309F479C01092190C10921A0C68
:1011600010921B0C10921C0C10921D0C10921E0C55
:1011700010921F0C1092200C0E94E6298AE698E13A
:101180000E94271D4B015C018EE698E10E94271DFD
:101190002B013C01AC019B01C501B4010F94002956
:1011A00018160CF0F0C0A5019401C301B2010F9410
:1011B0009A279B01AC010F94422020E030E040E8E8
:1011C0005FE30F94A0260F944E2920E030E048E41E
:1011D00052E40F94422068A379A38AA39BA320E042
:1011E00030E040EC5FE3C301B2010F94422090581D
:1011F00069837A838B839C8320E030E040EC5FE35B
:10120000C501B4010F94422090586C8F7D8F8E8F52
:101210009F8FAE01405E5F4FBE016F5F7F4FCE017B
:101220004C960E94B15F0E9429521092190C1092A4
:101230001A0C10921B0C10921C0C10921D0C109288
:101240001E0C10921F0C1092200C80E00E94B860BF
:10125000002319F081E00E94B860FF2009F47DC0EE
:1012600083E00E94F84A811178C00E94E62920910B
:10127000F7073091F8074091F9075091FA0760E0BD
:1012800070E086E193E40F949F262B013C012091AE
:10129000FB073091FC074091FD075091FE0760E08D
:1012A00070E086E193E40F949F264B015C018091EE
:1012B000210C9091220CA091230CB091240C8093CE
:1012C000700790937107A0937207B0937307009112
:1012D0002A1210912B12D8012D913D914D915C91C4
:1012E000C301B2010F949F2660936807709369074A
:1012F00080936A0790936B07F801248135814681BA
:101300005781C501B4010F949F2660936C077093B9
:101310006D0780936E0790936F0788E697E00E94B1
:10132000A71D8823A9F11C8E1D8E1E8E1F8E88E09E
:10133000E8E6F7E0DE01119601900D928A95E1F75B
:10134000AE01445E5F4FBE016B5F7F4FCE010196E1
:101350000E94B15F82E00E94B8600E94E6298091FD
:10136000990680939A068E2D0E94DF630E94641C6A
:101370000E94802F24CE012F10E0C9CE60E070E0E3
:1013800080E890E4CCCEA3019201C501B4010FCF57
:1013900060E081EF9EE00E94833C0E94E84A8FED6E
:1013A0009EE00E943D35D9CF14E00E941BA36093BC
:1013B00068117093691180936A1190936B118091F9
:1013C0002A0C811127C08EE40E94E81D882321F099
:1013D00082E09FE00E946E9B87E00E94F84A8111A4
:1013E0001FC00E94427A8823D9F0115001F130E0E9
:1013F00020E042E557E16DE27FE085E00E94283D74
:1014000061E080E29FE00E94503C88E09FE00E9403
:101410006E9BCBCF60E08FE40E941424882399F266
:101420000E94003D8BEC9FE00E946E9BC8CD61E066
:101430008EEB9FE00E94503C89E49FE00E946E9BEF
:1014400061E08DE397E10E94503C40E070E060E095
:101450008AE39FE00E946C5100912A1210912B1296
:10146000D8012D913D914D915C916091190C709135
:101470001A0C80911B0C90911C0C0F94A026AB01B0
:10148000BC0188E50E94662469837A838B839C83F0
:10149000F801248135814681578160911D0C70913E
:1014A0001E0C80911F0C9091200C0F94A026AB0174
:1014B000BC0189E50E9466246D837E838F839887B3
:1014C000BE016B5F7F4FCE0101960E94202D8823C5
:1014D00009F475CD80E00E94DF630E947D1C61E00D
:1014E00085E40E941424182F21E0482FBE016B5F71
:1014F0007F4FCE0101960F941C116B017C01AC0152
:101500009B010F949229811119C049815A816B81E5
:101510007C818DEE9FE00E94F13D4D815E816F8167
:10152000788588EE9FE00E94F13DB701A60183EE29
:101530009FE00E94F13D8AE00E9404350E94641CF5
:1015400011110E9459620E94802F39CD8091DD06D1
:10155000813009F034CD89E40E94361E082FF12C29
:10156000882319F00E942924F82E8AE40E94361E4E
:10157000E82E882379F00E942924182F002309F4EB
:10158000C0C0F4E0FF1508F0B9C085EF9FE00E94ED
:101590003D3515CD10E00111F4CF80E1E9E1FCE02B
:1015A000A8E6B7E001900D928A95E1F7002319F1C2
:1015B0006F2DFF0C770B880B990B0F94E31F209175
:1015C000CB053091CC054091CD055091CE050F94BF
:1015D00042202091C3053091C4054091C50550912A
:1015E000C6050F94A02660936807709369078093DF
:1015F0006A0790936B07EE2019F1612F110F770B9B
:10160000880B990B0F94E31F2091CF053091D005E3
:101610004091D1055091D2050F9442202091C705E9
:101620003091C8054091C9055091CA050F94A02674
:1016300060936C0770936D0780936E0790936F07AC
:1016400060E080E50E9414248823C1F10023D1F0DA
:10165000E0912A12F0912B12208131814281538135
:10166000609168077091690780916A0790916B0794
:101670000F949F26609368077093690780936A07A9
:1016800090936B07EE20D1F0E0912A12F0912B128B
:10169000248135814681578160916C0770916D0777
:1016A00080916E0790916F070F949F2660936C074F
:1016B00070936D0780936E0790936F0740E050E042
:1016C000BA0186E40E9466246B017C0120E030E0D0
:1016D000A9010F9400291816C4F420E030E040E777
:1016E00052E4C701B6010F949A2769837A838B83EA
:1016F0009C83CE0101960E94D76C61CCEE2009F448
:101700004CCF153008F449CF40CF60E070E0CB01FA
:10171000ECCF8FE08093E50752CC80912805882399
:1017200081F1893009F04BCC1CEDA12E12E0B12ED5
:1017300009E1C02E0CE0D02EE12C00E010E0D50134
:101740008D915D010E94361EF82E882361F01330C2
:1017500011F4082FFE2C0E943C24F6016083718353
:1017600082839383EF2C1F5FF4E0CF0ED11C1430E3
:1017700031F7EE2009F457C00E94E6290E94802F1D
:101780001ECCBCEDCB2EB2E0DB2EF12CE12C00E028
:1017900010E0D6018D916D010E94361E382E8823EF
:1017A000D9F10E943C244B015C01133059F0F70140
:1017B000EF53F74F20813181428153810F949F264F
:1017C0004B015C01F701E75EF34F208131814281DB
:1017D0005381C501B4010F949F262B013C012DEBD1
:1017E00037E346E855EB0F94002987FD0AC02DEB3F
:1017F00037E346E855E3C301B2010F94DC1F181626
:101800005CF41330C1F48092250C9092260CA092C7
:10181000270CB092280C032D1F5FB4E0EB0EF11CD7
:10182000143009F0B6CF002309F4A8CF85E29CE07C
:101830000E94C05DA3CFF701E551F84F5F01A301FE
:10184000920160817181828193810F94A026D501DC
:101850006D937D938D939C931397812F0E94441CCD
:10186000DBCF8091290590912A058837910511F4E5
:101870000C94AD9508F067C28D34910509F4D9C672
:1018800008F0EFC08A31910509F40EC608F092C045
:101890008431910509F454C508F06FC08131910578
:1018A00009F415C508F042C0029708F071CB80E535
:1018B0000E94361EC12CD12C7601882321F00E9473
:1018C000B6236B017C0183E50E94361E882361F0FC
:1018D0000E943C2420E030E04AE754E40F94422088
:1018E0000F9413286B017C010E94AF5D809130053D
:1018F00090913105892B09F4E5C40F94ED10809186
:10190000290590912A0566E170E1892B11F46EE0BA
:1019100070E130E020E04EE150E182E00E94283D9D
:1019200040E0C701B6010E944E8349CB429709F0BF
:101930002FCB83E50E94361E882311F40C94E59486
:101940000E941BA3609368117093691180936A11C0
:1019500090936B110E943C2420E030E04AE754E46D
:101960000F9442200F941328609314027093150271
:10197000809316029093170222CB8731910509F4C8
:1019800014C570F48531910509F40BC5469709F02B
:10199000FFCA8091D71382FD12CB0E9442AF0FCBBA
:1019A0008831910509F416C5499709F0F1CA0E94DA
:1019B0003D8505CB8032910509F4FAC5C0F58D311E
:1019C000910509F4DEC570F48B31910509F47FC5EA
:1019D0004C9709F0DDCA80913005909131050E9445
:1019E00034B4EDCA8E31910509F4D2C54F9709F090
:1019F000CFCA0E94642A6C8F7D8F8E8F9F8FBE010D
:101A00006F5F7F4FCE014C960E94F220CE0101966F
:101A10000E949CF10E94E84ABE016F5F7F4F82E9FD
:101A200090E10E945A538AE00E940435C8CA893462
:101A3000910509F4EAC550F48132910509F4E1C534
:101A4000C09709F0A5CA0E942D64B9CA8B349105CC
:101A500009F4EBC58C34910509F09ACA0E94153639
:101A6000AECA8B36910509F4C3C608F0F9C08435B7
:101A7000910509F45ECF30F58135910509F485C7EC
:101A800090F48E34910509F083CA70E060E083E53C
:101A90000E942D248E34910509F0D0C50E943D513D
:101AA0000E94D4F18CCA8235910509F486C783352A
:101AB000910509F06DCA8091E5078F7E8062809361
:101AC000E5077DCA8836910509F43CC608F099C03F
:101AD0008535910509F4BCC78C35910509F058CAC4
:101AE0000E94E74B87FD6BCA80912C0584FD09C0DD
:101AF00080912E0587FD05C080912F05837009F424
:101B0000D4C7ECEDCE2EE2E0DE2EFBE2EF2EFCE0C1
:101B1000FF2E10E0D6018D916D010E94361E8823A4
:101B200009F465C0133009F0B8C70E943C244B018A
:101B30005C0120E030E040EA51E40F94DC1F87FFB5
:101B40004EC0A501940160914B0C70914C0C80919A
:101B50004D0C90914E0C0F949A272B013C01AC0137
:101B60009B016091DA087091DB088091DC0890910C
:101B7000DD080F9442206093DA087093DB088093AD
:101B8000DC089093DD08A301920160915B0C7091D9
:101B90005C0C80915D0C90915E0C0F9442206093E0
:101BA0005B0C70935C0C80935D0C90935E0C609169
:101BB000EA087091EB088091EC089091ED080F9481
:101BC000E11FA30192010F9442200F941328609308
:101BD000EA087093EB088093EC089093ED088092EC
:101BE0004B0C90924C0CA0924D0CB0924E0C1F5F7F
:101BF000F4E0EF0EF11C143009F08CCF0E94CE25DA
:101C0000DEC98936910509F4C8C58A36910509F0FF
